:100000000C9437180C9470180C9470180C94701889
:100010000C9425890C9425890C9425890C942589A8
:100020000C9470180C9470180C9470180C94701830
:100030000C9470180C946F700C9470180C947018C9
:100040000C9470180C94856E0C949FCB0C947018C3
:100050000C9468400C945E400C9470180C947018CA
:100060000C9470180C9470180C9470180C947018F0
:100070000C9470180C9470180C9470180C947018E0
:100080000C94DE320C9470180C94701805A84CCDAA
:10009000B2D44EB93836A9020C50B9918688083CC2
:1000A000A6AAAA2ABE000000803F4E414E494E49F2
:1000B0005459494E46CDCCCC3D0AD7233C17B7D135
:1000C0003877CC2B329595E6241FB14F0A000020DB
:1000D000410000C84200401C4620BCBE4CCA1B0E5A
:1000E0005AAEC59D7400407A10F35A00A0724E18A3
:1000F000090010A5D4E80000E87648170000E40BDA
:1001000054020000CA9A3B000000E1F5050000809F
:10011000969800000040420F000000A086010000F9
:1001200000102700000000E8030000000064000049
:100130000000000A00000000000100000000002C88
:1001400076D888DC674F0823DFC1DFAE59E1B1B74D
:1001500096E5E3E453C63AE651997696E8E6C2841A
:1001600026EB898C9B62ED407C6FFCEFBC9C9F4032
:10017000F2BAA56FA5F490055A2AF75C936B6CF957
:10018000676DC11BFCE0E40D47FEF520E6B500D02D
:10019000ED902E0300943577050080841E08000042
:1001A000204E0A000000C80C333333330F986E1210
:1001B000831141EF8D2114893BE65516CFFEE6DB16
:1001C00018D1844B381BF77C1D901DA4BBE4242060
:1001D0003284725E228100C9F124ECA1E53D2743FF
:1001E0004F4D4D554E49434154494F4E004452598D
:1001F00052554E004552524F525300494E464F0001
:100200004543484F0053544F505045442E20005012
:1002100072696E7465722073746F707065642064A7
:10022000756520746F206572726F72732E20466937
:100230007820746865206572726F7220616E642028
:10024000757365204D39393920746F207265737468
:100250006172742E202854656D70657261747572B8
:10026000652069732072657365742E205365742050
:10027000697420616674657220726573746172744A
:10028000696E67290A004E6F20436865636B73755A
:100290006D2077697468206C696E65206E756D627B
:1002A00065722C204C617374204C696E653A200095
:1002B0004E6F20436865636B73756D207769746852
:1002C000206C696E65206E756D6265722C204C61C4
:1002D0007374204C696E653A2000636865636B73C4
:1002E000756D206D69736D617463682C204C61734A
:1002F00074204C696E653A20004C696E65204E751D
:100300006D626572206973206E6F74204C61737426
:10031000204C696E65204E756D6265722B312C2004
:100320004C617374204C696E653A20004D31313058
:100330000053657269616C20737461747573206D0C
:1003400069736D617463680A005344207265616467
:10035000206572726F720A002121204B494C4C209B
:1003600063617573656420627920746F6F206D75A9
:10037000636820696E6163746976652074696D6570
:10038000202D2063757272656E7420636F6D6D61D0
:100390006E643A20004D6564696120496E73657230
:1003A00074656400627573793A2070617573656471
:1003B00020666F7220696E7075740A0062757379B9
:1003C0003A2070617573656420666F72207573657D
:1003D000720A00627573793A2070726F6365737385
:1003E000696E670A00506C656173652052657365BC
:1003F00074005052494E5445522048414C54454493
:100400000025533A202553004B494C4C45442E209F
:10041000005072696E7465722068616C7465642E38
:10042000206B696C6C28292063616C6C6564210AFF
:10043000006563686F3A004572726F723A004F460A
:1004400046004F4E0042696C696E656172204C65D2
:1004500076656C696E6720477269643A0A004F4698
:10046000460A004661646520486569676874200033
:10047000426564204C6576656C696E672000466154
:10048000696C656420746F20656E61626C652042E2
:100490006564204C6576656C696E670A00496E7606
:1004A000616C6964206D6573682E0A0050726F621A
:1004B000696E6720506F696E740025532025692F7F
:1004C0002569002E0A002F0050726F62696E672046
:1004D0006D65736820706F696E7420002028445227
:1004E0005952554E2900473239204175746F2042C8
:1004F0006564204C6576656C696E67003F20284C0A
:100500002C522C462C4229206F7574206F66206275
:100510006F756E64732E0A003F2856296572626FEC
:100520007365206C6576656C20696D706C617573A0
:1005300069626C652028302D34292E0A00426164DE
:10054000205A2076616C75650A004E6F2062696CD6
:10055000696E65617220677269640A004732384CBF
:100560003000446576696174696F6E0025533A20E6
:1005700025730046696E6973686564210A003A2034
:100580007A3A2000206F662000476F696E672074FA
:100590006F3A20580043570A00206469723A0020DD
:1005A000616E676C653A00537461727420726164A5
:1005B0006975733A004D343820506F696E740025A8
:1005C000533A2025642F256400506F736974696F56
:1005D0006E696E67207468652070726F62652E2E7A
:1005E0002E0A003F4C656773206F66206D6F76653D
:1005F0006D656E7420696D706C61757369626C6590
:100600002028302D3135292E0A003F2028582C591A
:1006100029206F7574206F6620626F756E64732E6B
:100620000A0050726F6265206F7574206F662062D9
:100630006F756E6473003F53616D706C65207369F4
:100640007A65206E6F7420706C61757369626C6579
:100650002028342D3530292E0A004D3438205A2DCB
:1006600050726F6265205265706561746162696C79
:1006700069747920546573740A003F28562965729D
:10068000626F7365206C6576656C20696D706C6156
:10069000757369626C652028302D34292E0A005349
:1006A00074616E6461726420446576696174696F17
:1006B0006E3A20002052616E67653A2000204D613D
:1006C000783A2000204D696E3A2000205369676D0A
:1006D000613A20004D65616E3A200020204D323095
:1006E000312058004D617820416363656C6572610B
:1006F00074696F6E2028756E6974732F73322900C8
:1007000020204D3230332058004D617820666565D9
:100710006472617465732028756E6974732F732910
:100720000020520020204D323034205000416363BD
:10073000656C65726174696F6E2028756E6974737B
:100740002F7332292028503C7072696E742D6163BA
:1007500063656C3E20523C726574726163742D61F6
:100760006363656C3E20543C74726176656C2D61E8
:100770006363656C3E2900204A002054002053002A
:1007800020204D323035204200416476616E636531
:10079000642028423C6D696E5F7365676D656E7499
:1007A0005F74696D655F75733E20533C6D696E5F64
:1007B00066656564726174653E20543C6D696E5F68
:1007C00074726176656C5F66656564726174653EBE
:1007D000204A3C6A756E635F6465763E2900205549
:1007E00000204C0020204D323831205000536572DB
:1007F000766F20416E676C657300204400204900CD
:1008000020204D333031205000486F74656E6420D5
:10081000504944002E0A00206E6F74206469736191
:10082000626C65642E205368617265642077697418
:10083000680020496E76616C696420657874727511
:100840006465722000536C6565702E2E2E005A2050
:1008500050726F62652050617374204265640A00B3
:100860005A2050726F626520506173742042656433
:1008700000205A3A200020593A200042656420584E
:100880003A20004D65736820706F696E74206F7533
:1008900074206F662072616E67650A00436C69633D
:1008A0006B20746F20526573756D652E2E2E00615E
:1008B0006C736F20656E61626C6564290A004E6F0F
:1008C000204D6F76652E004E6F206D656469610A5C
:1008D00000456E642066696C65206C6973740A005B
:1008E000426567696E2066696C65206C6973740A7D
:1008F00000286E6F2066696C6529004E6F74205366
:1009000044207072696E74696E670A0053442070E7
:1009100072696E74696E6720627974652000437530
:100920007272656E742066696C653A20002E0A004A
:1009300044656C6574696F6E206661696C65642CD2
:100940002046696C653A200046696C652064656CD8
:10095000657465643A002569730025696D20256911
:1009600073002569682025696D2025697300256954
:1009700064202569682025696D2025697300256933
:100980007920256964202569682025696D202569FD
:1009900073005072696E742074696D653A20006F3F
:1009A0006B006F6666000002FB01F401ED01DF01E0
:1009B00044454255473A004D3131322053687574F1
:1009C000646F776E004D3131332053004D656761A0
:1009D000205A65726F204F46462E00434F4E4649BF
:1009E000475F4558504F5254004D45415450414384
:1009F0004B00434F4F4C45525F54454D504552417B
:100A000054555245004348414D4245525F54454D6F
:100A10005045524154555245004241425953544564
:100A20005050494E470041524353004D4F54494F97
:100A30004E5F4D4F44455300544845524D414C5F25
:100A400050524F54454354494F4E00455854454E1B
:100A50004445445F4D3230004C4F4E475F46494C51
:100A6000454E414D45004155544F5245504F52540B
:100A70005F53445F5354415455530053445F57529E
:100A80004954450052455045415400534443415256
:100A9000440050524F4D50545F535550504F525494
:100AA00000484F53545F414354494F4E5F434F4DAD
:100AB0004D414E445300454D455247454E43595FC5
:100AC00050415253455200434153455F4C494748BA
:100AD000545F4252494748544E45535300544F4780
:100AE000474C455F4C494748545300534F46545771
:100AF0004152455F504F574552004255494C445F63
:100B000050455243454E54004C4556454C494E477E
:100B10005F44415441005A5F50524F424500525584
:100B20004E4F5554004155544F4C4556454C00507E
:100B300052494E545F4A4F420050524F475245531C
:100B400053004155544F5245504F52545F54454DF8
:100B500050004155544F5245504F52545F504F53DF
:100B600000564F4C554D455452494300454550524F
:100B70004F4D0042494E4152595F46494C455F54E2
:100B800052414E534645520053455249414C5F58DD
:100B90004F4E5F584F4646004649524D57415245C9
:100BA0005F4E414D453A4D61726C696E20322E3078
:100BB0002E392E332D6B6164312028446563203239
:100BC0003720323032312031333A35303A30322921
:100BD00020534F555243455F434F44455F55524C58
:100BE0003A6769746875622E636F6D2F6B61642F4D
:100BF0004D61726C696E2050524F544F434F4C5FA1
:100C000056455253494F4E3A312E30204D414348BC
:100C1000494E455F545950453A4D656761205A65C4
:100C2000726F2045585452554445525F434F554EBC
:100C3000543A3120555549443A64626663636435D9
:100C4000352D656262612D343631352D6162643730
:100C50002D3139366161343338663330340A002F30
:100C60002F004D31343520533C696E6465783E2049
:100C70006F7574206F662072616E67652028302D55
:100C800031290A003F4A206F7574206F6620726117
:100C90006E67652028302E303120746F20302E335F
:100CA000290A0020580020204D61783A20002000B9
:100CB00020204D696E3A2000203B200020204D323C
:100CC0003131205300536F667420656E6473746F06
:100CD00070730046523A0020466C6F773A2000202D
:100CE0006F7574206F662072616E67650A005365C8
:100CF00072766F20003A200020536572766F2000D4
:100D0000206F7574206F662072616E67650A0053EC
:100D10006572766F2000206F7574206F6620726197
:100D20006E67650A00536572766F200050726F62BD
:100D300065204F6666736574205A0050726F626555
:100D4000204F6666736574205A0064697300656E8F
:100D50000043290A0061626C656420286D696E2079
:100D600074656D702000436F6C64206578747275D3
:100D70006465732061726520004D34323120696EE4
:100D8000636F727265637420706172616D65746502
:100D9000722075736167650A004D65736820706F16
:100DA000696E74206F7574206F662072616E67655E
:100DB0000A00454550524F4D204F4B0A00290A006A
:100DC00020746F20003F5A206F7574206F66207268
:100DD000616E6765202800290A0020746F20003F9B
:100DE00059206F7574206F662072616E67652028C8
:100DF0002D00290A0020746F20003F58206F757461
:100E0000206F662072616E676520282D004D383492
:100E100000446F6E65207072696E74696E6720663B
:100E2000696C650A004D3737004D333100496E76E5
:100E3000616C69642065787472756465720A004338
:100E400061703A00203B0020204D38353120580099
:100E50005A2D50726F6265204F6666736574004349
:100E60006F6F6C696E672E2E2E0048656174696E17
:100E7000672E2E2E0045312025530020573A00239F
:100E8000646566696E652044454641554C545F0073
:100E90004B6420004B6920004B70200050494420D7
:100EA0004175746F74756E652066696E69736865E7
:100EB00064212050757420746865206C61737420FF
:100EC0004B702C204B6920616E64204B6420636F53
:100ED0006E7374616E74732066726F6D2062656CE0
:100EE0006F7720696E746F20436F6E6669677572E5
:100EF0006174696F6E2E680A005049442041757410
:100F00006F74756E65206661696C65642120746913
:100F10006D656F75740A00504944204175746F7493
:100F2000756E65206661696C6564212054656D701D
:100F30006572617475726520746F6F206869676887
:100F40000A00504944204379636C6573002553209F
:100F500025692F256900204B643A2000204B693A0F
:100F60002000204B703A200020436C61737369634A
:100F700020504944200A002054753A2000204B7527
:100F80003A2000206D61783A2000206D696E3A2089
:100F90000020643A200020626961733A20005761A2
:100FA000697420666F7220686561742075702E2EDA
:100FB0002E00504944204175746F74756E6520731E
:100FC000746172740A00504944204175746F7475DD
:100FD0006E65206661696C6564212054656D70657D
:100FE00072617475726520746F6F20686967680A32
:100FF00000504944204175746F74756E65206661B8
:10100000696C656421204261642068656174657261
:101010002069640A00504944204175746F74756EEC
:1010200065004572723A207574663820666F6E747A
:10103000206E6F7420696E697469616C697A656489
:101040002E004572723A207574663820666F6E7491
:10105000206E6F7420696E697469616C697A656469
:101060002E004572723A207574663820666F6E7471
:10107000206E6F7420696E697469616C697A656449
:101080002E002568753A25303268750025303268A3
:10109000753A25303268750025303268752725305D
:1010A00032687500256875642025303268753A25E8
:1010B000303268750042656400456E636C6F73750D
:1010C00072650020202020202020002020202000E9
:1010D000453A00523A00657272001FE0201020105D
:1010E00020101020102020102010303008400480E4
:1010F00003001FE03FF03FF03FF01FE01FE03FF034
:101100003FF03FF00FC0078003003FFFF038007052
:1011100030FC3020FC102078102030102C00D02E15
:1011200031D02F7BD02F7BD02E31D02C00D020304F
:101130001020781020FC1030FC303800703FFFF099
:101140003FFFF03800703186302387102787902FBB
:1011500087D02F03D0203010207810207810203036
:10116000102F03D02F87D027879023871031863008
:101170003800703FFFF0001DC43F0000000C8619CE
:101180008000000D0E198000000F0B198000000D6B
:101190009F198000000DD3998000001CFBFF000008
:1011A000000000000000000000000000F380001FAD
:1011B00080007700001980005B1CF6131DAE5B35C4
:1011C000AB0635FB5B3DA70CBD9B4B30EB19B19BD0
:1011D000E39D8E9F9D8E0001E00000000001200035
:1011E00000000001E0000000000C0F00FE070225D7
:1011F00003BB017FFE08FE08FE050808060000404C
:10120000F0C88888987810050808060000C0F8889B
:1012100088888888F80505050600012030F8302008
:101220000508080600002070F820202020E00509AD
:10123000090600FF2070A8A8B88888702007050557
:10124000070001D86C366CD80509090600FFF8A81C
:101250008888888888A8F8050A0A0600FE20505069
:10126000505088A8A8887003030306000340A040DC
:10127000FFFFFFFFFFFFFFFFFFFFFFFFFFFFFFFF7E
:10128000FFFFFFFFFFFF0000000605FF0107070645
:10129000020080808080800080030303060105A097
:1012A000A0A005060606000050F85050F8500509A9
:1012B000090600FF2070A8A07028A8702005070765
:1012C000060000C8C81020409898050707060000CF
:1012D00040A0A040A890680103030602058080801A
:1012E0000309090601FF2040408080804040200320
:1012F00009090601FF80404020202040408005076A
:101300000706000020A8702070A82005050506002B
:10131000012020F820200203030601FFC0408005C1
:101320000101060003F8020202060100C0C0050721
:10133000070600000810102040408005070706003F
:1013400000708898A8C8887003070706010040C08D
:1013500040404040E0050707060000708808102064
:1013600040F8050707060000F808103008887005E7
:10137000070706000010305090F810100507070608
:101380000000F880F00808887005070706000030A4
:101390004080F0888870050707060000F8081010E4
:1013A0002020200507070600007088887088887054
:1013B0000507070600007088887808106002050598
:1013C000060100C0C000C0C00206060601FFC0C082
:1013D00000C0408003050506010120408040200533
:1013E0000303060002F800F803050506010180402A
:1013F000204080050707060000708810202000208C
:101400000507070600007088B8A8B88070050707B0
:10141000060000708888F88888880507070600009D
:10142000F04848704848F0050707060000708880BB
:1014300080808870050707060000F0484848484843
:10144000F0050707060000F88080F08080F80507A7
:1014500007060000F88080F08080800507070600FE
:1014600000708880809888700507070600008888CB
:1014700088F8888888030707060100E0404040405C
:1014800040E00507070600003810101010906005B6
:1014900007070600008890A0C0A0908805070706EF
:1014A0000000808080808080F805070706000088A3
:1014B000D8A8888888880507070600008888C8A8F3
:1014C00098888805070706000070888888888870D3
:1014D000050707060000F08888F080808005070770
:1014E00006000070888888A8906805070706000035
:1014F000F08888F0A09088050707060000708880B3
:1015000070088870050707060000F82020202020BA
:1015100020050707060000888888888888700507E6
:1015200007060000888888885050200507070600B5
:101530000088888888A8A8500507070600008888C2
:101540005020508888050707060000888850202012
:101550002020050707060000F80810204080F80347
:1015600009090601FFE080808080808080E0050717
:1015700007060000804040201010080309090601FA
:10158000FFE020202020202020E0050303060005A6
:101590002050880501010600FEF80303030601053B
:1015A000804020050505060000700878887805074A
:1015B000070600008080F0888888F0050505060091
:1015C000007080808870050707060000080878888A
:1015D0008888780505050600007088F0807005078A
:1015E00007060000304840E040404005070706007D
:1015F000FE708888887808700507070600008080DC
:10160000F0888888880307070601004000C0404032
:1016100040E00409090601FE10003010101010907F
:101620006005070706000080808890E09088030727
:1016300007060100C04040404040E00505050600A7
:1016400000D0A8A8A8A8050505060000B0C888888D
:10165000880505050600007088888870050707065C
:1016600000FEF0888888F080800507070600FE7875
:10167000888888780808050505060000B0C88080BD
:101680008005050506000078807008F0050707064C
:1016900000002020F82020201805050506000088FD
:1016A0008888986805050506000088888850200508
:1016B00005050600008888A8A85005050506000055
:1016C00088502050880507070600FE88888850202B
:1016D0004080050505060000F8102040F8030909C0
:1016E0000601FF204040408040404020010909069B
:1016F00002FF80808080808080808003090906014D
:10170000FF80404040204040408005030306000227
:1017100048A890FF5045544700504C410050726912
:101720006E742041626F72746564004D32350050F2
:10173000617573696E672E2E2E004D32340045455B
:1017400050524F4D2056657273696F6E204572720C
:101750006F7200454550524F4D20496E64657820A8
:101760004572726F7200454550524F4D20435243AF
:10177000204572726F72003F0049676E6F7265009C
:10178000526573657400496E697469616C697A6544
:1017900020454550524F4D0000FE0003FF8007C713
:1017A000C00701E00000E00000F0000070040070DD
:1017B0000E00701F00703F80F00E00E00F01E00788
:1017C000C7C003FF8000FE0000FE0003FF8007C7C4
:1017D000C00F01E00E00E03F80F01F00700E0070AF
:1017E0000400700000700000F00000E00701E00756
:1017F000C7C003FF8000FE000E000E000E000E00AA
:101800000E000E000E000E007FC03F801F000E0075
:10181000040004000E001F003F807FC00E000E0079
:101820000E000E000E000E000E000E00FFFFFF7FE8
:1018300080FFC0FFC0FFC07F807F80FFC0FFC0FF70
:10184000C03F001E000C0050726F6265205A204F8E
:101850006666736574002008204661637400200882
:10186000204D6178002008204D696E004F666600AB
:101870004F6E004175746F74656D70004520737410
:101880006570732F6D6D005A2053746570732F6DE2
:101890006D00592053746570732F6D6D005820537F
:1018A000746570732F6D6D00416476616E6365645D
:1018B0002053657474696E67730054656D7065724A
:1018C00061747572650053746570732F6D6D00439C
:1018D0006F6E66696775726174696F6E003F004E66
:1018E00065787420436F726E657200446F6E650098
:1018F0004E65787400486F6D696E672058595A00BC
:1019000053746F72652053657474696E6773004C0D
:101910006F61642053657474696E67730042656417
:10192000205472616D6D696E670050726F62652040
:101930005A204F6666736574004661646520486589
:1019400069676874004F6666004F6E0042656420E8
:101950004C6576656C696E67004C6576656C2042F7
:101960006564004732394E00473239004175746F63
:1019700020486F6D65004D6F74696F6E005265731E
:10198000746F72652044656661756C7473004C6F8A
:1019900061642053657474696E67730053746F7269
:1019A000652053657474696E67730050726F626569
:1019B000205A204F666673657400416476616E63D9
:1019C00065642053657474696E6773004D61696E58
:1019D000003F004261636B0053746F70004D323200
:1019E00000417474616368204D65646961004D3223
:1019F00031005072696E742066726F6D204D65649F
:101A000069610052656C65617365204D656469614B
:101A100000436F6E66696775726174696F6E00541A
:101A2000656D7065726174757265004D6F74696F74
:101A30006E00526573756D65205072696E74005446
:101A4000756E650053746F70205072696E7400502B
:101A500061757365205072696E7400496E666F20FF
:101A600053637265656E000A4D3234004D32332087
:101A70002573003F005374617274205072696E7454
:101A80000043616E63656C005072696E740043615F
:101A90006E6E6F7420656E74657220737562646912
:101AA000723A200002202E2E000152656672657384
:101AB00068004D61696E002100486F74656E642096
:101AC000746F6F20636F6C64004261636B005072CF
:101AD0006F63656564004D6F74696F6E0044697370
:101AE00061626C65205374657070657273004D3867
:101AF00034004D34382050726F6265205465737421
:101B0000004732384F0A4D3438205031300042659A
:101B100064204C6576656C696E67004175746F2052
:101B2000486F6D6500473238004D61696E001917C6
:101B30001417436F6F6C646F776E00507265686541
:101B4000617420240046616E205370656564004E08
:101B50006F7A7A6C65004D61696E0050726F6265D4
:101B6000205A204F666673657400466C6F77004696
:101B7000616E205370656564004E6F7A7A6C650003
:101B80005370656564004D61696E00486F6D696EE4
:101B900067204661696C6564006F70656E00545221
:101BA00049474745524544003A20007A5F6D696EC7
:101BB00000795F6D696E00785F6D696E00526570C7
:101BC0006F7274696E6720656E6473746F702073D2
:101BD00074617475730A0020746F6F206C6F6E6788
:101BE00020657874727573696F6E207072657665A2
:101BF0006E7465640A0020636F6C6420657874728B
:101C00007573696F6E2070726576656E7465640AAF
:101C100000486F6D65202573257325732046697212
:101C20007374005761726E696E673A20486F6D6910
:101C30006E672042756D702044697669736F7220FB
:101C40003C20310A000202040000E0C0000000C095
:101C500000000000000068430000634300007A4376
:101C60000000A0400000A04000000040FFFDFCFA82
:101C7000F8F6F4F2F0EEECEAE9E7E5E3E1E0DEDCC9
:101C8000DAD9D7D5D4D2D0CFCDCBCAC8C7C5C3C275
:101C9000C0BFBDBCBAB9B7B6B4B3B2B0AFADACAAF1
:101CA000A9A8A6A5A4A2A1A09E9D9C9A9998979543
:101CB000949392908F8E8D8B8A8988878684838275
:101CC00081807F7E7D7B7A79787776757473727187
:101CD000706F6E6D6C6B6A6968676665646362617C
:101CE000605F5E5D5C5B5A59585857565554535265
:101CF0005150504F4E4D4C4B4A4A49484746464535
:101D00004443424241403F3E3E3D3C3B3B3A3938F2
:101D10003837363535343332323130302F2E2E2DA0
:101D20002C2B2B2A29292827272625252423232243
:101D3000212120201F1E1E1D1C1C1B1B1A191918D7
:101D400018171616151514131312121111100F0F60
:101D50000E0E0D0D0C0C0B0A0A09090808070706E0
:101D6000060505040403030202010000000000014F
:101D700000000001000080005555550000004000A3
:101D800033333300AAAA2A0049922400000020001D
:101D9000C7711C0099991900D145170055551500B8
:101DA0003BB1130024491200111111000000100072
:101DB0000F0F0F00E3380E0043790D00CCCC0C0060
:101DC000C3300C00E8A20B0064210B00AAAA0A0091
:101DD000703D0A009DD80900427B09009224090049
:101DE000DCD30800888808001042080000000800C2
:101DF000F0C107008787070075500700711C0700B6
:101E00003EEB0600A1BC060069900600666606006F
:101E1000703E06006118060017F4050074D1050035
:101E20005BB00500B29005006272050055550500D3
:101E300078390500B81E0500050505004EEC0400C4
:101E400087D40400A1BD040090A7040049920400B7
:101E5000C17D0400EE690400C75604004444040038
:101E60005C3204000821040041100400000004005A
:101E70003FF00300F8E0030026D20300C3C30300D1
:101E8000CCB503003AA803000A9B0300388E030078
:101E9000C08103009F750300D0690300505E0300FA
:101EA0001D53030034480300913D03003333030006
:101EB00016290300381F030097150300300C030098
:101EC000030303000BFA020049F10200BAE8020022
:101ED0005CE002002DD802002DD0020059C802009B
:101EE000B0C0020031B90200DAB10200AAAA0200B1
:101EF000A0A30200BC9C0200FA9502005C8F0200C5
:101F0000DF88020082820200457C02002776020000
:101F100027700200436A02007C640200D05E020067
:101F20003F590200C85302000000614300006143B2
:101F300000007A430000E0C0000000C00000000084
:101F400053657474696E67732053746F72656400AF
:101F5000290A002062797465733B20637263200054
:101F600053657474696E67732053746F726564206F
:101F70002800454550524F4D206461746173697A61
:101F800065206572726F722E0A00290A002062793C
:101F90007465733B2063726320002073746F7265F5
:101FA000642073657474696E6773207265747269F6
:101FB00065766564202800202863616C63756C6118
:101FC00074656429210A0020213D200045455052B6
:101FD0004F4D20435243206D69736D6174636820D7
:101FE0002D202873746F7265642920002053697A4C
:101FF000653A2000496E6465783A2000204D617290
:102000006C696E3D563836290A00454550524F4D91
:102010002076657273696F6E206D69736D6174638C
:10202000682028454550524F4D3D00486172646319
:102030006F6465642044656661756C7420536574D3
:1020400074696E6773204C6F616465640A000000F8
:10205000FA430000FA430000A0400000C84100001D
:10206000A0420000A0420000C8430080C043F40129
:102070000000F40100006400000088130000202824
:102080006D6D2900203B204C6576656C696E67207C
:102090000020204D3432302053004175746F2042AF
:1020A0006564204C6576656C696E6700204600208B
:1020B000480020204D3134352053004D6174657245
:1020C00069616C2068656174757020706172616D02
:1020D000657465727300204A00202047323920570A
:1020E00020490020204D3134392043203B20556EBB
:1020F00069747320696E2043656C736975730A0097
:1021000054656D706572617475726520556E697481
:1021100073002020473231203B004C696E656172AC
:1021200020556E6974730024F4D43050C38E20C2DD
:10213000A24017828B7011127A910D816CD90AA876
:1021400061E108C7586607615143061E4B5D05C132
:1021500045A7041A411104093D9803713931034020
:1021600036DB0265339102D4305402802E1D0263A7
:102170002CEE01752AC501B028A001102781018F1E
:102180002564012B244B01E0223401AC211F018D79
:10219000200D01801FFC00841EED00971DDF00B89C
:1021A0001CD200E61BC600201BBC00641AB200B2A1
:1021B00019A8000A19A0006A189900D117910040C7
:1021C000178B00B516840031167E00B31579003ADE
:1021D000157300C7146F0058146A00EE1366008868
:1021E00013630025135E00C7125B006C12570015C5
:1021F000125400C111510070114F0021114B00D633
:102200001049008D1047004610440002104200C0E3
:102210000F4000800F3E00420F3C00060F3B00CBFA
:102220000E3800930E37005C0E3500270E3400F395
:102230000D3200C10D3100900D3000600D2E0032C6
:102240000D2D00050D2C00D90C2B00AE0C2900859E
:102250000C29005C0C2700350C27000E0C2600E82A
:102260000B2400C40B2400A00B23007D0B23005A79
:102270000B2100390B2100180B2000F80A1F00D990
:102280000A1E00BB0A1E009D0A1D00800A1D006375
:102290000A1C00470A1B002C0A1B00110A1A00F72F
:1022A000091A00DD091900C4091900AB09190092C7
:1022B0000917007B091800630917004C091600363E
:1022C000091600200916000A091500F5081500E096
:1022D000081400CC081400B8081400A408140090D6
:1022E0000813007D0812006B0813005808120046FE
:1022F000081200340811002308110012081100010F
:10230000081100F0071000E0071000D0071000C00F
:10231000071000B0070F00A107100091070E0083FF
:10232000070F0074070F0065070E0057070E0049DE
:10233000070E003B070D002E070E0020070D0013AF
:10234000070D0006070D00F9060C00ED060D00E074
:10235000060C00D4060C00C8060C00BC060C00B02D
:10236000060C00A4060B0099060C008D060B0082DB
:10237000060B0077060B006C060B0061060A00577F
:10238000060B004C060A0042060A0038060A002E18
:10239000060A0024060A001A060A001006090007A9
:1023A000060A00FD050900F4050900EB050900E235
:1023B000050900D9050900D0050900C7050900BEB7
:1023C000050900B5050800AD050800A50509009C34
:1023D000050800940508008C050800840508007CA9
:1023E000050800740508006C050700650508005D18
:1023F000050700560508004E050700470507004081
:1024000005080038050700310507002A05070023E5
:102410000507001C050600160507000F0507000844
:1024200005060002050700FB040600F5040700EEA0
:10243000040600E8040600E2040700DB040600D5F9
:10244000040600CF040600C9040600C3040600BD4C
:10245000040600B7040600B1040500AC040600A69B
:10246000040600A00405009B0406009504050090E6
:102470000406008A04050085040500800406007A2D
:1024800004050075040500700405006B0405006672
:10249000040500610405005C0405005704050052B2
:1024A0000405004D04050048040500430405003EF2
:1024B0000404003A04050035040500300404002C2F
:1024C00004050027040400230405001E0404001A68
:1024D00004040016040500110404000D040400099E
:1024E0000405000404040000040400FC030400F8D4
:1024F000030400F4030400F0030400EC030400E808
:10250000030400E4030400E0030400DC030400D837
:10251000030400D4030400D0030400CC030400C867
:10252000030300C503030024F404D9201BC40C5C7E
:102530000E9804C4095F0265077101F405F900FBF8
:1025400004B30048048700C1036900580355000321
:10255000034500BE023A008402310053022A0029DA
:1025600002250004022000E4011C00C8011900AF8C
:10257000011700980114008401130071011000611B
:1025800001100051010E0043010D0036010B002B1C
:10259000010B0020010B00150109000C01090003CB
:1025A000010800FB000800F3000800EB000700E44E
:1025B000000600DE000600D8000600D2000600CCAF
:1025C000000500C7000500C2000500BD000400B9F9
:1025D000000400B5000400B1000400AD000400A92F
:1025E000000400A5000300A20003009F0004009B5C
:1025F0000003009800030095000200930003009080
:102600000003008D0002008B00030088000200869A
:1026100000020084000300810002007F0002007DB0
:102620000002007B000200790002007700010076C2
:102630000002007400020072000100710002006FCD
:102640000002006D0001006C0002006A00010069D8
:1026500000020067000100660001006500010064DF
:102660000002006200010061000100600001005FE3
:102670000002005D0001005C0001005B0001005AE7
:1026800000010059000100580001005700010056E8
:1026900000010055000100540001005300000053E8
:1026A0000001005200010051000100500001004FE4
:1026B0000001004E0000004E0001004D0001004CE2
:1026C0000001004B0000004B0001004A00010049DE
:1026D00000010048000000480001004700010046DA
:1026E00000000046000100450000004500010044D4
:1026F00000010043000000430001004200000042CE
:102700000001004100000041000100400001003FC5
:102710000000003F0001003E0000003E0001003DBF
:102720000000003D0001003C0000003C0000003CB7
:102730000001003B0000003B0001003A0000003AAD
:1027400000010039000000390001003800000038A5
:10275000000000380001003700000037000100369B
:102760000000003600000036000100350000003592
:102770000000003500010034000000340000003487
:10278000000100330000003300000033000100327C
:102790000000003200000032000100310000003172
:1027A0000000003100010030000000300000003067
:1027B0000001002F0000002F0000002F0000002F5C
:1027C0000001002E0000002E0000002E0001002D50
:1027D0000000002D0000002D0000002D0001002C45
:1027E0000000002C0000002C0000002C0001002B39
:1027F0000000002B0000002B0000002B0001002A2D
:102800000000002A0000002A0000002A0001002920
:102810000000002900000029000000290000002914
:102820000001002800000028000000280000002807
:1028300000000028000100270000002700000027FA
:1028400000000027000000270001002600000026ED
:1028500000000026000000260000002600010025E0
:1028600000000025000000250000002500000025D4
:1028700000000025000100240000002400000024C6
:1028800000000024000000240001002300000023B9
:1028900000000023000000230000002300000023AC
:1028A000000000230001002200000022000000229E
:1028B0000000002200000022000000220001002190
:1028C0000000002100000021000000210000002184
:1028D0000000002100000021000100200000002075
:1028E0000000002000000020000000200000002068
:1028F00000000020000000200001001F0000001F59
:102900000000001F0000001F0000001F0000001F4B
:102910000000001F0001001E0000001E0000001E3D
:102920000000001E00000039300000332500008741
:10293000190000B00F0000DB080000BD04000074A7
:102940000200003F01000020436F756E7420583A6A
:102950000045310045002C2073797374656D207338
:10296000746F7070656421204865617465725F4999
:10297000443A200048656174696E67204661696C5D
:1029800065640048656174696E67206661696C659D
:1029900064004572723A204D415854454D50004DE7
:1029A000415854454D50207472696767657265647B
:1029B000004572723A204D494E54454D50004D49E4
:1029C0004E54454D502074726967676572656400A6
:1029D000202F0020403A007C3C3E5E2B3D3F2F5B89
:1029E0005D3B2C2A225C0043616E6E6F74206F7019
:1029F000656E2073756264697220005344206361C0
:102A00007264206F6B0A006F70656E526F6F742076
:102A10006661696C65640A00766F6C756D652E6918
:102A20006E6974206661696C65640A004E6F20539C
:102A30004420636172640A002E0A006F70656E2084
:102A40006661696C65642C2046696C653A200046B5
:102A5000696C652073656C65637465640A00205356
:102A6000697A653A200046696C65206F70656E650D
:102A7000643A2000454E4420535542524F55544924
:102A80004E450A002220706F73002220706172652B
:102A90006E743A2200535542524F5554494E4520C8
:102AA00043414C4C207461726765743A220053753F
:102AB0006263616C6C204F766572666C6F7700455F
:102AC00078636565646564206D6178205355425272
:102AD0004F5554494E452064657074683A006672DB
:102AE00065736800646F696E67002066696C653A9B
:102AF00020004E6F77200057726974696E672074EA
:102B00006F2066696C653A20006D61726C696E6653
:102B1000772E6F726700322E302E392E332D6B6177
:102B20006431001FFFFFFFFFFFFF60000000000196
:102B3000FF400000000000FF8000000000007F83D5
:102B4000CF00000C303F87FF80000C301F8679805B
:102B5000000C000F8C30C7838C30E78C30CFC7CC93
:102B600031F38C30DCECEC33B98C30D86C6C33192D
:102B70008C30D06C0C33198C30D86C0C33198C30F1
:102B8000DC6C0E3B198C30CF7C079F198C30C77CD6
:102B9000038F1940000000000002600000000000E8
:102BA000061FFFFFFFFFFFF870012C0190012701B6
:102BB000B0012201C0011D01F00118011002130132
:102BC00030020E016002090190020401C002FF0000
:102BD0000003FA004003F5008003F000D003EB008F
:102BE0002004E6007004E100E004DC004005D700AA
:102BF000C005D2004006CD00D006C8008007C30043
:102C00003008BE00F008B900C009B400B00AAF0037
:102C1000B00BAA00D00CA500000EA000500F9B0026
:102C2000C01096005012910000148C00C01587004F
:102C3000B0178200B0197D00D01B7800001E730011
:102C400040206E0090226900F024640040275F005D
:102C500090295A00E02B5500102E500020304B00D8
:102C600010324600E033410090353C001037370009
:102C700070383200A0392D00B03A2800A03B230064
:102C8000603C1E00103D1900903D1400103E0F00E6
:102C9000703E0A00C03E0500003F0000403FFBFFC1
:102CA000803FF6FFC03FF1FF2020506C616E6E65E3
:102CB0007242756666657242797465733A200020C7
:102CC00046726565204D656D6F72793A200020432C
:102CD0006F6D70696C65643A2044656320323720FB
:102CE000323032310A00204C6173742055706461B7
:102CF0007465643A20323032312D30392D30332032
:102D00007C20417574686F723A20286B61642C20B6
:102D1000416E796375626963204D656761205A650C
:102D2000726F2041424C20313256290A004D6172A7
:102D30006C696E20322E302E392E332D6B6164314A
:102D40000A0020536F66747761726520526573655F
:102D5000740A00205761746368646F67205265735A
:102D600065740A002042726F776E206F757420526E
:102D7000657365740A002045787465726E616C2015
:102D800052657365740A00506F77657255700A005A
:102D900073746172740A004732385859004D3130EB
:102DA0003031006572726F722077726974696E6774
:102DB00020746F2066696C650A00446F6E6520732D
:102DC0006176696E672066696C652E0A004D32393E
:102DD00000456E6473746F70730025532025632063
:102DE000256320256320256300205A3A0020593AA4
:102DF0000020583A00656E6473746F7073206869C0
:102E0000743A2000000000010200090A00000000DE
:102E1000040308070000000000000000000000009C
:102E200000000000004D6F76652025736D6D004D2C
:102E30006F766520302E316D6D004D6F76652031D7
:102E40006D6D004D6F76652031306D6D004D6F7684
:102E5000652041786973004D6F76652045787472FE
:102E600075646572004D6F7665205A004D6F76650A
:102E70002059004D6F76652058005072696E74209D
:102E800066726F6D204D6564696100FFFFFF205A17
:102E90003A200020593A200042656420583A200028
:102EA0004D656761205A65726F2052656164792EA5
:102EB000005072696E74696E672E2E2E0050726912
:102EC0006E742050617573656400220A00556E6B44
:102ED0006E6F776E20636F6D6D616E643A202200B5
:102EE0006F6B00204500205A0020590020204D39EA
:102EF0003220580053746570732070657220756EAF
:102F00006974003B2000DB0FC93F45BCDA3F8FB33B
:102F10000240FCF0274056946140FE4B9B4084A544
:102F2000D840E0231841346A5641E859974164DBA0
:102F3000D5416E271742B4B75542CE1A9742C8AE54
:102F4000D542B5885A43D40684BFA65FA7BF744351
:102F5000E0BF10B11AC01C2C58C0E8F697C0B849A1
:102F6000D6C04E4E17C124D355C1802497C1A0B5F9
:102F7000D5C1121A17C244AE55C2781797C26CACAD
:102F8000D5C267885AC320746F6F206C6F6E67203C
:102F9000657874727573696F6E2070726576656E90
:102FA0007465640A0020636F6C64206578747275C0
:102FB00073696F6E2070726576656E7465640A0061
:102FC0006F6B0A00526573656E643A200020453AC3
:102FD00000205A3A0020593A00583A0000002200D6
:102FE000250028002B0000002100240027002A00D3
:102FF00002020202020202020404040404040404A1
:1030000003030303030303030101010101010101A0
:1030100001020408102040800102040810204080B2
:1030200001020408102040808040201008040201A2
:103030004572726F722077726974696E6720746F5F
:1030400020454550524F4D210A00544845524D41AC
:103050004C2052554E4157415900546865726D617C
:103060006C2052756E617761790072D919E0112474
:103070001FBECFEFD0E4DEBFCDBF84B7809368150D
:1030800014BE0FB6F894A895809160008861809373
:103090006000109260000FBE12E0A0E0B1E0EEE927
:1030A000FEED01E00BBF02C007900D92A439B107FD
:1030B000D9F725E1A4E9B2E001C01D92A836B20714
:1030C000E1F718E1C6E3D8E104C02197FE010E94B0
:1030D00022ECC533D107C9F70E9437DA0C9443EFCD
:1030E0000C940000FC01A081B1811C92A281B381EB
:1030F0008C918F5F8C930280F381E02D90818CE026
:10310000989F800D1124E1E6F3E113AE84AF08959A
:10311000FC0184910895FC0180810895009751F08D
:10312000FC0180E09191992331F0907C9038D1F3AB
:103130008F5FF8CF80E00895119800C087FD43C0ED
:10314000419800C0119A00C000C0119800C086FDCF
:1031500046C0419800C0119A00C000C0119800C03C
:1031600085FD3BC0419800C0119A00C000C0119875
:1031700000C084FD30C0419800C0119A00C000C05A
:10318000119800C083FD25C0419800C0119A00C06D
:1031900000C0119800C082FD1AC0419800C0119A69
:1031A00000C000C0119800C081FD0FC0419800C050
:1031B000119A00C000C0119800C0419800C0119A37
:1031C00000C000C00895419ABCCF419AF0CF419A07
:1031D000E5CF419ADACF419ACFCF419AC4CF419AF5
:1031E000B9CF90E080E00895CF93DF93DB01F90140
:1031F0009C919130C1F0943080F094509C93883031
:10320000D1F480819181009771F00197918380833F
:10321000480F591FEA01188206C08C3539F49C5FAB
:103220009C93943041F4DF91CF9108958B3339F71B
:1032300081E08C93F8CF20813181B9016F5F7F4F9E
:1032400071836083420F531FEA01888380819181DB
:103250008F3591056CF7E7CF0F931F9381E00091B5
:10326000B3141091B4142091B5143091B614409158
:10327000AF145091B0146091B1147091B21404174E
:1032800015072607370708F480E01F910F9108956E
:1032900090E080E008952091F703833021F425FD2C
:1032A0000CC024FD0CC030E0A90102C05595479523
:1032B0008A95E2F7CA018170089581E0089580E05F
:1032C00008958091130484FD0BC08091150487FD3F
:1032D00007C090911604937081E019F480E008957E
:1032E00081E008952FEB280F2A3108F047C0E22F24
:1032F000F0E08091130490911404A0911504B09112
:10330000160404C0B695A795979587952A95D2F788
:1033100080FD02C081700895E750FC4FE081EE23EC
:1033200041F180916C0790916D07E80FF92FF11D25
:10333000808190ED980F9A3030F08E3251F4818177
:1033400080538A3098F4F093E803E093E70381E038
:1033500008958D3211F08B3249F4818190ED980FF0
:103360009A3088F38E3211F48281EACFF0E0E0E007
:10337000EACF1092E8031092E703E9CF80E00895C6
:10338000CF93DF9385E4AEDF882309F188E0409195
:103390001304509114046091150470911604972F32
:1033A0009170C92F90E0D92FCC0FDD1F71FB222720
:1033B00020F930E0220F331F220F331FC22B67FB8F
:1033C000442740F9C42B8C2BDF91CF91089580E0E6
:1033D000DECF88DF882341F081E02091E703309140
:1033E000E803232B09F480E00895B0E0A0E0EBEFC0
:1033F000F9E10C9446EC6B01E9014A3009F4D5C0BF
:10340000453109F081C0DB011296ED91FC91F2800B
:1034100096818781139A00C00000E6E2F0E03197C0
:10342000F0F7092F182FEF2CE29420EFE22230E181
:10343000B32EBF0CE80188EF7FDE00C0000086E2FB
:1034400090E00197F0F7BFE1BF1508F49BC08F2D06
:103450008077806871DE8E2D6FDE00C0000086E20E
:1034600090E00197F0F780E867DE80E065DE00C05D
:10347000000086E290E00197F0F78AEF5DDE00C081
:10348000000086E290E00197F0F7005F1F4F88810F
:10349000807F52DE89918295807F4EDEC017D107F2
:1034A000B1F700C0000086E290E00197F0F7F394D6
:1034B000E0E1EE0EFB10BECF1398D6011296ED910F
:1034C000FC9180819281980F92832181921708F05C
:1034D0009FC194819F5F94839381890F821710F01D
:1034E0008FEF820F8383458150E0440F551F70E0BA
:1034F00060E0868197810E94EFEE81E0CDB7DEB774
:10350000E9E00C9462ECDEC1FB01028113814233DD
:1035100009F485C108F48DC1463409F475C14734F6
:1035200009F482C14B3349F789812B81D801129666
:103530007C91129713963C91213009F4BFC123303E
:1035400009F0A0C148EF480F582F91E0341708F454
:1035500090E031E0541708F030E0492F432B61E050
:10356000571708F460E0462311F4932331F2FA80F0
:1035700030E0F901E656FE4FD0802A563E4FF90161
:10358000E08099C180EE8F0D8068807FD5DD8F2D22
:103590008295807FD1DD00C0000086E290E0019737
:1035A000F0F780E8C9DD80E861CF0B9A1398399A6B
:1035B0004198099A119A139A00C0000086E290E09F
:1035C0000197F0F788E790E0CEE9DFE0FE01319760
:1035D000F1F70197D9F788EFAFDD00C0000086E270
:1035E00090E00197F0F780E2A7DD80E0A5DD00C064
:1035F000000086E290E00197F0F780E09DDD80E832
:103600009BDD00C0000086E290E00197F0F780E0CB
:1036100093DD80E191DD00C0000086E290E001973B
:10362000F0F7CE010197F1F7CE010197F1F7CE0146
:103630000197F1F7CE010197F1F7CE010197F1F76C
:10364000CE010197F1F7CE010197F1F7CE01019775
:10365000F1F7CE010197F1F7CE010197F1F7CE0115
:103660000197F1F7CE010197F1F7CE010197F1F73C
:10367000CE010197F1F72197F1F780E25DDD80E45B
:103680005BDD00C0000086E290E00197F0F780E289
:1036900053DD80E651DD00C0000086E290E0019736
:1036A000F0F7D0E0C0E08C2F8077806845DD8D2F6B
:1036B00043DD00C0000086E290E00197F0F780E86B
:1036C0003BDD80E039DD00C0000086E290E001973C
:1036D000F0F78AEF31DD00C0000086E290E001974C
:1036E000F0F780E2119800C0419800C0119A00C024
:1036F00000C0119800C0419800C0119A00C000C0DD
:10370000119800C0419800C0119A00C000C01198E3
:1037100000C0419800C0119A00C000C0119800C0BC
:10372000419800C0119A00C000C0119800C0419893
:1037300000C0119A00C000C0119800C0419800C09C
:10374000119A00C000C0119800C0419800C0119AA1
:1037500000C000C0119800C0419800C0119A00C07C
:1037600000C0119800C0419800C0119A00C000C06C
:10377000119800C0419800C0119A00C000C0119873
:1037800000C0419800C0119A00C000C0119800C04C
:10379000419800C0119A00C000C0119800C0419823
:1037A00000C0119A00C000C0119800C0419800C02C
:1037B000119A00C000C0119800C0419800C0119A31
:1037C00000C000C000C00000E6E2F0E03197F0F772
:1037D000815009F087CF88EFAFDC00C0000086E29F
:1037E00090E00197F0F7CF5FD05FC03209F05BCF78
:1037F00080E0A2DC80ECA0DC00C0000086E290E06B
:103800000197F0F7139879CEF8018581888375CEFA
:1038100080E0CDB7DEB7E9E00C9462EC53C0B901AB
:10382000C8010E94E9CB69CED80111968C9188839A
:1038300064CE443191F0473109F05FCE1882D8014F
:1038400012968C911297898315968C9115978150B9
:103850008A8313968C918B8350CED80115964C9108
:10386000159750E0440F551F70E060E016968D915B
:103870009C910E94EFEEF801128280818150838337
:1038800014823BCE381708F438CE871708F435CEAB
:10389000FA80E12CD12C243070F46ACEBE01C8012C
:1038A0000E94E9CB898198819D0D98838E0D898333
:1038B000FF0C09F422CEF7FEF6CFF0CF58E0580FF8
:1038C000482F43CEEF92FF920F931F93CF93DF9336
:1038D000EC018B017A018A859B858617970731F069
:1038E000888199810E94D6CD1B870A87B70188817C
:1038F00099810E94D6C52E813F81820F932F911D01
:103900009F838E8390E080E0CDB7DEB7E6E00C9435
:1039100065ECB0E0A0E0EFE8FCE10C9445ECEC01D4
:103920007B018A018A859B858617970731F08881FC
:1039300099810E94D6CDFB86EA8688859985019675
:1039400009F5CC80DA808E81D80EA880B980D501A7
:103950005596ED91FC91C5010995C80E780110E0CE
:10396000F70121917F0121111FC08E819F81810F5D
:10397000911D9F838E8390E080E0CDB7DEB7EAE0B3
:103980000C9461ECEE80FF80B801888199810E94DF
:10399000D6C58E0D9F2D911D28853985281739078D
:1039A00080F681E090E0E9CF4C2D6D2DC5010E949D
:1039B0002ECED80E180FD4CFB0E0A0E0E2EEFCE19E
:1039C0000C9448ECEC01D62E1CAD0BAD7C0184E0D0
:1039D000E80EF11CE98DFA8DC7010995412F480FBA
:1039E0002D2D602FC7010E942ECE9BAD890F8BAF6E
:1039F00081E090E0CDB7DEB7E7E00C9464ECA6E0A0
:103A0000B0E0E5E0FDE10C943EEC7E836D83342E66
:103A1000FC014080518062807380C301B20120E1CB
:103A20003EE040E050E00E9485EB49015A018901E7
:103A30008CE3C82ED12CE12CF12CC301B201A701DB
:103A400096010E9485EB69837A838B839C83CA01EC
:103A5000B901A70196010E9485EB6B017C0133201F
:103A600061F1C301B20120E831E541E050E00E947C
:103A700085EB29013A015901DF92CF92C40168E137
:103A800070E00E94FBEB9F938F935F924F9284EACA
:103A900090E19F938F93FE81FF938D818F930E947E
:103AA000F0E40FB6F894DEBF0FBECDBF88E0FAE0B9
:103AB0004F165104D8F089E019C081149104D1F453
:103AC0008A818F9399819F93DF92CF9288E990E1C9
:103AD0009F938F93EE81EF93FD81FF930E94F0E41B
:103AE0000FB6F894DEBF0FBECDBF85E02696E1E1AC
:103AF0000C945AEC0436110568F4DF926F939F9290
:103B00008F928CE890E19F938F939E819F93ED819C
:103B1000EF93E4CFDF926F939F928F9282E890E1D0
:103B20009F938F939E819F93ED81EF930E94F0E48A
:103B30000FB6F894DEBF0FBECDBF86E0D7CF809121
:103B4000E7039091E803009731F04AE050E070E01D
:103B500060E00C9478E360E070E0CB010895809120
:103B6000E7039091E803009731F04AE050E070E0FD
:103B700060E00C944BE260E070E0CB010895EFDF71
:103B800097FD0AC0ECDF6F3F71058105910509F0D3
:103B90002CF4E5DF862F089580E008958FEF0895D7
:103BA000CF93C62F16DC882311F0E9DFC82F8C2FA6
:103BB000CF9108958091E7039091E803892B39F024
:103BC000DEDF91E0811101C090E0892F089591E03E
:103BD000FCCFCF93DF93C82FD62FFBDB882321F0B8
:103BE000E9DFDF91CF9108958C2F7CDB8111F9CF34
:103BF0008D2FF7CFB4DFCB010895CF93DF93EB0187
:103C0000E8DB882311F0F6DFEC01CE01DF91CF91E4
:103C100008950F931F93CF938091E7039091E8034A
:103C20000097D9F0FC018F01C1912C2F2F7D81F0DD
:103C3000C53411F0C536B9F7F801108270E060E0C4
:103C40000E94F5E0F801C083CF911F910F91089574
:103C500070E060E00E94F5E0F7CF60E070E0CB013B
:103C6000F3CFCF92DF92EF92FF926A017B01B1DB3B
:103C7000882319F0CEDF6B017C01C701B601FF90EC
:103C8000EF90DF90CF900895CF92DF92EF92FF9266
:103C9000CF93C82F0E9495CA6B017C0124EA30E7BC
:103CA0004DE75FE360913101709132018091330102
:103CB000909134010E9457E587FD18C08AEF90E08B
:103CC000A0E0B0E08C0D9D1DAE1DBF1D8093620471
:103CD00090936304A0936404B0936504C093270198
:103CE000CF91FF90EF90DF90CF90089580E090E02B
:103CF000DC01E8CFCF9380912304811154C010924E
:103D00009C1310929D1310929E1310926A1310929E
:103D1000691310926C1310926B1310926E1381E062
:103D200080936D1382E280936F131092741310923C
:103D30007313E8E8F3E126E933E18FEF81932E175F
:103D40003F07E1F7C1E0C09385132FEF3BEA3093C3
:103D50007B1320937A13C0937C1310927D131092DF
:103D60007E1390E490937F13109280132EEF3BEA22
:103D700030939713209396132FE131E0309368131B
:103D8000209367139EE190938C1391E190938D1390
:103D90009CE190938A1380938913809388130E94E7
:103DA00028CCC093230481E08093220483EC90E12B
:103DB000909384128093831210928612109285122F
:103DC00053985B9A52985A9A3898409A0E949BA1AD
:103DD00010927204CF910895FC0180E0309749F071
:103DE0009491992331F0907C903809F08F5F31964F
:103DF000F7CF0895B0E0A0E0E0E0FFE10C9445ECDF
:103E0000EC015B018A01FB01099587FD10C0C82EFA
:103E1000D12CF12CE12C2196F801C082D182E282D2
:103E2000F382CE01CDB7DEB7EAE00C9461EC982FB7
:103E3000907E903CA9F48F7190E0B0E0A0E06C011E
:103E40007D0156E0CC0CDD1CEE1CFF1C5A95D1F711
:103E5000CE010196F50109958F73C82A2296DCCF11
:103E6000982F907F903E11F58F7090E0B0E0A0E029
:103E70006C017D0136E0CC0CDD1CEE1CFF1C3A957C
:103E8000D1F7CE010196F50109958F73C82A46E056
:103E9000CC0CDD1CEE1CFF1C4A95D1F7CE0102961E
:103EA000F50109958F73C82A2396B6CF982F987F6E
:103EB000903F79F5877090E0B0E0A0E06C017D0163
:103EC00086E0CC0CDD1CEE1CFF1C8A95D1F7CE01E0
:103ED0000196F50109958F73C82A96E0CC0CDD1C7C
:103EE000EE1CFF1C9A95D1F7CE010296F5010995BB
:103EF0008F73C82A26E0CC0CDD1CEE1CFF1C2A9513
:103F0000D1F7CE010396F50109958F73C82A24963F
:103F100083CF982F907C903841F4807C803869F46E
:103F20002196CE01F5010995F8CF8E7F8D3F28F0BF
:103F30002196CE01F5010995F8CFC12CD12C76013F
:103F40006BCF9CE0899F802D112491E0980F909376
:103F500021042CE0280F2093550730E02E5F3F4FBF
:103F6000409199134217130619F014F080E0089558
:103F700020919B139217D0F7662341F08E5F0E9429
:103F80000DCD809155078E5F0E940DCD8091550714
:103F900090919913891750F320919B1390912104CC
:103FA000291720F310929C1380939D1381E00895AC
:103FB00020912004022E000C330B8217130641F0CF
:103FC0008093200468EE71E185E693E10C94D6CDF0
:103FD0000895ACE0B0E0EFEEFFE10C9447EC6F3FEA
:103FE00071058105910509F070F481E693E1E4DC47
:103FF000E0916913F0916A133196849190E02C96C8
:10400000E8E00C9463ECF0909C13E0909D132091F9
:10401000220421110FC042E650E16E2D8F2D0E9427
:1040200087CE90E080E0F80EF0929C13E0929D1312
:104030009927E5CFC0906913D0906A1325E633E144
:104040003A8329832F2D30E03C832B832E2D30E0C3
:104050003E832D8318861F822FEF3FEF3A872987F3
:104060001C861B8609E81CE19E012F5F3F4FAB01B8
:10407000BC01C6010E94FCACB60185E693E10E943A
:10408000D6CD8F819885CFCF4F925F926F927F92DE
:104090008F929F92BF92CF92DF92EF92FF920F93F7
:1040A0001F93CF93DF93CDB7DEB728970FB6F89461
:1040B000DEBF0FBECDBF7C016A014901FB019081CB
:1040C0008CE0989F800D1124982FF7012081822F7A
:1040D000880F820F880F80939C1390939D13411536
:1040E000510561F1FA82E9827C836B8301111FC063
:1040F000AE014B5F5F4FB401C6017CDE6C016D8188
:104100007E818F8198856115710581059105B1F0DA
:1041100060DFF70180818F5F8083853148F3CE01B6
:1041200001960E947218E4CFB12C860129C08A0141
:10413000B12C26C0452846284728B1F728960FB647
:10414000F894DEBF0FBECDBFDF91CF911F910F91CD
:10415000FF90EF90DF90CF90BF909F908F907F90D7
:104160006F905F904F900895B39407C0B1102DC029
:1041700001151105C9F20F5F1F4F01151105A9F2B5
:10418000AE014B5F5F4FB401C60134DE6C014D8060
:104190005E806F8078844114510461047104A9F039
:1041A000F0E24F1651046104710401F3D301C2011E
:1041B0008D97A109B1090297A105B10530F04BE235
:1041C000441651046104710479F6F7018081482F87
:1041D0004B0D5527551F4631510534F0853020F0E1
:1041E000CE0101960E94721881E0411451046104CD
:1041F000710409F480E0B80EF70180818B0D808393
:10420000BB2009F497CFBA94AE014B5F5F4FB40166
:10421000C801F0DD8C016D817E818F819885D9DEAA
:10422000EFCFCF93DF93FC0125AD211104C021E036
:1042300025AF0E9428CCC0916713D0916813E091FC
:104240009613F091971382E00995E0919613F091FF
:10425000971381E0099530E020E044E1BE0185E656
:1042600093E10E9423CC28E933E147E1BE0185E6D2
:1042700093E10E9423CCE0919613F091971380E094
:104280000995DF91CF9108954F925F926F927F923F
:104290008F929F92AF92BF92CF92DF92EF92FF9256
:1042A0001F93CF93DF9300D000D0CDB7DEB70E942D
:1042B00095CA6B017C01809127018F3FC1F10E945B
:1042C00095CA8090620490906304A0906404B090BA
:1042D0006504681979098A099B0997FD28C08091AE
:1042E000391390913A138F5F8F70891701F1E09124
:1042F0002701E53008F054C024E0E29FF0011124CA
:10430000E256FE4F80819181A281B38189839A8395
:10431000AB83BC8320E030E0A901BE016F5F7F4F1B
:1043200082E791E00E9450C08FEF809327010E94A6
:104330009BA18091730482FF3CC080917104811124
:104340003AC091E09093710480917804892780931A
:1043500031071092780483E0809367011092730410
:104360000E9495CA6C507E4F8F4F9F4F609374048C
:1043700070937504809376049093770468E873E1F2
:1043800082E090E00E94738B16E01150A1F00E9431
:10439000178B62E070E080E090E00E9409CAF5CFE0
:1043A0008091680190916901A0916A01B0916B01BF
:1043B000ADCF1092710480916D0490916E04A09124
:1043C0006F04B0917004A7019601281B390B4A0BAA
:1043D0005B0BDA01C901B7FF05C08091790488231E
:1043E00009F4B9C1D701C6018C599F4FAF4FBF4FD8
:1043F00080936D0490936E04A0936F04B093700447
:1044000060917204062E000C770B77FF03C0719544
:10441000619571099091720480916C04981365C044
:10442000633008F062C0109272048091720480932D
:104430006C04643008F069C0809131078111E7C0D5
:1044400080915F1390916013865F9B4241F480914D
:104450002801882309F4EDC08150809328010E942F
:1044600057758090860790908707A0908807B09036
:10447000890781110E946475D501C4013AE0B6959F
:10448000A795979587953A95D1F7009741E0A407AE
:10449000B10520F08FEF9FEFA0E0B0E096958795F3
:1044A000209167012111D7C030917904311180C169
:1044B00080915F1390916013865F9B4209F45FC106
:1044C00080917A0481115BC18091680490916904A4
:1044D000A0916A04B0916B04C81AD90AEA0AFB0ACF
:1044E000F7FC5BC10E94EF8C58C1633009F09DCF8F
:1044F0008091720487FD07C081E0880F880F809348
:10450000720464E092CF8FEFF8CF8091540721E0DE
:1045100030E040E050E0882309F456C08090500716
:1045200090905107A0905207B090530781149104C6
:10453000A104B104E9F170E090E080E00E945BE545
:1045400020E030E040E85EE30E94BCE52B013C0146
:10455000C701B601681979098A099B090E945BE5C0
:104560009B01AC01C301B2010E94EFEC20E030E0FE
:104570004AE754E40E94BCE54B015C0120E030E0D6
:1045800040EA52E40E9414EE24E630E040E050E0BD
:1045900087FF12C020E030E040EF51E4C501B401D4
:1045A0000E9414EE2AE030E040E050E087FF04C0B3
:1045B00021E030E040E050E0C0925007D092510737
:1045C000E0925207F0925307A09172040A2E000C59
:1045D000BB0B0E94CDEB24E030E040E050E00E94B5
:1045E000A7EB80914C0790914D07A0914E07B09199
:1045F0004F07820F931FA41FB51F80934C07909302
:104600004D07A0934E07B0934F0710927204D70145
:10461000C6018856954CAF4FBF4F80936804909366
:104620006904A0936A04B0936B0481E080936701EE
:1046300007CF8CE0809328018091660490916704F5
:10464000009729F00197909367048093660481E0B6
:104650008093670104CF009741F040916604509128
:1046600067044817590708F023CF80917904811116
:1046700011C0223038F0243008F43FC0243011F447
:104680001092670181E693E1CCDD81E080934B07D6
:104690008093790483E08CDC81E080938513E09142
:1046A0005F13F0916013099510924B078091790484
:1046B000811127C01092310780915F139091601390
:1046C000865F9B4209F0FCCE0E9495CADC01CB01BB
:1046D0008C199D09AE09BF0980906604909067040B
:1046E000B12CA12C88169906AA06BB0608F0E0CECC
:1046F0009093670480936604DBCE81E0809367012A
:10470000C1CF85E693E10E94A6CD91E0811101C061
:1047100090E090937904882369F280915F139091DF
:104720006013865F9B42B9F40E9495CADC01CB01FD
:104730008C199D09AE09BF09C0906604D09067042A
:10474000F12CE12CC816D906EA06FB0620F490935A
:104750006704809366040F900F900F900F90DF9185
:10476000CF911F91FF90EF90DF90CF90BF90AF90CF
:104770009F908F907F906F905F904F90089548E941
:10478000C40E4AE3D41EE11CF11CC0926804D0920E
:104790006904E0926A04F0926B04809179048111BB
:1047A000DACF809167018130B1F610926701D3CFE3
:1047B000009709F46FCF51CFACE0B0E0E2EEF3E246
:1047C0000C9447ECF0909C13E0909D1320912204F0
:1047D000211112C042E450E16E2D8F2D0E9487CE30
:1047E00090E080E0F80EF0929C13E0929D139927E0
:1047F0002C96E8E00C9463ECC0906913D0906A1397
:1048000025E633E13A8329832F2D30E03C832B8347
:104810002E2D30E03E832D8318861F827A8769878C
:104820001C861B8609E81CE19E012F5F3F4F48E86C
:1048300058E1BC01C6010E9491ADB60185E693E145
:104840000E94D6CD8F819885CDCFA4E0B0E0EBE279
:10485000F4E20C9443EC7C01062F5A01122F862FB0
:10486000660F990B9C012E563E4F690186E0882EFB
:10487000912C11160CF03DC0AE014F5F5F4F68E800
:1048800078E1C701B7DA7C0169817A818B819C81EB
:10489000611571058105910561F16D337105810522
:1048A000910509F450C06E3771058105910509F431
:1048B0004AC06A3271058105910501F507FF11C0F3
:1048C00089EB90E10E3F11F085EB90E136E01302A9
:1048D000B001112471DF66E070E00E940FEC161B3E
:1048E00060C065E470E080E090E073DB115069F532
:1048F00010E0812F2496ECE00C945FEC643271059B
:104900008105910571F4A114B104D1F0E6E01E0215
:10491000B0011124C50150DFB4010E940FEC161B39
:10492000A8CF603471058105910551F41150F6014D
:104930006081062E000C770B880B990B4ADB99CF10
:1049400048DB115096CF07FDBBCF61E089819A818A
:10495000AB81BC81CD97A105B10509F460E0600F82
:104960006A30A4F01150862F6AE00E94EEEB092F06
:10497000682F880F770B605D7F4F072E000C880B28
:10498000990B27DB112309F4B3CF602F062E000CFF
:10499000770B605D7F4F072E000C880B990B19DB9E
:1049A0001150112309F4A4CF86E01802B00111249C
:1049B000C70102DF66E070E00E940FEC161B99CF82
:1049C000E1E6F3E183AF64AF6FEF7FEFCA01F4CEAE
:1049D000ACE0B0E0EEEEF4E20C9447ECF0909C1307
:1049E000E0909D1320912204211112C042E250E177
:1049F0006E2D8F2D0E9487CE90E080E0F80EF09211
:104A00009C13E0929D1399272C96E8E00C9463EC9C
:104A1000C0906913D0906A1325E633E13A83298365
:104A20002F2D30E03C832B832E2D30E03E832D83D1
:104A300018861F827A8769871C861B8609E81CE115
:104A40009E012F5F3F4F4BE858E1BC01C6010E9419
:104A500091ADB60185E693E10E94D6CD8F81988510
:104A6000CDCF6FEF7FEFB4CFB0E0A0E0EAE3F5E2A7
:104A70000C9445EC5C016B01AFD9E82EC6010E9495
:104A80008E18F12C03E110E0081B1109C5E20E1588
:104A90001F050CF4CFE18C2F90E09C012E5F3F4F5F
:104AA000409199134217130609F08CF5099720914C
:104AB0009B13281719065CF140915707509158072E
:104AC0006091560710929C13C0939D1325E1C50178
:104AD000BCDED1E0C114D104A9F06AE370E080E04B
:104AE00090E077DA0E151F05A4F4C45F8091991346
:104AF000C81740F020919B134C2F4950550B241799
:104B000015064CF4CDB7DEB7EAE00C9461ECD0E0CA
:104B1000E1CFDD23B9F3802F880F080F000F00933A
:104B20009C13C0939D1360E270E080E090E051DA46
:104B3000C60197DFE7CFACE0B0E0E1EAF5E20C9424
:104B400043EC982F862F6A017901B02E692FF9D98D
:104B5000882309F487C010912204C701002371F152
:104B60003BD9A82E8090691390906A13111142C00E
:104B70002FEF3FEF122F23E12A1940915707509151
:104B8000580760915607C60160DEAA2009F46AC082
:104B9000B6E08B9F600111246AE370E080E090E052
:104BA00018DA57E0C516D10408F442C060E270E09C
:104BB00080E090E00EDAC81AD90AF3CF0E948E186E
:104BC000A82E8090691390906A13112389F2FE0138
:104BD00033968AE0DF011D928A95E9F785E693E135
:104BE0009A83898302E61CE19E012F5F3F4F4BE8C9
:104BF00058E112C0FE0133968AE0DF011D928A95CA
:104C0000E9F785E693E19A83898302E61CE19E0138
:104C10002F5F3F4F48E858E1B701C4010E9491ADB2
:104C2000B40185E693E10E94D6CD2F813885A2CFCD
:104C300040915507212F30E0A6E0AA9EC001112423
:104C40002E5F3F4F281739070CF49C0180E8821B28
:104C500080939C1340939D13BB2041F06FEF7FEF37
:104C6000C701AADD2C96ECE00C945FECC701F9DEDD
:104C7000F9CF0C9417AE4F925F926F927F928F9202
:104C80009F92BF92CF92DF92EF92FF920F931F936A
:104C9000CF93DF9310921804109217042FE3209300
:104CA0001B0410921A04109219041092130410920B
:104CB000140410921504109216049C01F9019081BD
:104CC0002F5F3F4F9032D1F39E34C9F4818190ED34
:104CD000980F9A3020F08D3211F08B3281F4329699
:104CE0009F012F5F3F4F808180538A3008F46DC051
:104CF0009F012F5F3F4F8081803209F468C0F0939D
:104D00006D07E0936C078F010F5F1F4FC0816AE250
:104D100070E0C8010E9409EF009731F0FC01319763
:104D200080818032E1F31182CD3421F0C43511F05D
:104D3000C734D9F5F80180810F5F1F4F8032D1F35E
:104D400080538A3090F5C0931B0490E080E06AE0C5
:104D5000AF014F5F5F4F689F9001699F300D112435
:104D6000C901C0972081820F911D27FD9A95FA01F4
:104D7000208120532A3060F390931A048093190401
:104D8000DF0131962C912032D9F3CD3461F58E318B
:104D9000910539F0F0F48731910519F08C319105C6
:104DA00011F5B0931804A0931704DF91CF911F91D0
:104DB0000F91FF90EF90DF90CF90BF909F908F90DA
:104DC0007F906F905F904F900895F90189CFF9011E
:104DD0008FCF8537910538F08737910510F3803AEA
:104DE00013E09107F1F280906C0790906D0740E01E
:104DF00050E0BA0130E020E0C12CD12C7601C39400
:104E0000FD013196DC91DD2309F484C0D132F1F447
:104E1000CD34E1F480329105C9F4409313045093EA
:104E200014046093150470931604F0931804E0932F
:104E3000170463E270E0CF010E9409EF009709F4C4
:104E4000B4CFFC011082B1CFDF01DACFD154DA3117
:104E500008F05BC0DF011D91103291F0A0EDA10FB1
:104E6000AA30E8F01E3271F4A181A053AA30B8F044
:104E70002115310519F49F0121503109B12C13C0BE
:104E8000FD01E8CF1D3211F01B3291F7A181B0ED89
:104E9000BA0FBA3020F0AE3259F7A281E6CFBE2E5B
:104EA000B818309759F3AD2FB0E02601370104C090
:104EB000440C551C661C771CDA95D2F744295529F9
:104EC00066297729A750BC4FBC92A081A154AA3172
:104ED00008F4BACFDF01D191DD2309F491CF00EDC1
:104EE000B02EBD0E19E01B15A8F713EDB12EBD0EA7
:104EF00011E01B1578F7DB3269F3FD013196DC9187
:104F0000D03209F07DCFDF01F8CF21153105E9F668
:104F10009D01DBCF309318042093170440931304B2
:104F20005093140460931504709316043ECFFC0153
:104F30006591759185919491089580E00C947E8798
:104F40008F929F92AF92BF92CF92DF92EF92FF9299
:104F5000CF93DF93EC0180909B0490909C04A090F1
:104F60009D04B0909E0420E030E0A901C501B40189
:104F70000E9457E5882309F452C0C880D980EA808E
:104F8000FB80A7019601C501B4010E9457E51816E0
:104F90000CF04AC02091E3033091E4034091E50313
:104FA0005091E603C701B6010E9457E5882321F11D
:104FB000C092E303D092E403E092E503F092E603AB
:104FC0002091DF033091E0034091E1035091E2032F
:104FD000C701B6010E94BCE59B01AC0160E070E036
:104FE00080E89FE30E9474EC6093140170931501B4
:104FF000809316019093170160911401709115012F
:105000008091160190911701DF91CF91FF90EF9061
:10501000DF90CF90BF90AF909F908F90089560E009
:1050200070E080E89FE3F0CF60E070E0CB01ECCF70
:10503000682F70E090E080E00C94BAADB0E0A0E0A2
:10504000E4E2F8E20C943FECEC01209193043091FF
:1050500094044091950450919604688179818A81E5
:105060009B810E9474EC4B015C012091970430916C
:1050700098044091990450919A046C817D818E81AD
:105080009F810E9474EC6B017C01A50194016091E9
:105090000C0170910D0180910E0190910F010E9401
:1050A00057E5882309F454C080920C0190920D01B9
:1050B000A0920E01B0920F012091D7033091D80336
:1050C0004091D9035091DA03C501B4010E94BCE5B7
:1050D0002B013C010E9488ED4B015C0120E030E097
:1050E00040EA50E40E9457E5181634F4812C912CC4
:1050F000C0EAAC2EC0E4BC2E20E030E0A901C5011E
:10510000B4010E9414EE87FF03C0812C912C54013E
:10511000A5019401C301B2010E9474EC6093CF0316
:105120007093D0038093D1039093D203C501B4014F
:105130000E9457ED6093CD03062E000C770B6F5F36
:105140007F4F6630710514F066E070E06093CB032A
:10515000D0910A011091CD03A70196016091100131
:105160007091110180911201909113010E9457E5F5
:10517000811123C0D11375C02091B3033091B403C2
:105180004091B5035091B6036091CF037091D00365
:105190008091D1039091D2030E94BCE52091B70386
:1051A0003091B8034091B9035091BA030E9475EC55
:1051B000CDB7DEB7E0E10C945BECC0921001D09269
:1051C0001101E0921201F09213012091DB03309162
:1051D000DC034091DD035091DE03C701B6010E945C
:1051E000BCE54B015C010E9488ED6B017C0120E075
:1051F00030E040EA50E40E9457E5181634F4C12C20
:10520000D12CB0EAEB2EB0E4FB2E20E030E0A90177
:10521000C701B6010E9414EE87FF03C0C12CD12C38
:105220007601A7019601C501B4010E9474EC609358
:10523000D3037093D4038093D5039093D603C7010F
:10524000B6010E9457ED6093CE03062E000C770B3B
:105250006F5F7F4F6630710514F066E070E0609319
:10526000CC03C091CE03D11305C080910B018C17E4
:1052700009F470C08091CD039091CE0390930B01FF
:1052800080930A010C2E000CDD0B27E01203C001F5
:105290001124FC01EC0FFD1FEE0FFF1FEE0FFF1F8F
:1052A000E055FB4F20813181428153812093C70318
:1052B0003093C8034093C9035093CA030091CC03B1
:1052C000002E000C110BFC01E00FF11FEE0FFF1F71
:1052D000EE0FFF1FE055FB4F60817181828193814A
:1052E0000E9474EC6093C3037093C4038093C5035E
:1052F0009093C6032091CB0337E02303F0011124E0
:10530000CE0FDF1FCC0FDD1FCC0FDD1FC055DB4FD5
:10531000288139814A815B812093BF033093C00388
:105320004093C1035093C203E00FF11FEE0FFF1F24
:10533000EE0FFF1FE055FB4F6081718182819381E9
:105340000E9474EC6093BB037093BC038093BD0315
:105350009093BE038090D3039090D403A090D50384
:10536000B090D6032091C3033091C4034091C5038C
:105370005091C603C501B4010E94BCE52091C7034A
:105380003091C8034091C9035091CA030E9475EC43
:105390006B017C01C092B703D092B803E092B903CD
:1053A000F092BA032091BB033091BC034091BD033E
:1053B0005091BE03C501B4010E94BCE52091BF031A
:1053C0003091C0034091C1035091C2030E9475EC1B
:1053D000A70196010E9474EC6093B3037093B40329
:1053E0008093B5039093B603C7CEACE0B0E0EBEF8B
:1053F000F9E20C944CEC182F882379F020E030E08F
:10540000A9016091A0047091A1048091A2049091DF
:10541000A3040E9457E58823F1F080919F0481172F
:10542000D1F00E9483728CE0E6E8F1E0DE01119693
:1054300001900D928A95E1F7CE010196FFDD8091F2
:105440009F04882361F082E791E00E94D972109254
:105450009F040E947E852C96E3E00C9468EC81E02A
:1054600080939F0482E791E00E94A572F2CFCF92D1
:10547000DF92EF92FF9280E0B8DF109297041092D3
:1054800098041092990410929A0410929304109226
:10549000940410929504109296041092A404109211
:1054A000A5041092A6041092A7041092A0041092D2
:1054B000A1041092A2041092A30440EB54E027E050
:1054C000C12CD12C60ECE62E6FE7F62E90E080E048
:1054D000FC01EE0FFF1FEE0FFF1FE40FF51FC08250
:1054E000D182E282F38201968730910589F72150BB
:1054F000445E5F4F2111EACFFF90EF90DF90CF9095
:1055000008954F925F926F927F928F929F92AF9287
:10551000BF92CF92DF92EF92FF921F93CF93DF93D0
:10552000EC01162F20919B0430919C0440919D0426
:1055300050919E04688179818A819B810E9457E500
:10554000882309F497C0B0909F0480E04EDFC880A4
:10555000D980EA80FB8020E030E0A901C701B601D4
:105560000E9414EE87FF03C0C12CD12C7601C0929B
:105570009B04D0929C04E0929D04F0929E042DEB3B
:1055800037E346E855EBC701B6010E9457E587FDB2
:105590000BC02DEB37E346E855E3C701B6010E9487
:1055A00014EE18160CF076C0A701960160E070E0CA
:1055B00080E89FE30E94EFEC6093DF037093E003C9
:1055C0008093E1039093E20380EF9FEFA9E7B4ECAF
:1055D0008093E3039093E403A093E503B093E60381
:1055E000BB2009F447C04090720150907301609055
:1055F0007401709075018090760190907701A09071
:105600007801B0907901C0907A01D0907B01E09050
:105610007C01F0907D0181E0E8DE112359F1A301C6
:105620009201609172017091730180917401909167
:1056300075010E9457E581111BC0A501940160917D
:1056400076017091770180917801909179010E94A3
:1056500057E581110DC020917A0130917B01409175
:105660007C0150917D01C701B6010E9457E581116F
:105670000E94A485DF91CF911F91FF90EF90DF9062
:10568000CF90BF90AF909F908F907F906F905F90E2
:105690004F90089560E070E0CB018ECF8F929F9283
:1056A000AF92BF92CF92DF92EF92FF92C090A00490
:1056B000D090A104E090A204F090A30420E030E098
:1056C000A901C701B6010E9457E58823E1F1A701AE
:1056D000960160E070E080E89FE30E94EFEC6B01D0
:1056E0007C018090A4049090A504A090A604B090A2
:1056F000A70420E030E0A901C501B4010E9457E5EC
:10570000882329F1A501940160E070E080E89FE31F
:105710000E94EFECC092D703D092D803E092D90355
:10572000F092DA036093DB037093DC038093DD0374
:105730009093DE03FF90EF90DF90CF90BF90AF90FB
:105740009F908F900895C12CD12C7601CACF60E034
:1057500070E0CB01DFCFCF92DF92EF92FF926B012F
:105760007C0183E3C816D104E104F10470F082E304
:10577000C81AD108E108F10862E370E080E090E027
:105780000E9409CA0E94616FECCFC701B6010E9456
:1057900009CA0E94616FFF90EF90DF90CF9008954B
:1057A000BC0190E080E00C94BAAD80916A07813032
:1057B00069F09091B71492FB882780F992FF07C097
:1057C00097FB882780F991E08927089581E0089563
:1057D0009091B71494FB882780F994FF06C081E06C
:1057E0009091A912911101C080E00895ACE0B0E061
:1057F000ECEFFBE20C943FEC1092540780913107E0
:1058000010923107882361F020E040E070E060E012
:105810008DE39FE90E94B38B2C96E0E10C945BEC46
:105820002091390130913A0140914C0750914D0738
:10583000CA01820F931F2436310509F0E9C34730AE
:10584000510544F006978A3091050CF0F0C38AE0C8
:1058500090E0F7C306964A3F5F4FACF380914B0749
:10586000882309F4D0C16091951270919612072E89
:10587000000C880B990B0E945DE511E020919112BC
:105880003091921240919312509194120E9414EE12
:1058900018160CF010E01093610480907A0190903B
:1058A0007B01A0907C01B0907D0120E030E0A90157
:1058B000C501B4010E9457E5C12CD12CE0EAEE2EBF
:1058C000E0ECFE2E87FD06C0C12CD12C70EAE72E3D
:1058D00070E4F72E20E030E04AE754E4C501B4015B
:1058E0000E94BCE5A70196010E9475EC2DEC3CECF2
:1058F0004CEC5DE30E94BCE50E9457ED6B017C011E
:1059000080E2F7FE09C0F094E094D094C094C11CEA
:10591000D11CE11CF11C8DE240907201509073018A
:10592000609074017090750120917601309177013B
:10593000409178015091790129873A874B875C879C
:1059400080937B0460E230E1C31637E2D306E104C2
:10595000F1048CF0C701B60120E137E240E050E0ED
:105960000E94A7EBCA01B9012AE030E040E050E014
:105970000E94A7EB605D60937C0460E248EEC41671
:1059800043E0D406E104F1048CF0C701B60128EE2F
:1059900033E040E050E00E94A7EBCA01B9012AE0E1
:1059A00030E040E050E00E94A7EB605D60937D0432
:1059B000C701B60124E630E040E050E00E94A7EBCA
:1059C0006AE0862E912CA12CB12CCA01B901A50147
:1059D00094010E94A7EB605D60937E04C701B6014D
:1059E000A50194010E94A7EB6B01CA01B901A501B1
:1059F00094010E94A7EBCC2009F433C32EE220933C
:105A00007F04605D6093800450E3C50EC092810402
:105A10006BE774E089E594E00E9414EF20E030E049
:105A2000A901C301B2010E9457E520E030E040E047
:105A30005FEB87FD04C020E030E040E05FE3C3019E
:105A4000B2010E9475EC0E9457EDCB010E94F789CC
:105A5000BC0184E594E00E9414EF20E030E0A9014D
:105A600069857A858B859C850E9457E520E030E02A
:105A700040E05FEB87FD04C020E030E040E05FE302
:105A800069857A858B859C850E9475EC0E9457ED0F
:105A9000CB010E94F789BC018FE494E00E9414EFCF
:105AA0008091B71400E117E283FD28C091DE8823BE
:105AB00009F4E9C28091AF149091B014A091B1148F
:105AC000B091B2140097A105B10509F4DCC2BC0184
:105AD000CD01615F784D8F4F9F4F20E137E240E06D
:105AE00050E00E9485EB6091B3147091B4148091E2
:105AF000B5149091B6140E9485EB89010E944D89DE
:105B00004B015C018D829E82AF82B886D62E809139
:105B100026018017C1F100932601C80164E670E0F8
:105B20000E94FBEB7B0188E48E9DB0018F9D700D80
:105B3000112490E080E00E945BE52AE037ED43E22B
:105B40005CE30E94BCE50E945CED60934E0401158D
:105B5000110509F09BC21092490410923F0480E89D
:105B600080933E0489E494E0FC0101900020E9F771
:105B7000CF0189549440982F990F890F880F90E88E
:105B8000981B90933D0480912501D816E1F18092F5
:105B9000250141E08D819E81AF81B8858038914596
:105BA000A140B10508F440E06DE274E0CE01059635
:105BB0000E94FF1C982F990F990F891B880F8058FE
:105BC00080932C04282D2370822EE9F401151105F1
:105BD000A9F0A0E1B7E2A01BB10B2D813E814F815E
:105BE00058850E94C3EB980150E040E00E9485EB8D
:105BF000211531054105510509F06EC210923F048F
:105C000080E880933E040E9495CA0091250410917B
:105C1000260420912704309128046B017C01C01ACE
:105C2000D10AE20AF30A9701860137FD11C02091DB
:105C300024042095209324046A547C4F8F4F9F4F57
:105C4000609325047093260480932704909328047E
:105C5000D090240411E0D11001C010E081E00E9436
:105C6000D81F80919913873180F480919B138430E1
:105C700060F036E7E32E31E1F32E03E126E044E065
:105C800069E085E693E10E94ACCE8091991384315E
:105C9000B8F480919B13823098F0DD2009F435C26E
:105CA00080918A07882309F430C280E491E17C0165
:105CB00002E123E042E068E685E693E10E94ACCE93
:105CC000809199138C3108F06EC0409091125090E1
:105CD00092126090931270909412A0909512B090CE
:105CE0009612843198F480919B13883078F08091DB
:105CF000610480FF0DC282EF90E17C010CE022E0A4
:105D000048E064E485E693E10E94ACCE809199136B
:105D1000883040F4B7FEFFC146ED50E167E082E411
:105D20000E94E024809199138C31B0F480919B13F0
:105D3000843190F020E030E040E05FE3C301B20145
:105D40000E9475EC0E9457ED77FF0EC246ED50E1C0
:105D50006CE182E40E94E024809199138C3118F563
:105D600080919B138431F8F080918A078823D9F0C1
:105D700024E6829FC001112481589F4F6FEF70E08D
:105D80000E940FECCB010E94768A27E620939C1399
:105D90002CE120939D130E94312565E270E080E0A4
:105DA00090E00E94E91F14DD882379F18091991316
:105DB000843358F580919B138A3238F107E028E04C
:105DC0004AE26AE285E693E10E9453CD05E022E0D3
:105DD0004CE262E385E693E10E9453CD24E04AE081
:105DE00061E38AE20E9423CD60916713709168138A
:105DF00082E3809381138BE28093821321E833E165
:105E000042E385E693E10E9423CC80919913853388
:105E100050F480919B13813330F024E04AE461E335
:105E200086E30E9423CD80919913843368F4809196
:105E30009B13823348F002E020914E0442E367E373
:105E400085E693E10E9453CD80919913803358F5F4
:105E500080919B13883238F180912B04811751F087
:105E600080912A0410932B048F5F833008F0A5C122
:105E700080932A0480912A048111A2C1809149044F
:105E8000882389F080913D0480939C1380E3809364
:105E90009D1389E494E00E94312565E270E080E082
:105EA00090E00E94E91F80919913883208F05DC04C
:105EB00080919B138D3108F458C02BE040E86DE1D0
:105EC00080E00E9423CD80919913873208F04DC065
:105ED00080919B138F3108F448C083E080939C131A
:105EE00006E200939D1368E570E080E090E00E9478
:105EF000E91F8BE080939C1300939D13DD2009F430
:105F000091C184E594E00E94312588E280939C133E
:105F100006E200939D1369E570E080E090E00E9446
:105F2000E91F80E380939C1300939D13DD2009F407
:105F30009EC18FE494E00E9431258DE480939C13F0
:105F400006E200939D136AE570E080E090E00E9415
:105F5000E91F85E580939C1300939D13DD2009F4D0
:105F6000ABC189E594E00E94312580919913833378
:105F700048F580919B138B3228F183E00E94D81F53
:105F800083E080939C1303E300939D1366E070E02D
:105F900080E090E00E94E91F81E00E94D81F80917C
:105FA000390190913A010E94768A2CE020939C134B
:105FB00000939D130E94312565E270E080E090E03F
:105FC0000E94E91F80919913813408F025CC8091BB
:105FD0009B13863308F420CC10929C138EE380939D
:105FE0009D1382E290E10E948E18082F863108F0FE
:105FF00088C182E290E10E943125053109F40CCC80
:1060000060E270E080E090E00E94E91F0F5FF5CF52
:10601000243631054CF48536910504F58A30910516
:1060200034F48AE090E009C084369105BCF0883EE3
:10603000E3E09E0714F087EE93E02817390709F490
:106040000DCC90933A018093390110924C07109235
:106050004D0710924E0710924F0700CC84E690E057
:10606000F0CF662351F02EE220937F04605D6093B1
:10607000800480E280938104CBCC80E28093800412
:1060800080937F04F6CF10E000E038CD2E2D80E223
:10609000243628F08E2D64E60E94E2EB805D80932A
:1060A0007F0490E22A3040F03AE0822F632F0E9472
:1060B000E2EB0E94E2EB905D90938004822F6AE015
:1060C0000E94E2EB905D909381046FE774E089E4B5
:1060D00094E00E9414EF46CD29833A834B835C837E
:1060E00081E0203831454140510508F480E0482FD7
:1060F0006FE374E0CE0101960E94FF1C982F990F68
:10610000990F891B880F80587CCD8AE091E1CFCD13
:106110008AED90E1F2CDC5010E94768AFC01808172
:1061200093E0803229F4818192E0803209F491E099
:10613000892F880F880FE92EE81A8E2D855B8093B2
:106140009C1387E080939D1323E030E0291B3109E5
:10615000CF01820F931F0E94312569E070E080E03B
:1061600090E00E94E91FDECDCB010E94768AFC01FF
:10617000808193E0803229F4818192E0803209F4B9
:1061800091E0892F880F880FF92EF81A8F2D855BE3
:1061900080939C138CE180939D1323E030E0291BB6
:1061A0003109CF01820F931F0E94312569E070E011
:1061B00080E090E00E94E91FCFCD10922A045ACED1
:1061C0008230B1F480913F04882391F043ED50E197
:1061D00060E386E30E94E02480913E0480939C1358
:1061E00080E380939D138FE394E00E9431255BCE82
:1061F00080912D04882309F456CE86E380939C1366
:1062000000E300939D136FEF7FEF80ED90E10E941C
:10621000DC2380912C0480939C1300939D138DE2CA
:1062200094E0E3CF87E00E94A78080FF15C024E5BB
:10623000E22E24E0F22EF70161917F01662309F43A
:1062400064CE6F320CF06FE3062E000C770B880BD8
:10625000990B0E94E91FEFCF80915A0780FD51CE24
:106260006FEF7FEF8BEC90E10E94DC234ECE87E056
:106270000E94A78081FF15C09FE4E92E94E0F92ECB
:10628000F70161917F01662309F457CE6F320CF05C
:106290006FE3062E000C770B880B990B0E94E91F09
:1062A000EFCF80915A0781FD44CE6FEF7FEF8BECEB
:1062B00090E10E94DC2341CE87E00E94A78082FF0C
:1062C00015C089E5E82E84E0F82EF70161917F0181
:1062D000662309F44ACE6F320CF06FE3062E000CF1
:1062E000770B880B990B0E94E91FEFCF80915A071B
:1062F00082FD37CE6FEF7FEF83EC90E10E94DC23CD
:1063000034CE809129041817B1F000912110109318
:10631000290482E290E10E948E18081708F050C00C
:106320000F5FE02FF0E0EE5DFF4E8081807C8038D3
:10633000B9F300932110E0902110F12C97012E5D0C
:106340003F4E7901C9010E948E18182F60E870E055
:10635000C7010E94E824153108F05ECA60E270E0CF
:1063600080E090E00E94E91F143109F455CA60E210
:1063700070E080E090E00E94E91F133109F44CCAFC
:1063800060E270E080E090E00E94E91F123109F4C1
:1063900043CA212F30E02E5F3F4F4AEF4203B00146
:1063A000439F700D112460587F4F82E290E10E945C
:1063B000E82460E270E080E090E00E94E91F2CCACF
:1063C00010922110B8CF80916A07823059F000DA1C
:1063D000882349F08091B71482FB882780F991E0E7
:1063E0008927089581E0089581E00895DC01EC910A
:1063F0008E2F90E0FC01EE0FFF1FE80FF91FE05019
:10640000FD4E80818F7780830895892B79F41092D7
:10641000900082E080939100109295001092940079
:10642000C19A809171008260809371000895B0E0FC
:10643000A0E0EDE1F2E30C9442ECEC016B01888109
:106440008C3008F0A6C090E0FC01EE0FFF1FE80FB3
:10645000F91FE050FD4E80818F770E9442B0198273
:106460001A8288812CE0622F0E94E2EB829FB001A9
:10647000112430E020E0AB01420F531FFA01EE0F70
:10648000FF1FE40FF51FE050FD4E908197FD07C000
:106490002F5F3F4F2C30310571F790E0B6DF7880E9
:1064A000E72CF12C8701000F111FF801EE0DFF1DE5
:1064B000E050FD4E80818068808377FC6AC080E276
:1064C000C81682E0D8060CF03FC08A8128E532E089
:1064D000281B310987FD3395220F331F220F331FED
:1064E000032E000C440B550B898178E8872E912CE4
:1064F000881A910887FD9394880C991C880C991C24
:10650000092C000CAA08BB0860E070E0CB01D7FCA6
:106510000AC0B601653B710514F064EB70E0072E0C
:10652000000C880B990B281939094A095B090E944C
:1065300076EB24EB30E040E050E00E94A7EB820EC7
:10654000931EA41EB51E64018BE08715D8F0298127
:1065500088E890E0821B910927FD9395880F991F89
:10656000880F991FC816D906CCF402972FB7F89454
:106570000E0D1F1DF801E050FD4E880F991F9283EC
:1065800081832FBF6EE571E080E090E0E4D8CE011A
:106590002DDFCDB7DEB7EDE00C945EEC2A8188E507
:1065A00092E0821B910927FD9395880F991F880F10
:1065B000991FC816D906CCF6C601D7CF1F920F92E5
:1065C0000FB60F9211240BB60F922F933F934F9358
:1065D0005F936F937F938F939F93AF93BF93EF934B
:1065E000FF938091A40387FF27C01092950010921B
:1065F00094008091A4038F5F8093A4038091A403EF
:10660000082E000C990B209124132817190629F045
:1066100024F08091A4038C30DCF18091940090915F
:106620009500049680349C4908F47DC080919400C4
:1066300090919500049679C08091A403082E000CD7
:10664000990B209124132817190699F294F2E091DE
:10665000A4038E2FEE0F990BFC01EE0FFF1FE80F26
:10666000F91FE050FD4E808187FFC3CFE091A40366
:106670008E2FEE0F990BFC01EE0FFF1FE80FF91F95
:10668000E050FD4E808160E08F770E94ADC9B1CFB0
:106690002091940030919500E091A4038E2FEE0F8D
:1066A000990BFC01EE0FFF1FE80FF91FE050FD4EA4
:1066B00081819281820F931F90939900809398001B
:1066C000E091A4038E2FEE0F990BFC01EE0FFF1F3C
:1066D000E80FF91FE050FD4E808187FF11C0E09167
:1066E000A4038E2FEE0F990BFC01EE0FFF1FE80F96
:1066F000F91FE050FD4E808161E08F770E94ADC9A7
:10670000FF91EF91BF91AF919F918F917F916F9189
:106710005F914F913F912F910F900BBE0F900FBE45
:106720000F901F90189580E49CE9909399008093B6
:1067300098008FEF8093A403E3CF9091C00095FF62
:10674000FCCF8093C6000895CF93DF93EC0189912D
:10675000882311F0F2DFFBCFDF91CF910895CF9323
:10676000DF93EC018991882311F0E7DFFBCF8DE007
:10677000E4DF8AE0E2DFDF91CF910895CF93DF93EA
:10678000EC01FE0184912196882311F0D6DFF9CF28
:10679000DF91CF910895CF93DF93EB01EFDFCE012F
:1067A000D3DFDF91CF9108950F931F93CF938C0187
:1067B000C62F8FE39EE0E2DFC801E0DF8AE3BDDFA2
:1067C00080E38C0FBADF8AE0B8DFCF911F910F9181
:1067D0000895CF92DF92EF92FF926A017B01CEDFA4
:1067E00042E0C701B6010E9461B0FF90EF90DF90D8
:1067F000CF900895CF93DF9360E57EE00E94A5C01F
:10680000C0913413D0913513488159816A817B81BD
:1068100087E49EE0DEDF4C815D816E817F8189EEC1
:106820009EE2D7DF409130135091311360913213C3
:106830007091331386EE9EE2CCDF84E49EE09EDF0F
:106840008EE790E29BDF8AE078DFDF91CF910895B9
:10685000C0DF8AE072CFAEE4B0E0E1E3F4E30C9491
:106860003DEC70E060E085E40E94FD1D9AA789A7D9
:1068700081117CC26EEB70E083E50E94FD1D3C013E
:1068800065E070E083E40E94FD1D8C0160E085E519
:106890000E94E91D8DAF60E085E190E10E941E9CA1
:1068A0000E9495CA69877A878B879C87809164014B
:1068B000909165010E976816790654F086EC9FE07A
:1068C0005DDF0E943BC1C25BDF4FE2E10C9459ECFB
:1068D00029853A854B855C85205E314B4F4F5F4F54
:1068E0002BAB3CAB4DAB5EAB82EB9FE047DF0E9436
:1068F000BD6E8FE78093971281E08093660160E020
:106900008EE99FE00E941E9C89859A85AB85BC8597
:10691000898B9A8BAB8BBC8B8BA79CA7ADA7BEA793
:10692000198E1A8E1B8E1C8E19A21AA21BA21CA2D3
:1069300019821A821B821C822FE730E040E050E06F
:106940002D873E874F87588B80E090E4ACE1B6E41A
:106950008D839E83AF83B8871D8A1E8A1F8A188EF7
:10696000FFE7CF2ED12CE12CF12C2F961FAE2F97C5
:106970001FA618AA19AA1AAA1DA21EA21FA218A60B
:1069800091E09FAB312C212C812C912C540193014F
:10699000072C000C440B550B22962CAF3DAF4EAF8D
:1069A0005FAF2297402F002E000C550B5CAF4BAF12
:1069B000C3014E969C01092E000C440B550B2696E4
:1069C0002CAF3DAF4EAF5FAF2697CC979C01990F90
:1069D000440B550B2A962CAF3DAF4EAF5FAF2A97B5
:1069E00036E0631A7108C301072C000CAA0BBB0B1D
:1069F0002E968CAF9DAFAEAFBFAF2E978091660144
:106A0000882309F48DC00E9495CA2B013C01109186
:106A10007F05112309F473C00E94286F10927F052F
:106A20008090911290909212A0909312B090941234
:106A3000A50194016D897E898F89988D0E9414EE3D
:106A400087FF04C08D8A9E8AAF8AB88EA501940103
:106A50006D817E818F8198850E9457E5181624F4F8
:106A60008D829E82AF82B88622966CAD7DAD8EAD52
:106A70009FAD22970E945DE56D8F7E8F8F8F98A3CB
:106A80009FA92D8D3E8D4F8D58A1992309F472C178
:106A9000C501B4010E9414EE18168CF5D301C20191
:106AA00029893A894B895C89821B930BA40BB50B0E
:106AB000AC01BD01485853416109710977FD1FC000
:106AC0004D855E856F8578894C195D096E097F0952
:106AD0007595679557954795409397128DA39EA3FB
:106AE000AFA3B8A78D8D9E8DAF8DB8A18D8B9E8BDA
:106AF000AF8BB88F49865A866B867C861FAA2696EE
:106B00006CAD7DAD8EAD9FAD26970E945DE5A50174
:106B100094010E9457E587FF21C087E19FE02EDEA8
:106B2000109266010E94BD6ECCCE4BEEC42ED12CCD
:106B3000E12CF12C76C124E130E040E050E02D87DB
:106B40003E874F87588B34E1C32ED12CE12CF12C9A
:106B500076C1CD86DE86EF86F88A71C1D301C20187
:106B60002BA53CA54DA55EA5821B930BA40BB50BD5
:106B7000B7FD47C089A50E94326E8AE0DEDDD301F1
:106B8000C2018053984FAF4FBF4F8BA79CA7ADA7B3
:106B9000BEA72F969FAD2F9791116FC02FA538A933
:106BA00049A95AA9C501B4010E9414EE18160CF0A7
:106BB00050C020E030E040E050E4C501B4010E9444
:106BC00075EC6FA778AB89AB9AABA3019201205EFD
:106BD000314B4F4F5F4F2BAB3CAB4DAB5EAB2E966B
:106BE0006CAD7DAD8EAD9FAD2E970E945DE5A5018C
:106BF00094010E9457E5881F8827881F2F968FAF22
:106C00002F9789859A85AB85BC858D8F9E8FAF8F99
:106C1000B8A329893A894B895C89281739074A071B
:106C20005B0720F42D8F3E8F4F8F58A38D8D9E8D47
:106C3000AF8DB8A1481A590A6A0A7B0A91E8491629
:106C40009FE4590692E16906710460F189EF9EE0C4
:106C500066CFD301C2012BA93CA94DA95EA9821B15
:106C6000930BA40BB50B44E759E263E879E2B7FD57
:106C7000C8CF80E00E94CC6EC4CF2A966CAD7DADAB
:106C80008EAD9FAD2A970E945DE59B01AC01C501C9
:106C9000B4010E9457E587FFB4CF4AE450E36AE5A8
:106CA00070E3E7CFABADBCADA215B3050CF05BC094
:106CB000B3E02B1631040CF456C08CE99EE05EDD87
:106CC0008FE79EE05BDD49815A816B817C8188E999
:106CD0009EE0BEDD8FE79EE051DD49A15AA16BA188
:106CE0007CA184E99EE0B4DD8FE79EE047DD498D1D
:106CF0005A8D6B8D7C8D80E99EE0AADD2DAD22231F
:106D000009F4DFCD89819A81AB81BC81809398128F
:106D100090939912A0939A12B0939B122CEA35EC9F
:106D200047E25EE369A17AA18BA19CA10E94BCE528
:106D300060939C1270939D1280939E1290939F1269
:106D400020E030E543EC50E4698D7A8D8B8D9C8D8D
:106D50000E94BCE56093A0127093A1128093A212CE
:106D60009093A312AECD0E94442148CE81EF9FE0C4
:106D700005DDA9CDC501B4010E9457E587FFBFCE4F
:106D8000D301C20129853A854B855C85821B930B13
:106D9000A40BB50BAC01BD01485853416109710901
:106DA00077FDADCE2114310409F4FCC02DA13EA124
:106DB0004FA158A5280F391F4A1F5B1F298B3A8BFB
:106DC0004B8B5C8B2DA13EA14FA158A5281B390BE5
:106DD0004A0B5B0BC701B6010E9476EB29893A8901
:106DE0004B895C890E94A7EBCD84DE84EF84F88810
:106DF000C20ED31EE41EF51E34E1C316D104E10415
:106E0000F1040CF498CE4CEEC416D104E104F10464
:106E10000CF08BCE50E8C516D104E104F1040CF45B
:106E200098CECD86DE86EF86F88A8EEF90E0A0E0E1
:106E3000B0E08C199D09AE09BF096C017D0186E99E
:106E40009FE09CDC6D857E858F8598890E94392620
:106E500081E99FE093DCC701B6010E9439264D818C
:106E60005E816F8178858AE89FE0B3DC4D895E8919
:106E70006F89788D83E89FE0ACDC33E02316310422
:106E80000CF490C0C701B6010E945DE520E030E03F
:106E900040E850E40E94BCE569837A838B839C833D
:106EA0002D813E814F8158856D897E898F89988D8E
:106EB0000E9474EC2BED3FE049EC5FE30E94BCE5DF
:106EC0009B01AC0169817A818B819C810E94EFECEE
:106ED0006FAB78AF89AF9AAF69897A898B899C89C2
:106EE0000E945DE52FE632E143E85AE30E94BCE5EB
:106EF0006D837E838F8398872AE939E949E15FE3CF
:106F00006FA978AD89AD9AAD0E94BCE569837A839B
:106F10008B839C839B01AC010E9475EC2D813E818B
:106F20004F8158850E94EFEC69A37AA38BA39CA3A1
:106F300020E030E040E05EE36D817E818F819885C6
:106F40000E94BCE529813A814B815C810E94BCE5AD
:106F5000698F7A8F8B8F9C8F4FA958AD69AD7AADB1
:106F60008DE79FE036DC4D815E816F81788587E714
:106F70009FE06EDC88E69FE001DC49815A816B81ED
:106F80007C8182E69FE025DC49A15AA16BA17CA10E
:106F90008CE59FE01EDC498D5A8D6B8D7C8D86E5DE
:106FA0009FE056DC8D859E85AF85B8898C0D9D1D33
:106FB000AE1DBF1DB595A7959795879580939712A0
:106FC0004CAD4F930F933F922F9282E49FE09F939B
:106FD0008F932DE43FE03F932F931F920E94019CDB
:106FE0005FEF251A350A0FB6F894DEBF0FBECDBF8E
:106FF0002D8D3E8D4F8D58A12D833E834F83588715
:10700000498A5A8A6B8A7C8A1FAB79CD69E877E016
:107010000E94A5C060915C0D70915D0D80915E0D28
:1070200090915F0D0E945BE5AB01BC0180E897E0A9
:10703000D0DB40918C0D50918D0D60918E0D709133
:107040008F0D8DE797E0C5DB4091900D5091910D2C
:107050006091920D7091930D8AE797E0BADB4091B1
:107060006E0750916F07609170077091710787E705
:1070700097E0EECBCF93DF936DE277E00E94A5C05F
:10708000CCE4DDE04CA95DA96EA97FA984E297E07C
:10709000A0DB48AD59AD6AAD7BAD81E297E099DBED
:1070A0004CAD5DAD6EAD7FAD8AE797E0D1DBDF9192
:1070B000CF910895CF93DF9369E077E00E94A5C058
:1070C000CCE4DDE04CA15DA16EA17FA180E097E062
:1070D00080DB48A559A56AA57BA589EE9EE279DBF0
:1070E0004CA55DA56EA57FA586EE9EE272DB48A944
:1070F00059A96AA97BA983EE9EE2AADBDF91CF9111
:107100000895CF93DF9364EE76E00E94A5C0CCE4AF
:10711000DDE0688179818A819B810E945BE5AB011A
:10712000BC018BED96E055DB6C817D818E819F816A
:107130000E945BE5AB01BC0189EE9EE24ADB6885FB
:1071400079858A859B850E945BE5AB01BC0186EE53
:107150009EE23FDB6C857D858E859F850E945BE589
:10716000AB01BC0183EE9EE273DBDF91CF9108950A
:10717000AF92BF92CF92DF92EF920F931F93CF9374
:10718000DF935B01EA016901882309F452C084EDB1
:1071900096E0F4DAF501608171818281938146E0A5
:1071A0000E9461B0E1100AC08BEC96E0E7DA6881DA
:1071B00079818A819B8146E00E9461B084EC96E0EF
:1071C000DDDAF601608171818281938143E00E9462
:1071D00061B08DEB96E0D2DAF80160817181828135
:1071E000938143E00E9461B084EB96E0C7DAF60138
:1071F0002081318142815381F801608171818281D6
:1072000093810E9474EC43E00E9461B0EE2099F0FB
:107210008AE093DA8FE996E0B1DA688179818A8130
:107220009B8146E00E9461B08AE087DA8AE085DAD5
:1072300002C0E110EFCFDF91CF911F910F91EF903E
:10724000DF90CF90BF90AF900895A6E5B0E0EBE25D
:10725000F9E30C943DEC2DB63EB687E00E94C28067
:1072600081110AC061E086E50E94D01D8DA38530A2
:1072700090F08AE796E082DA0FB6F8943EBE0FBE31
:107280002DBE0FB6F8943EBE0FBE2DBECA5ADF4FBC
:10729000E2E10C9459EC2DA1222319F08AE596E045
:1072A0006DDA6AE080E50E94D01D182F8CEF810F07
:1072B0008F3218F086E396E0DECF60E085E40E942E
:1072C000E91D882309F447C031E038AFE09034135A
:1072D000F0903513D7012D913D914D915C916091C6
:1072E00072017091730180917401909175010E94F7
:1072F00075ECAB01BC0188E50E94311E69877A8775
:107300008B879C87F7012481358146815781609165
:1073100076017091770180917801909179010E94B6
:1073200075ECAB01BC0189E50E94311E6D877E873B
:107330008F87988BBE01635F7F4FCE0109960E94B5
:107340007DC181110BC063E682E296E00E941E9C23
:107350008AE096E090CF83E088AFB8CF8CE40E94BB
:107360007219082F882309F44EC10E94BF1D8EA3F5
:10737000803118F083EE95E07ECFFEA1F13009F464
:1073800044C160E083E50E94E91D22968FAF2297F9
:10739000882321F0011102C037E03EA38DA1833084
:1073A00018F089EC95E0EAD990919F0429969FAF57
:1073B000299780E00E94F5290E942D841D8A1E8A4B
:1073C0001F8A188E198E1A8E1B8E1C8E83EF9FE4D7
:1073D000A3ECB7E48D8F9E8FAF8FB8A383EF9FE4AC
:1073E000A3ECB7EC89A39AA3ABA3BCA3A12FB0E0F5
:1073F000BBABAAABEDB7FEB724E0129FE019F109D1
:1074000011240FB6F894FEBF0FBEEDBF8DB79EB727
:10741000019624969FAF8EAF24972DA148ADBE0153
:10742000635F7F4FCE0109960E94B3C20E9495CA46
:10743000611571058105910511F00E94ECE019AA12
:107440001CAA1DAA1EAA1FAAAEA1A150BB0B63961F
:10745000BFAFAEAF6397812F90E0B0E0A0E067963A
:107460008CAF9DAFAEAFBFAF6797B9A9AB2FB0E000
:10747000BCA7ABA7EAA9FBA9AE17BF070CF07BC25C
:107480001196B8A7AFA3FF93EF93BF93AF9385EB8C
:1074900095E09F938F938FEB95E09F938F931F922F
:1074A0000E94019C2DB73EB7275F3F4F0FB6F8945F
:1074B0003EBF0FBE2DBF3EA1332309F48CC10E94F5
:1074C0009DE02AE030E040E050E00E94A7EB0E94FF
:1074D0005DE520E030E040EA50E40E9414EE0FEF5A
:1074E0001FEF181614F001E010E00E949DE028E65E
:1074F00031E040E050E00E94A7EB0E945DE52B01E7
:107500003C010E949DE027E130E040E050E00E9415
:10751000A7EB6B5F7F4F8F4F9F4F0E945DE569AF79
:107520007AAF8BAF9CAF8DA18430B9F449AD5AAD21
:107530006BAD7CAD87EA95E04CD9B301A2018FE930
:1075400095E047D989E995E019D90130110511F481
:1075500083E4F3D885E995E011D9B801110F880BC0
:10756000990B0E945DE521966CAF7DAF8EAF9FAF0A
:10757000219720E030E040E153E40E94BCE52D96E5
:107580006CAF7DAF8EAF9FAF2D971FA6EFA5639613
:10759000AEADBFAD6397EA171B060CF01CC1229677
:1075A000FFAD2297F11134C00E949DE024E130E04C
:1075B00040E050E00E94A7EB675E7F4F8F4F9F4FE8
:1075C0000E945DE521962CAD3DAD4EAD5FAD21979E
:1075D0000E94BCE59B01AC01C301B2010E9475ECA5
:1075E0002B013C0120E030E044EB53E40E9457E5DE
:1075F0001816ACF420E030E044EB53E4C301B201D0
:107600000E9474ECEDCF1EA2BCCE22E02EA3B9CE18
:107610002D962CAD3DAD4EAD5FAD2D97DDCF20E06D
:1076200030E0A901C301B2010E9414EE87FF0BC034
:1076300020E030E044EB53E4C301B2010E9475EC5A
:107640002B013C01ECCF0091341310913513D8017C
:1076500014962D913D914D915C9117976D857E8586
:107660008F8598890E9474EC61966CAF7DAF8EAF68
:107670009FAF619726E33AEF4EE85CE3C301B201A6
:107680000E94BCE56B017C010E94ECEC28966CAF7B
:107690007DAF8EAF9FAF2897F80120813181428165
:1076A000538169857A858B859C850E9474EC4B019A
:1076B0005C0129AD3AAD4BAD5CAD28966CAD7DADAE
:1076C0008EAD9FAD28970E94BCE59B01AC01C50122
:1076D000B4010E9475EC4B015C0189829A82AB82F5
:1076E000BC82C701B6010E9449EE29AD3AAD4BAD4F
:1076F0005CAD0E94BCE561962CAD3DAD4EAD5FAD7D
:1077000061970E9475EC6B017C01CD82DE82EF8275
:10771000F88620E030E040EE50ECC501B4010E9454
:1077200057E587FF3AC080E090E0A0EEB0EC898397
:107730009A83AB83BC8320E030E040E050ECC7018B
:10774000B6010E9457E587FF37C080E090E0A0E0D7
:10775000B0EC8D839E83AF83B887FDA1F43071F4C4
:1077600049815A816B817C8189E895E032D84D81CD
:107770005E816F81788589EE9EE26AD8198A1A8ABD
:107780001B8A1C8ABE016F5E7F4FCE0101960E944C
:1077900032C42FA52F5F2FA7F9CE20E030E041E6BD
:1077A00053E4C501B4010E9414EE181624F680E0DB
:1077B00090E0A1E6B3E4BBCF20E030E041E653E443
:1077C000C701B6010E9414EE18163CF680E090E066
:1077D000A1E6B3E4BECF20E048ADBE01635F7F4FBA
:1077E000CE0109960E94B3C24B015C01EBA5FCA53A
:1077F000EE0FFF1FEE0FFF1F24968EAD9FAD249757
:10780000E80FF91F80829182A282B382A5019401C0
:107810006D8D7E8D8F8D98A10E9414EE181624F424
:107820008D8E9E8EAF8EB8A2A501940169A17AA11A
:107830008BA19CA10E9457E587FF04C089A29AA250
:10784000ABA2BCA2A50194016CA97DA98EA99FA998
:107850000E9475EC6CAB7DAB8EAB9FAB8FA198A5F6
:10786000092E000CAA0BBB0B8FA398A7A9A7BAA738
:10787000BC01CD010E945DE56BA77CA78DA79EA7EB
:107880009B01AC016CA97DA98EA99FA90E94EFEC78
:107890002B013C014D8A5E8A6F8A788E2496AEADAC
:1078A000BFAD2497B8ABAFA710E0C12CD12C7601A7
:1078B000EFA5F8A96191719181919191F8ABEFA732
:1078C000A30192010E9474EC9B01AC010E94BCE5F3
:1078D0009B01AC01C701B6010E9475EC6B017C01F4
:1078E0001F5FF9A9F11720F72BA53CA54DA55EA5B3
:1078F0000E94EFEC0E9453EE698F7A8F8B8F9C8FE2
:107900002DA12230A0F16FA178A589A59AA50E948A
:1079100017AE84E895E00E94BE3367966CAD7DADEE
:107920008EAD9FAD67970E9417AE8EE795E00E94DF
:10793000BE3343E0C501B4010E9461B080E20E9401
:107940009D3381E03DA133300CF480E0E12C8E01C9
:107950000F5D1F4F9E01235E3F4FAE01475E5F4F9D
:10796000BE016B5E7F4F04DC8AE00E949D3389A9D3
:107970008F5F89AB7ACD0E949D2783E795E00E94B7
:10798000BE3381E09DA119160CF080E0EE24E39453
:107990008E010F5D1F4F9E01235E3F4FAE01475E7C
:1079A0005F4FBE016B5E7F4FE3DB698D7A8D8B8D00
:1079B0009C8D0052110926E042E00E9434E09F9322
:1079C0008F9382E695E09F938F938CE695E09F934B
:1079D0008F931F920E94019C0E94148429968FAD60
:1079E00029970E94F5290E94A48546CC8F929F92E8
:1079F000AF92BF92EF92FF920F931F93CF93DF93BB
:107A000085E494E00E94BE33C0E0D7E0D15021F07D
:107A100080E20E949D33FACF8C2F0E941828CF5FFE
:107A2000C73099F78AE00E949D3300EB14E0C0E074
:107A300080E20E949D338C2F0E9418287801D7E0A5
:107A400080E20E949D33F70180809180A280B38004
:107A500020E030E0A901C501B4010E9414EE87FDC9
:107A600003C08BE20E949D3343E0C501B4010E9434
:107A700061B0D150FCE1EF0EF11CD111E1CF8AE0F1
:107A80000E949D33CF5F0C5F1F4FC73089F68AE09D
:107A90000E949D33DF91CF911F910F91FF90EF9046
:107AA000BF90AF909F908F900895811107C08EE393
:107AB00094E00E94BE338AE00C949D3382E494E00B
:107AC000F8CF87E394E00C94BE3381E394E00C9408
:107AD000BE33811101C0F9CF0895CF93DF93C82F32
:107AE00069E078E00E948EC08C2FF3DFCDE8D2E110
:107AF0004B855C856D857E8580E098E00E94E9334A
:107B000020E030E543EC50E46F85788989899A89D3
:107B10000E94BCE5AB01BC018DEF97E00E94E93308
:107B20002CEA35EC47E25EE36B897C898D899E897E
:107B30000E94BCE5AB01BC018AEF97E00E94E933EB
:107B40008AE00E949D33DF91CF910895CF9384E521
:107B50000E94E919C0E08823F1F00E94BF1DC82FE0
:107B60001816CCF4B2DF8DE40E949D338091190485
:107B700090911A040E94D02B82E398E00E94BE33B9
:107B80006C2FCC0F770B880B990B0E9417AE8AE0F5
:107B90000E949D33CFEF8C2FCF910895ACE1B0E0E0
:107BA000E4EDFDE30C943DEC83E50E947219182F7F
:107BB000882309F41CC10E94DA1D8D838091720113
:107BC00090917301A0917401B0917501898F9A8F82
:107BD000AB8FBC8F20917601309177014091780175
:107BE000509179012D8B3E8B4F8B588F80917A016C
:107BF00090917B01A0917C01B0917D018D879E8742
:107C0000AF87B88B112331F09D81911103C080E0C3
:107C10000E94F5298091130490911404A0911504F9
:107C2000B091160435E1B695A795979587953A9545
:107C3000D1F79C01AD0121703327442755272987AF
:107C40003A874B875C8720E030E0A9016091A0046F
:107C50007091A1048091A2049091A3040E9457E521
:107C6000882309F4C8C083E40E947219882309F4A8
:107C700093C00E94091E698B7A8B8B8B9C8B40EB87
:107C800054E05F834E838A0157E05887412C512C82
:107C900098EC692E92EC792E812C912C28ECA22E56
:107CA00022E4B22E312C212CF101EE0FFF1FEE0F3A
:107CB000FF1FE00FF11FC080D180E280F380A70199
:107CC0009601C501B4010E9457E5181614F4460147
:107CD0005701A7019601C301B2010E9414EE87FF6C
:107CE00002C0260137018FEF281A380A97E02916BB
:107CF0003104D1F6A885A150A887045E1F4FA111B9
:107D0000D1CFA3019201C501B4010E9475EC20E01E
:107D100030E040E05FE30E94BCE529893A894B8965
:107D20005C890E9475EC4B015C012DEB37E346E862
:107D300055EB0E9457E587FD0AC02DEB37E346E877
:107D400055E3C501B4010E9414EE18162CF580E02D
:107D50000E94F52917E0EE80FF8007E0F7016191AE
:107D60007191819191917F016F01F4E0CF1AD10857
:107D7000A50194010E9474ECD6016D937D938D93BF
:107D80009C931397015051F71150EE81FF817C961F
:107D9000FF83EE831111DFCF89859A85AB85BC8582
:107DA000892B8A2B8B2B79F020E030E0A9016091A0
:107DB000A0047091A1048091A2049091A3040E9458
:107DC00057E5811113DE8AE50E947219882359F064
:107DD0000E94091E69837A838B839C8360E0CE01B5
:107DE00001960E94812A8D810E94F52914C020915C
:107DF0009F042D83E3CEFD81F11108C029853A85CA
:107E00004B855C85232B242B252BE9F25EDE8DE947
:107E100094E00E94BE339D81992349F080919F0494
:107E2000811105C04EDE8EE794E00E94BE334DDE28
:107E300080E794E00E94BE3380919F0436DE45DEE9
:107E400083E694E00E94BE33C0909B04D0909C04D3
:107E5000E0909D04F0909E0420E030E0A901C7016D
:107E6000B6010E9414EE18160CF040C042E0C701A3
:107E7000B6010E9461B08DE00E949D338AE00E94AD
:107E80009D33298D3A8D4B8D5C8D6091720170917F
:107E9000730180917401909175010E9457E58111E1
:107EA0001FC02D893E894F89588D60917601709150
:107EB000770180917801909179010E9457E58111B5
:107EC0000FC020917A0130917B0140917C0150914B
:107ED0007D016D857E858F8598890E9457E581118A
:107EE0000E94A4856C96E2E10C9459EC8EE594E036
:107EF0000E94BE33C6CFCF93DF93EB010E94BE3307
:107F0000BE01DD0F880B990B0E9417AEDF91CF9158
:107F10000895EC018B01F42E0E94BD6E209709F4A8
:107F20007CC0D3DDCE010E94BE338AE00E949D3327
:107F30000115110511F404E21EE20E947A1E1F933E
:107F40000F93DF93CF9381E094E09F938F9381E031
:107F50008F930E94019C0E94EF8CC0916613C6957E
:107F6000C69581E693E10E941121DC2FDD0F1D2FC4
:107F70001C0F8DB79EB707960FB6F8949EBF0FBE25
:107F80008DBF83E00E94D81F10929C13C0939D1355
:107F900082E290E10E94312510929C13D0939D13B0
:107FA0006FEF7FEF82EF93E00E94DC2310929C132F
:107FB00010939D136FEF7FEF85EE93E00E94DC231B
:107FC00085E693E10E94A6CD8111DBCF7ADD81E1C8
:107FD00094E00E94BE3389EE93E0019739F000C02F
:107FE0000000EEE5F9E03197F0F7F7CFF89489EE6D
:107FF00093E0019739F000C00000E6EEF3E031971E
:10800000F0F7F7CF0E94BD6EFF2021F00E9424718F
:10801000A895FECF0E94DF70FBCF0115110511F46A
:1080200004E21EE2C8E0D4E088CFCF93DF93EB01F7
:108030000E94BE33CE010E94D02B8AE00E949D3365
:10804000DF91CF9108950F931F93CF93DF93C82FA4
:108050006DEE77E00E94A5C08C2F3BDD84EE97E0AB
:108060000E94BE3380E00E941828C5EED6E0088149
:10807000198181EE97E00E94BE33C8010E94D02B87
:108080006A817B818EED97E0D0DFDF91CF911F91E8
:108090000F9108958091960D9091970D2FEF3FEFDE
:1080A000981751F0E92FF0E0EA56F24F228130E0C4
:1080B0009F5F9F779093970DC90108951F920F922C
:1080C0000FB60F9211240F900FBE0F901F901895AE
:1080D0001F920F920FB60F9211240BB60F922F938F
:1080E0008F939F93EF93FF939091C6002091970DEC
:1080F000E091960D81E08E0F8F77281729F0F0E040
:10810000EA56F24F9283E82FE093960DFF91EF919C
:108110009F918F912F910F900BBE0F900FBE0F90DC
:108120001F9018958EBD0DB407FEFDCF08958FEFFB
:108130008EBD0DB407FEFDCF8EB5089590916400FD
:108140009B7F90936400982F906A96959CBD80FDCC
:1081500003C091E0863009F490E09DBD0895A8E049
:10816000B0E0E5EBF0E40C943DECB82E80917F0E8E
:10817000843008F0F6C131E6D32E80917F0E843032
:1081800008F021C18091960D9091970D891B8F77F2
:1081900009F419C17FDF97FF0AC093DC81E393E004
:1081A0000E94BE338091960D8093970DE6CF8A3062
:1081B00019F08D3009F0FEC010927E0E80911C0ED9
:1081C00090911D0EFC01E85EF14F1682892B19F487
:1081D0000E94616FD2CF10921D0E10921C0E0EE104
:1081E0001EE0F8018191803209F446C08E3409F016
:1081F0009DC06CE273E0C8010E94D6E47C01892B2B
:1082000041F06EE470E0C80104960E9409EF009707
:1082100009F4C8014AE050E070E060E001960E9475
:108220004BE22B013C018091180E9091190EA09108
:108230001A0EB0911B0E0196A11DB11D48165906CC
:108240006A067B0629F060E089EF92E0EF2851F1A1
:108250006AE270E0C8010E9438EF9C01009729F1A2
:10826000982F901BF12C992349F09150F801E90FB8
:10827000F11D8081F826F7CF8F01B3CF4AE050E09F
:1082800070E060E0C90101960E944BE22F2D30E0C2
:1082900050E040E0621773078407950751F060E0F3
:1082A0008AED92E00E9421C068CF60E080EB92E00E
:1082B000F9CF4092180E5092190E60921A0E7092D9
:1082C0001B0E80912C078130E1F467E470E0C80157
:1082D0000E9409EF0097A9F04AE050E070E060E0EA
:1082E00001960E944BE2623071058105910548F4C8
:1082F0008FE092E00E94BE3360E085E092E00E9451
:108300001E9CF80180818D3481F58381823309F4CC
:1083100045C0883301F1803341F58181843329F5EB
:108320008281813311F50E9480851FC08091B7142E
:1083300080FFC7CF6DEC7DE2C8010E94D6E40097B4
:1083400031F0FC01838180538A3008F0BACF60E0BD
:1083500086E892E0A7CF8281803339F4818181332E
:1083600021F4109266011092780480911E0E8B33D6
:1083700009F403CF80917F0E843008F0FECE809107
:10838000810E8D9DC00111246EE17EE08E57914FCC
:108390000E9414EF80E00E94E1BFEFCE8281813322
:1083A00021F78181813309F741E070E060E087EBDC
:1083B00099E0AFDD2CE13EE04EE15EE06EE77EE06D
:1083C0000E94F418DACE8091B71483FDCAC082FFF0
:1083D000C8C087FDC6C01A82198281E6F82E94E0D3
:1083E000E92E29E6D22E80917F0E843008F0B9C0A4
:1083F0000E942C198111B5C041E050E0BE016D5FB3
:108400007F4F86EA92E10E94ABD30B8110E0019787
:1084100011F00FEF1FEF8091AE129091AF12A0916B
:10842000B012B091B1128093B3149093B414A0938E
:10843000B514B093B6140E942C190F3F100741F4E5
:10844000811106C03EDB89E493E00E94BE33CBCFAE
:108450004091810E242F30E00A3061F00D3051F050
:10846000882309F470C089819A81009719F00196D8
:108470009A8389831092A50389819A81F29EF001E3
:10848000F39EF00D1124E158F14FDF01A80FB91F41
:1084900013961C92892BA9F50E94616F0E942C19DA
:1084A000882309F4A0CF86EA92E10E94746A809141
:1084B000AE148823F1F181508093AE148D9DC001DC
:1084C000112462E08059994F0E9462D7E091AE1466
:1084D00024E0E29FF0011124E459F94F40815181D9
:1084E000628173814093B3145093B4146093B514B4
:1084F0007093B61486EA92E10E94B0D20E94F3CE45
:1085000072CF1A82198283818D3479F48481823307
:1085100061F48581853349F4868180538A3028F05F
:108520008091B7148B7F8093B71481E00E94E1BFE4
:10853000B5CF0E94E5CE8091B71488608093B714C0
:10854000E0922C0750CF4F9DA00111244E57514F60
:108550009E012F5F3F4F65EA73E0802F0E94F41861
:1085600042CF0E9495CA6B017C01BB2041F0C092B2
:108570001C04D0921D04E0921E04F0921F0480910E
:10858000F3039091F403A091F503B091F6030097E3
:10859000A105B10529F140911C0450911D04609181
:1085A0001E0470911F04840F951FA61FB71FA701FB
:1085B0009601281B390B4A0B5B0BDA01C901B7FD89
:1085C0000FC07FDA60916C0770916D0788E593E0CA
:1085D0000E9412D740E070E060E090E080E0E9CED9
:1085E0008091190190911A01A0911B01B0911C0179
:1085F000892B8A2B8B2B79F09091391380913A1328
:10860000981709F4C4C0C0921C04D0921D04E092D3
:108610001E04F0921F048091AA039091AB03A091D5
:10862000AC03B091AD0346015701881A990AAA0A12
:10863000BB0AD501C401B7FDC0C190913913809127
:108640003A1320910801981709F4D5C0E0913A1324
:108650003BE5E39FF0011124EF50F84F808128178C
:1086600099F0809308010E9495CAB09008010B2DE3
:1086700010E084E00E9442B00115110509F0BEC06F
:1086800060E084E00E94ADC980917E05882309F4F2
:1086900087C100912F0110913001C80102972091EC
:1086A000951230919612281739070CF479C18090F1
:1086B0003A138C82812C912C5401809139132C8196
:1086C000821709F4FDC0822F90E03BE5389FF0014E
:1086D000399FF00D1124E556F84F45895689678971
:1086E000708D452B462B472B81F4418D528D638D28
:1086F000748D452B462B472B41F4458D568D678D48
:1087000070A1452B462B472BE9F14BE5489F900183
:10871000499F300D1124C9018556984F1C01FC0159
:1087200061817281838194810E9453EE6D837E8387
:108730008F839887F10161A172A183A194A10E9406
:108740005BE52B013C01F10165A176A187A190A514
:108750000E945BE59B01AC01C301B2010E94EFECFA
:108760002D813E814F8158850E94BCE52B013C0143
:10877000AC019B01C501B4010E9414EE87FF02C049
:10878000530142018C818F5F8F708C8396CFBB2009
:1087900019F01092AE033FCF0E9495CA00911C04BD
:1087A00010911D0420911E0430911F048090190126
:1087B00090901A01A0901B01B0901C01080D191D8A
:1087C0002A1D3B1D601B710B820B930B97FDE1CFA4
:1087D0008091AE0381111FCF81E08093AE0380E0D2
:1087E0000E94F47081E00E94F47082E00E94F470B4
:1087F0000E94DF7010CF80918A0731CF0F3F1105A3
:1088000011F461E03ECFE8E0FEE2E491E150EA30AD
:1088100008F051C0F0E0E15FFB4B0C9422EC1944EE
:108820001E4423442D445B445B4437443F44474447
:10883000514484B5806884BDB7BC26CF84B58062BE
:1088400084BDB8BC21CF8091800080688093800077
:10885000109389000093880017CF80918000806278
:108860008093800010938B0000938A000DCF80913D
:10887000B00080688093B000B092B30005CF8091C3
:10888000B00080628093B000B092B400FDCE8091C1
:108890009000806880939000109399000093980056
:1088A000F3CE8091900080628093900010939B00A3
:1088B00000939A00E9CE003811050CF0A2CFE0CE6B
:1088C000B801110F880B990B0E945DE52B013C014B
:1088D0002091290130912A0140912B0150912C01C6
:1088E000C501B4010E94BCE5A30192010E9475EC90
:1088F0004B015C0100912D0110912E01AC019B01F7
:10890000C301B2010E9414EE18168CF0B801012EBA
:10891000000C880B990B0E945DE52B013C01A50121
:1089200094010E9457E5181614F424013501809033
:10893000A6039090A703A090A803B090A903A30159
:108940009201C501B4010E9414EE1816D4F420E07F
:1089500037ED43EA5CE3C301B2010E94BCE52B01A1
:108960003C0128E431EE4AE75FE3C501B4010E940F
:10897000BCE59B01AC01C301B2010E9475EC2B0167
:108980003C014092A6035092A7036092A803709204
:10899000A903C301B2010E9457EDCB010E94D6CAC0
:1089A000F4E6CF0ED11CE11CF11CC092AA03D092B8
:1089B000AB03E092AC03F092AD030E94616F809133
:1089C0002C07882309F4D2C010910901113061F1FC
:1089D0008091B71480648093B71481E0809309017B
:1089E00064EF71E080E090E00E94AB2B0E94B5D56F
:1089F0008091B71484FFD2C0123028F460E085E97A
:108A000093E00E941E9C83E0809367010E9495CAB8
:108A10006C597F4F8F4F9F4F60936D0470936E041E
:108A200080936F04909370040E9495CA6B017C013F
:108A3000109118011123F1F08091F8038823D1F0EF
:108A40004091AF035091B0036091B1037091B203B4
:108A500046015701841A950AA60AB70AB501A4016E
:108A600077FD1AC0833009F494C00CF083C08130C4
:108A70000CF088C0212F30E0A8EEB3E00E94D3EBC9
:108A8000C60ED71EE81EF91EC092AF03D092B003E7
:108A9000E092B103F092B2030E94178B0E9444212E
:108AA0008091F203882379F10E9495CA6B017C01C1
:108AB0008091EE039091EF03A091F003B091F10348
:108AC000A7019601281B390B4A0B5B0BDA01C90180
:108AD000B7FD19C02091F20330E0A8EEB3E00E9488
:108AE000D3EBC60ED71EE81EF91EC092EE03D0923D
:108AF000EF03E092F003F092F10380E00E94326E07
:108B00008AE00E949D338091ED03882379F10E94D1
:108B100095CA6B017C018091E9039091EA03A091D1
:108B2000EB03B091EC0346015701881A990AAA0A8F
:108B3000BB0AD501C401B7FD19C02091ED0330E097
:108B4000A8EEB3E00E94D3EBC60ED71EE81EF91EB6
:108B5000C092E903D092EA03E092EB03F092EC03B7
:108B60000E94CEB08BE393E10E9426702896E2E14A
:108B70000C9459EC843009F07DCF0E94653D84EA65
:108B800093E004C00E94653D83ED93E00E94BE33F4
:108B900071CF0E94653D8CEB93E0F8CF112309F46F
:108BA00043CF31CFA2E1B0E0E8EDF5E40C943EEC28
:108BB00090914B0D93FD7FC0082F0E94A63D182F6A
:108BC00087FD79C089E40E94E919882309F48BC0E4
:108BD0000E94BF1D282F30E01216130614F421E066
:108BE00030E0220F331F220F331FF901E855FB4FEE
:108BF00080819181198A0E94D6CA809195129091A4
:108C000096128635910574F0002381F00E949A89AE
:108C10000DC082E50E94E919882309F46CC00E9406
:108C2000FA1DE9CF0E94E2890E943BC16091951232
:108C300070919612072E000C880B990B0E945DE52F
:108C4000209191123091921240919312509194126E
:108C50000E9414EE181644F029898FE59EE0222325
:108C600029F049894A8B48C08AE69EE09F938F93FA
:108C700085E79EE09F938F931F920E94019C0F9027
:108C80000F900F900F900F9031E03A8B35C060E05D
:108C900070E0CB014FC0C701B6010E9457E587FFC6
:108CA0000EC080916601882321F0109266010E9417
:108CB0003BC130927E056296E1E10C945AEC46018C
:108CC000570100E098C08FE30E949D33CFC020E0A1
:108CD00030E040E450E40E9414EE18160CF004C199
:108CE0002601370101C183E50E94E919898B8111B1
:108CF00096CF01118ECF1A8A83E50E94E919882345
:108D000031F00E94FA1D9093300180932F0182E48C
:108D10000E94E919882331F00E94FA1D90932E01D8
:108D200080932D0186E40E947219882309F4AFCF45
:108D30000E94091E6093290170932A0180932B01E0
:108D400090932C013324339420E030E0A9010E9459
:108D500057E5811101C0312C30927E05002309F4C2
:108D6000AACF5A89552309F4A6CF10927E0581E037
:108D7000809366011D821E821F82188619861A86BC
:108D80001B861C8680E09CE3ACE1B6E48D879E8761
:108D9000AF87B88B812C912C90E8A92E9FEBB92E30
:108DA00000E0412C512C3201609195127091961285
:108DB000072E000C880B990B0E945DE56B017C016E
:108DC000A50194010E9457E58823A9F020919112F2
:108DD000309192124091931250919412998991116D
:108DE0005ACFC701B6010E9457E5082F001F002780
:108DF000001F460157010E9495CA6B017C01DC01EE
:108E0000CB0129853A854B855C85821B930BA40B8E
:108E1000B50BB7FD2EC0D701C60188519C4FAF4F8F
:108E2000BF4F89879A87AB87BC87812F0E94326E9C
:108E30008BE79EE00E94BE3341145104610471042B
:108E400009F441CFC301B201605F784D8F4F9F4F4E
:108E50006C197D098E099F0928EE33E040E050E04F
:108E60000E9485EBCA01B9010E9439268AE00E945E
:108E70009D3380E074D90E9495CA60931C0470935E
:108E80001D0480931E0490931F0420919112309131
:108E90009212409193125091941229833A834B83FA
:108EA0005C83C501B4010E9474EC9F7741145104A6
:108EB0006104710409F00BCF20E030E040E85FE38B
:108EC0000E9457E587FF10C03A89412C512C32018E
:108ED000332331F085E0482E8DE0582E612C712C23
:108EE0004C0C5D1C6E1C7F1C0023C1F18D819E818A
:108EF000AF81B885892B8A2B8B2B61F0D701C601F6
:108F00002D813E814F815885821B930BA40BB50B9D
:108F1000B7FD24C029813A814B815C816D857E85B6
:108F20008F8598890E9474EC20E030E040EC5FE38C
:108F30000E9457E587FDB5CED701C601805A9541FD
:108F4000AF4FBF4F8D839E83AF83B88729813A810E
:108F50004B815C812D873E874F87588B80916601BE
:108F6000882309F49ECE411451046104710461F018
:108F700030E1C31A37E2D30AE108F108C418D50872
:108F8000E608F708F7FE8DCE1A8A0ECFA1E3B0E00F
:108F9000ECECF7E40C943DEC89AB2091F8032CA7A2
:108FA00081E08093F80380911B048D3409F48AC317
:108FB000843511F40C94535A873491F48091190438
:108FC00090911A048D31910509F4F9C108F082C01D
:108FD0008430910509F4A0C130F4029708F4FBC075
:108FE0000E9404D773C18531910509F46FC14C9774
:108FF000B9F787E00E94A780811111C08091130406
:1090000090911404A0911504B0911604EEE0B69569
:10901000A79597958795EA95D1F780FD57C10E944E
:10902000837210923C0160919F048CE40E94E91DC0
:10903000A82E80E00E94F5290E9495CA60931C0426
:1090400070931D0480931E0490931F040E942D842E
:1090500081E08093E3060E946A86C0901304D0905A
:109060001404E0901504F090160479E1F694E79466
:10907000D794C7947A95D1F7C0FE0DC081E00E94C5
:10908000A780182F82E00E94A78011110C94FC5B2E
:1090900011E0811101C010E080911304909114043B
:1090A000A0911504B091160467E1B695A795979520
:1090B00087956A95D1F780FF02C00C94765A1123E8
:1090C00011F40C94795AB12E10E08C2D8170982EE9
:1090D0000C94925A8A35910509F4E5C250F58E3107
:1090E000910509F46FC18A9709F07ACF80912C0716
:1090F000833008F4EBC089E40E94E919082FF12CB1
:10910000882319F00E94FA1DF82E8AE40E94E919BA
:10911000E82E882309F4C5C10E94FA1D182F0111F9
:10912000C3C1173008F4C6C183E898E00E94BE337B
:10913000CDC08B35910509F4B9C28C35910509F084
:109140004FCF42E9C42E41E0D42E52E7E52E51E044
:10915000F52E212C312C10E0F60181916F010E9437
:10916000E919082F882349F10E94091E4B015C016F
:10917000D7012D913D914D915C910E9474EC2B0192
:109180003C012DEB37E346E855EB0E9457E587FDA0
:109190000AC02DEB37E346E855E3C301B2010E9454
:1091A00014EE181654F4133011F0202E032DF7018D
:1091B00080829182A282B382302E1F5FF4E0EF0E94
:1091C000F11C143049F6222009F474C20E947E85F5
:1091D0000E94A4857BC080912C07833008F476C060
:1091E000F3E8CF2EF4E0DF2EA2E7EA2EA1E0FA2E7C
:1091F00010E088E5810F0E94E919882309F470C006
:109200000E94091E4B015C01812F0E944B1988238B
:1092100059F0D7012D913D914D915C91C501B4015B
:109220000E9475EC4B015C01F60180829182A28262
:10923000B3821F5FF4E0CF0ED11C24E0E20EF11CDC
:109240001330B9F685E40E94E919882309F453C064
:109250000E94091E6B017C0183E00E944B19882348
:1092600071F020917E0130917F01409180015091F9
:109270008101C701B6010E9475EC6B017C01C092AF
:109280008F04D0929004E0929104F092920440E016
:1092900050E0BA0186E40E94311E20E030E0A901CE
:1092A0000E9414EE181684F40E94091E29E838E87A
:1092B00048E85CE30E94BCE5609335017093360199
:1092C00080933701909338010E94058199A99111EB
:1092D00002C00E94DAC0ACA5A093F8030C94B5516B
:1092E000F70180819181A281B381F601808391830E
:1092F000A283B3839ECF80917E0190917F01A09144
:109300008001B091810180938F0490939004A09389
:109310009104B0939204BBCF80E50E94E919C12C5F
:10932000D12C7601882321F00E949F1D6B017C01C6
:1093300083E50E94E919882361F00E94091E20E05C
:1093400030E04AE754E40E94BCE50E945CED6B010A
:109350007C010E94837280912210811105C060E01F
:1093600085E498E00E941E9C0E9495CAC60ED71EF6
:10937000E81EF91E0E9495CA6C197D098E099F0985
:1093800097FFA4CF80E00E94AF40F4CF60E070E090
:1093900080EA90E40C949B5AA3019201C701B601A4
:1093A0000C94E35A60E080E698E00E941E9C0E94C4
:1093B000653D8EE498E00E94BE330C94D45B0E941D
:1093C000585C84CF0091341310913513F80120813B
:1093D000318142815381609172017091730180915A
:1093E0007401909175010E9475ECAB01BC0188E598
:1093F0000E94311E69837A838B839C83D8011496E3
:109400002D913D914D915C911797609176017091EE
:10941000770180917801909179010E9475ECAB0100
:10942000BC0189E50E94311E6D837E838F839887FE
:10943000BE016B5F7F4FCE0101960E947DC18823E4
:1094400009F444CF80E00E94F5290E942D8461E058
:1094500085E40E94E91D21E0482FBE016B5F7F4F2C
:10946000CE0101960E94B3C26B017C0149815A81F1
:109470006B817C818BE798E00E94E9334D815E81AE
:109480006F81788586E798E00E94E933B701A601ED
:1094900081E798E00E9428340E9414840E94A485E9
:1094A00015CF10E0002331F0B6E0BF1508F43CCE34
:1094B000E11037CE80E1E2E7F1E0A3E8B4E001900B
:1094C0000D928A95E1F7002319F16F2DFF0C770BB0
:1094D000880B990B0E945DE52091A0043091A104B6
:1094E0004091A2045091A3040E94BCE520919304F2
:1094F0003091940440919504509196040E9475EC2B
:10950000609383047093840480938504909386040D
:10951000EE2019F1612F110F770B880B990B0E9428
:109520005DE52091A4043091A5044091A6045091DA
:10953000A7040E94BCE520919704309198044091C3
:10954000990450919A040E9475EC6093870470937B
:1095500088048093890490938A0460E080E50E94E7
:10956000E91D8823C1F10023D1F0E0913413F0917B
:109570003513208131814281538160918304709140
:10958000840480918504909186040E9474EC609319
:109590008304709384048093850490938604EE2062
:1095A000D1F0E0913413F091351324813581468157
:1095B000578160918704709188048091890490910B
:1095C0008A040E9474EC60938704709388048093EB
:1095D000890490938A0440E050E0BA0186E40E9436
:1095E000311E6B017C0120E030E0A9010E9414EEE5
:1095F00087FF03C0C12CD12C760129E838E848E860
:109600005CE3C701B6010E94BCE56B017C01809060
:10961000350190903601A0903701B090380120E0DC
:1096200030E0A9010E9457E5882341F0C09235013E
:10963000D0923601E0923701F09238010091390161
:1096400010913A0184E690E090933A0180933901B9
:10965000C0906C01D0906D01E0906E01F0906F01B0
:1096600080E090E0A0E8BFE380936C0190936D01EF
:10967000A0936E01B0936F010E9405818092350125
:1096800090923601A0923701B092380110933A01BE
:1096900000933901C0926C01D0926D01E0926E018D
:1096A000F0926F0113CE1092F70310CE8FE08093EB
:1096B000F7030CCE332009F48BCD8EE791E00E94A6
:1096C000827F86CD8091190490911A048337910589
:1096D00011F40C94325408F04AC18B34910509F40A
:1096E00026C608F0E9C08831910509F450C408F095
:1096F000BAC08231910509F46DC708F06EC082309E
:10970000910508F4BAC3419709F06ACC0E94611927
:10971000882309F40EC40E94C01900917505102F0A
:109720001095182309F4D2CDF12CE12CD12CA12EC7
:10973000B12CC5010E2C02C0959587950A94E2F7CD
:1097400080FF08C08E2D0E942B71F701E15EFD4F56
:109750008081D82A3FEFE31AF30A83E0E816F10488
:1097600041F713FF05C00E94ED709D2D9360D92E27
:10977000102B10951D2109F4A9CD88E20E949D337C
:10978000F12CE12CC12ED12CC6010E2C02C09595D6
:1097900087950A94E2F780FF09C0F701EE56FE4F65
:1097A00080810E949D3380E20E949D33AFEFEA1AD0
:1097B000FA0AB3E0EB16F10439F713FF09C085E4A8
:1097C0000E949D3380E30E949D3380E20E949D337E
:1097D0008FEA98E00E94BE3379CD8531910509F476
:1097E000C0C358F5449709F0FBCB8091B71484FFB0
:1097F000B1C380EE98E00E94BE338091B71484FF1D
:1098000017C08CED92E10E94A36B8BE1ECEDF2E1CD
:10981000DE01119601900D928A95E1F770E060E00B
:10982000CE0101960E948AD8CE0101960E94736DE6
:1098300081ED98E00E94BE3349CD8631910509F44F
:1098400093C3479709F0CCCB8091170490911804EB
:10985000FC012191222309F496C32032D1F7DF01C4
:1098600011971C92F6CF8D31910509F41EC4A0F416
:109870008A31910509F4A4C308F494C38B3191058E
:1098800009F4B9C34C9709F0ABCB809117049091C0
:1098900018040E9417D71ACD8F31910509F4A2C47C
:1098A00008F409C48032910509F45CC4C09709F03A
:1098B00097CB0E9425390ACD8936910509F443C515
:1098C00058F58335910509F47DC6A8F48D349105CA
:1098D00009F435C508F42FC58135910509F45DC635
:1098E0008235910509F07CCB8091F7038F7D8061F3
:1098F0008093F703EBCC8535910509F405C708F48F
:1099000069C68C35910509F424C78836910509F09C
:1099100067CB80E047D9DACC8E36910509F46DC566
:1099200088F48B36910509F45DC508F422C58C36A0
:10993000910509F4B1C58D36910509F051CB81E04F
:1099400031D9C4CC8037910509F4ACC508F468C599
:109950008137910509F4B1C58237910509F040CBF3
:109960000E94CEB08BE393E10E942670AFCC8C3284
:1099700021E0920711F40C94755808F062C18B3CF9
:10998000910511F40C94985508F067C0893791053A
:1099900011F40C94205550F58637910511F40C9470
:1099A000E35498F48537910509F01ACB8091170498
:1099B00090911804009709F4F2C2DC012C91222343
:1099C00009F4EDC20E94BCBF81CC8737910511F428
:1099D0000C941C558837910509F002CB81E08093E7
:1099E000E3068093E2060E946A8670CC8A3991056C
:1099F00009F485C5A0F48139910509F0F1CA70E038
:109A000060E083E50E94FD1D823010F40C9428551F
:109A10000E94613D82E69CE00E94BE3357CC8B39A8
:109A2000910509F493C5893C910509F0D9CA809143
:109A3000130484FF02C00C946E558091150488783D
:109A400011F00C946E5580911604837011F00C94F3
:109A50006E5581E00E94813839CC8D3D910511F41D
:109A60000C94275708F052C08D3C910511F40C94CA
:109A7000215610F40C94CC55833D910511F40C94AF
:109A80008E568C3D910509F0ABCA82E40E94721992
:109A9000882341F08091390190913A0190931E0101
:109AA00080931D0182E50E947219882341F0809104
:109AB0001D0190911E0190933A018093390183E535
:109AC0000E94E919882331F00E94FA1D90933A010F
:109AD000809339018091130490911404A09115048E
:109AE000B0911604892B8A2B8B2B09F0EFCB609158
:109AF000390170913A0183ED9CE00E947B3F85E241
:109B00000E949D338AE00E949D33E0CB8931A1E021
:109B10009A0711F40C94F25720F58831914009F01E
:109B20005FCA80E50E94E919882309F4CFCB0E941F
:109B3000FA1D8C01892B11F00C94E55783E50E94E6
:109B4000E919882311F40C947A570E94FA1D97FFA3
:109B500002C00C947457BC0185E293E10E94173255
:109B6000B5CB8A31F1E09F0711F40C94365882325C
:109B7000914009F035CA8AE50E94E919882311F459
:109B80000C9450580E94091E20E030E040E050EC58
:109B90000E9414EEC12CD12CE12C60ECF62E87FD36
:109BA00013C00E94091E20E030E040E050E40E9413
:109BB00057E5C12CD12CE12C50E4F52E181624F0D9
:109BC0000E94091E6B017C012091680D3091690D86
:109BD00040916A0D50916B0DC701B6010E94BCE522
:109BE0000E9457EDCB010E945EC161E080E50E94BA
:109BF000E91D882311F40C945658A7019601609131
:109C000030137091311380913213909133130E946D
:109C100075EC6093301370933113809332139093EB
:109C200033130E94653D4091301350913113609180
:109C30003213709133138BE39DE00E9428340C940F
:109C40005658843F31E0930711F40C94445908F0BE
:109C5000A5C08139B1E09B0711F40C942859B0F4E8
:109C60008E32F1E09F0711F40C94DE5810F40C943E
:109C700094588F3231E0930711F40C9424598039B1
:109C8000914009F0ADC90E94837220CB8A39B1E0BE
:109C90009B0709F40EC448F48239914009F0A0C929
:109CA0000E949D270E94A48511CB843A21E092074F
:109CB00011F40C943559853A914009F091C96FEF30
:109CC0007FEF89E40E94FD1D8C016FEF7FEF8AE436
:109CD0000E94FD1D7C018AE50E94E919D12C8111A9
:109CE00008C081E50E94E919D82E882311F40C944C
:109CF000F45BC02E81E0800F883010F00C943C594A
:109D0000BE2C81E08E0D883010F00C943C59102F41
:109D10000E94091E2B013C01A02E07FDA12C17FF5C
:109D200002C046E0C42E8E2DE7FCE12C87FF02C066
:109D300036E0B32E27E0322ECA1408F4C7CAFE2C30
:109D40003A9C40011124BF1410F40C9439590F2D82
:109D500010E020E030E0A901DD2069F0F401E00F1F
:109D6000F11FEE0FFF1FEE0FFF1FE055FB4F20818D
:109D7000318142815381080D191D000F111F000F01
:109D8000111F00551B4FC301B2010E9475ECF80171
:109D90006083718382839383F394D5CF8C30A2E068
:109DA0009A0711F40C945A5920F5863FE1E09E077A
:109DB00011F40C944C5910F40C944859873F21E04D
:109DC000920711F40C945059883F914009F008C94A
:109DD00081E0809374050E94BDA2109274058823CF
:109DE00009F474CA0E94653D82EB9DE00E94BE3377
:109DF0006DCA803AA3E09A0709F4E7C1A0F483355D
:109E0000934009F0EDC88091150487FF02C00C94BF
:109E1000725980911604837011F00C94725981E08C
:109E20000E94FA3353CA873EF3E09F0711F40C9463
:109E3000435A893E934009F0D3C80E9483728091AF
:109E4000B714877F8B7F8093B7140E944D896D3341
:109E500071058105910520F089E29EE00E94005C79
:109E600085E29EE00E94005C81E19EE00E94BE339C
:109E70008DE09EE00E94005C29CA80E50E94E919FD
:109E8000C12CD12C7601882321F00E949F1D6B01EB
:109E90007C0183E50E94E919882361F00E94091E74
:109EA00020E030E04AE754E40E94BCE50E945CED0B
:109EB0006B017C010E9483728091170490911804B9
:109EC000009711F10E94BCBF1091F80383E08093CA
:109ED000F80381E080937804C114D104E104F10413
:109EE00031F00E9495CAC60ED71EE81EF91E809159
:109EF00078048823B9F0C114D104E104F10451F4C9
:109F000080E00E94AF40F3CF60E08CE998E00E94CF
:109F10001E9CDACF0E9495CA6C197D098E099F0993
:109F200097FDEECF109278041093F8030E943BC186
:109F3000CDC960E08EEB98E00E941E9C80E00E94FC
:109F40002B7181E00E942B7182E00E942B710E9494
:109F5000ED70BCC90E94653D87EC98E00E94BE335D
:109F6000B5C90E94B5D5B2C98091B71482FF02C0AD
:109F700087FFACC90E94E5CE8091B7148F7E8064C4
:109F80008093B714A3C960E00E9462D79FC90E9462
:109F9000E82B882321F00E94F3CE0E949A890E9428
:109FA0003BC194C98091B71482FF05C087FD03C0EF
:109FB0008B7F8093B7140E94CD890E943BC186C9D4
:109FC0008091B71484FF82C983E50E94E919882330
:109FD00009F47CC90E94AF1DAB01BC014093B314CE
:109FE0005093B4146093B5147093B61486EA92E15A
:109FF0000E94B0D26BC98091130490911404A09177
:10A000001504B091160432E0B695A79597958795FB
:10A010003A95D1F780FF1CC08EE199E00E94BE33D3
:10A020008091A912882379F0BE016F5F7F4F86EA85
:10A0300092E10E94976ACE0101960E94A4338AE0C1
:10A040000E949D3343C981EF98E00E94BE33F7CF51
:10A050008091B71482FF24C0C090B314D090B41480
:10A06000E090B514F090B6148CE099E00E94BE33F5
:10A07000C701B6010E94BAAD8FE20E949D33609184
:10A08000AF147091B0148091B1149091B2140E94E9
:10A09000BAAD8DE00E949D338AE00E949D3316C9BF
:10A0A0008BEF98E00E94BE3311C98091B7148E7F68
:10A0B0008093B7140BC98091B71484FF07C90E941D
:10A0C0009AD28091B71484FF01C94091170450912E
:10A0D0001804BE01645E7F4F80E00E9425D68C018B
:10A0E000009709F4F3C86C8D7D8D19821C8222E0E3
:10A0F000AC01CE0101960E94786D811115C0F12C42
:10A10000CE0101960E94736DB801FF2011F188E421
:10A1100099E00E9412D71092B3141092B4141092C6
:10A12000B5141092B614D2C8CE0101960E9435D350
:10A13000882329F361E0CE0101960E947D6A009791
:10A14000F1F225EEFC0120831C820E942FCFF82E15
:10A15000D7CF80E399E00E94CB338DE299E00E9453
:10A16000BE33B4C88091B71482FF03C087FF0E943A
:10A1700083728091B71484FFA9C860E080E50E94D3
:10A18000E91D182F682F80911704909118040E94E0
:10A1900062D783E50E94E919882381F00E94AF1DF0
:10A1A000AB01BC014093B3145093B4146093B51445
:10A1B0007093B61486EA92E10E94B0D20E94F3CE68
:10A1C000111184C80E949A8981C820911704309186
:10A1D00018049091B71492609093B714C9010E942B
:10A1E00017D774C80E944D896B017C0120E831E5C6
:10A1F00041E050E00E9485EBC9016DE671E00E94EC
:10A20000FBEB4B015C01C701B60120E13EE040E001
:10A2100050E00E9485EBCA01B90128E130E040E03E
:10A2200050E00E9485EB2B013C011B01C701B601E8
:10A230002CE330E040E050E00E9485EB6B017C01B4
:10A24000CA01B9012CE330E040E050E00E9485EB08
:10A250008E010F5F1F4F8114910411F1DF92CF9295
:10A260007F936F935F924F92BF92AF929F928F9224
:10A270008EE799E09F938F931F930F930E94F0E4D2
:10A280000FB6F894DEBF0FBECDBFC8010E94BCBFA1
:10A290000E94653DB80182E999E00E9412D716C874
:10A2A000A114B10489F0DF92CF927F936F935F92F4
:10A2B0004F92BF92AF928EE699E09F938F931F9338
:10A2C0000F930E94F0E4DCCF4114510479F0DF9247
:10A2D000CF927F936F935F924F9282E699E09F9324
:10A2E0008F931F930F930E94F0E4CACF61157105FD
:10A2F00069F0DF92CF927F936F938AE599E09F9305
:10A300008F931F930F930E94F0E4BACFDF92CF9206
:10A3100086E599E09F938F931F930F930E94F0E43B
:10A320000F900F900F900F900F900F90AECF0E9454
:10A330009A890C9466490E94CD890C9466490E94C2
:10A34000E2890C9466490E94A63D182F87FD0AC039
:10A350008FE999E00E94BE33812F0E94326E8AE01D
:10A360000E949D33FCA5F093F803E196E2E10C9482
:10A3700059EC60E080E50E94D01D81110C94664983
:10A380008091130490911404A0911504B0911604C7
:10A3900060918A07062F10E080FD02C00FEF10E0E9
:10A3A00089E40E94E919882311F40C94E85B0E9467
:10A3B000BF1D90E01816190614F481E090E0880F94
:10A3C000991F880F991FFC01E855FB4F02811381EB
:10A3D0000F3F110519F010F00FEF10E000938A07FE
:10A3E0000C94664960E080E50E94D01D81110C94B8
:10A3F000664910928A070C9466498EE40E94E91916
:10A40000882311F40C9466490E94AF1D6093180EC6
:10A410007093190E80931A0E90931B0E0C9466493C
:10A4200083E50E94E919882321F00E94BF1D8093D3
:10A430004B0D0E94653D80EB99E00E94BE338091F8
:10A440004B0D882331F110E000E020E080914B0DAE
:10A4500090E0002E02C0959587950A94E2F780FF60
:10A4600012C0FF24F394F20E222319F08CE20E9412
:10A470009D33F801EE0FFF1FEA55F64F8591949139
:10A480000E94BE332F2D0F5F1F4F05301105F1F6CF
:10A49000D6CD82EA99E0D9CD109278041092660167
:10A4A0000C94664941E070E060E087EB99E00E941F
:10A4B000893F0E9480850C94664983E50E94E919D2
:10A4C000882369F00E94BF1D8D3320F4809318010A
:10A4D0000C9466498CE3809318010C9466490E94A1
:10A4E000653D1091180185EC99E00E94BE33812FE3
:10A4F0000E9418288AE00E949D330C94664983E5E7
:10A500000E94E919882311F40C9466490E94BF1D2A
:10A51000182F8C3308F08CE38093ED030E9495CACA
:10A520006B017C01212F30E0A8EEB3E00E94D3EB59
:10A53000C60ED71EE81EF91EC092E903D092EA03A8
:10A54000E092EB03F092EC030C94664983E50E94E1
:10A55000E919882311F40C9466490E94BF1D182F35
:10A560008C3308F08CE38093F2030E9495CA6B0150
:10A570007C01212F30E0A8EEB3E00E94D3EBC60EA1
:10A58000D71EE81EF91EC092EE03D092EF03E092B0
:10A59000F003F092F1030C9466490E9494721092B9
:10A5A0008A070E94BD6E0E94E28968EE73E080E037
:10A5B00090E00E94AB2B60E08CEC99E00E941E9C26
:10A5C0000C9466498091F7038F7E80628093F70335
:10A5D0000C94664983E50E94E9198823F1F00E94F2
:10A5E00095CA60931C0470931D0480931E0490937D
:10A5F0001F040E94091E20E030E04AE754E40E9454
:10A60000BCE50E945CED6093190170931A01809380
:10A610001B0190931C010C9466490E9461198823C8
:10A6200009F46EC00E9483720E94C019082F109115
:10A630007505182311F40C946649F12CE12CC82EF1
:10A64000D12CAA24A394B12CC6010E2C02C095953E
:10A6500087950A94E2F780FF12C08E2D0E94F47055
:10A66000882369F0F701E15EFD4F808195010E2C92
:10A6700001C0220F0A94EAF7822B809518232FEF4E
:10A68000E21AF20A33E0E316F104F1F603FF04C024
:10A690000E94DF708111147FF12CE12CC12ED12C8E
:10A6A000C6010E2C02C0959587950A94E2F780FFAB
:10A6B0000FC0F701EE56FE4F80810E949D33F701D7
:10A6C000E15EFD4F90818091750589230E9438D904
:10A6D0008FEFE81AF80A93E0E916F10409F713FD81
:10A6E00002C00C94664985E40E949D3380E30E9479
:10A6F0009D338091750583700E9438D90C9466490A
:10A700000E9494720C94664983E50E947219882312
:10A7100011F40C9466490E9495CA60931C047093CE
:10A720001D0480931E0490931F040E94091E20E0C4
:10A7300030E04AE754E40E94BCE50E945CED60937F
:10A74000F3037093F4038093F5039093F6030C9452
:10A7500066490E94A63D87FF02C00C94664980911D
:10A76000130484FD0DC08091150487FD09C08091FC
:10A770001604837029F481E00E94ADC00C946649F0
:10A78000B2E9CB2EB1E0DB2E1CE4E12E1DE0F12E70
:10A7900010E0D6018D916D010E94E919882349F0DE
:10A7A000133089F00E94091EF701648B758B868B2C
:10A7B000978B1F5FF4E0EF0EF11C143051F70E94ED
:10A7C0005B720C9466490E94091E4B015C0120E0FB
:10A7D00030E040EA51E40E9457E587FF3AC0A50106
:10A7E000940160916C0D70916D0D80916E0D909142
:10A7F0006F0D0E94EFEC2B013C01AC019B016091BD
:10A800007C0D70917D0D80917E0D90917F0D0E9449
:10A81000BCE560937C0D70937D0D80937E0D9093CD
:10A820007F0D60917E0770917F07809180079091E6
:10A8300081070E945BE5A30192010E94BCE50E9492
:10A840005CED60937E0770937F0780938007909301
:10A85000810780926C0D90926D0DA0926E0DB0925A
:10A860006F0DA7CF88E99BE00E94BE3360E088E8C7
:10A870009BE00E94D43360E083E79BE00E94D433E6
:10A8800061E08CE69BE00E94D43360E081E69BE0CF
:10A890000E94D43361E082E59BE00E94D43361E002
:10A8A00082E49BE00E94D43360E089E39BE00E9455
:10A8B000D43361E08FE29BE00E94D43361E085E213
:10A8C0009BE00E94D43360E08EE19BE00E94D43391
:10A8D00061E086E19BE00E94D43361E088E09BE088
:10A8E0000E94D43360E08AEF9AE00E94D43360E0A3
:10A8F0008BEE9AE00E94D43360E08DED9AE00E94E6
:10A90000D43360E087EC9AE00E94D43360E086EBB9
:10A910009AE00E94D43360E081EA9AE00E94D43346
:10A9200060E082E99AE00E94D43361E08BE89AE02B
:10A930000E94D43360E084E89AE00E94D43361E05E
:10A940008BE79AE00E94D43360E086E69AE00E94AA
:10A95000D43360E088E59AE00E94D43360E08BE471
:10A960009AE00E94D43361E088E39AE00E94D433F5
:10A9700060E08BE29AE00E94D43360E086E29AE0E5
:10A980000E94D43361E089E19AE00E94D43360E010
:10A9900085E09AE00E94D43360E082EF99E00E9463
:10A9A000D43360E082E892E10E944819682F617018
:10A9B00089EE99E00E94D43360E08BED99E00E942B
:10A9C000D4330C946649009117041091180494E054
:10A9D000F12C40E09150F9F0F8018081282F2B7F75
:10A9E000213499F421812133B1F4813411F185347A
:10A9F00009F441E098012E5F3F4F89012F5F3F4FDF
:10AA0000F80180818032C9F3E5CF803521F481815E
:10AA100080538A3078F341110E94653DFF2021F078
:10AA20008FE59CE00E94BE33C8010E94AF330C94B6
:10AA30006649FF24F394DECF0E944F860C9466494A
:10AA40001092E3061092E2060E946A860C94664910
:10AA50008C01112788E40E94E9198823A9F00E943B
:10AA6000FA1D8A3A910574F10E94FA1D863F9105FC
:10AA700064F50E94FA1DF801EE0FFF1FEE0FFF1F95
:10AA8000E855FB4F9183808386E40E94E91988236F
:10AA900011F40C9466490E94FA1D97FD19C00E949A
:10AAA000FA1D8F3F910509F0B4F40E94FA1D000FC2
:10AAB000111F000F111FF801E855FB4F938382838C
:10AAC0000C9466498AEA90E0D6CF85EF90E0D3CF28
:10AAD00090E080E0ECCF8FEF90E0E9CF0E94A63DC0
:10AAE00087FF02C00C94664902E911E06CE4E62E8F
:10AAF0006DE0F62E76E9C72E71E0D72ED8018D9144
:10AB00008D010E94E919882359F00E94091E0E94B4
:10AB10005CEDF70160837183828393830E941772D7
:10AB2000F4E0EF0EF11CC016D10641F70C94664913
:10AB30008091130484FD0DC080911504887849F438
:10AB400080911604837029F481E00E945A380C9495
:10AB500066490E94A63D87FF02C00C94664952E9EF
:10AB6000E52E51E0F52E10E000E0D7018D917D013A
:10AB70000E94E919882349F00E94091EF801E45B4C
:10AB8000F24F64A375A386A397A30C5F1F4F0031F8
:10AB9000110559F70C9466498091140487FD09C08A
:10ABA000809115048E7029F481E00E943A380C944B
:10ABB000664983E50E94E919882391F00E94091EE5
:10ABC0006093800D7093810D8093820D9093830D1F
:10ABD0006093880D7093890D80938A0D90938B0DEF
:10ABE00080E50E94E919882351F00E94091E6093B4
:10ABF000800D7093810D8093820D9093830D82E57B
:10AC00000E94E919882351F00E94091E6093840D67
:10AC10007093850D8093860D9093870D84E50E9437
:10AC2000E919882311F40C9466490E94091E609367
:10AC3000880D7093890D80938A0D90938B0D0C94E1
:10AC400066498091130481FD0DC08091140481FD3B
:10AC500009C0809115048C7029F481E00E940638A7
:10AC60000C94664982E40E94E919882351F00E94FD
:10AC70009F1D60935C0D70935D0D80935E0D9093AE
:10AC80005F0D83E50E94E919882351F00E94091E97
:10AC900060938C0D70938D0D80938E0D90938F0D1E
:10ACA00084E50E94E919882351F00E94091E6093EF
:10ACB000900D7093910D8093920D9093930D8AE473
:10ACC0000E94E919882311F40C9466490E94091E18
:10ACD0006B017C012AE037ED43E25CE30E9414EE55
:10ACE00087FD14C02AE939E949E95EE3C701B601E5
:10ACF0000E9457E5181654F0C0926E07D0926F0765
:10AD0000E0927007F09271070C9466490E94613DD1
:10AD100084E89CE00E94BE330C94664983E50E945F
:10AD20007219882331F00E94DA1D80933B010C9444
:10AD3000664965EC7CE081E00E94A5C010913B0172
:10AD4000105D8CEB9CE00E94BE33812F0E949D33EE
:10AD500088EB9CE00E94BE3380913B010E94553DF0
:10AD600080913D0190913E01A0913F01B091400141
:10AD70008CA39DA3AEA3BFA340904101509042017C
:10AD8000609043017090440180904501909046018D
:10AD9000A0904701B0904801C0904901D0904A016D
:10ADA000E0904B01F0904C0180914D0190914E014B
:10ADB000A0914F01B091500188A799A7AAA7BBA75E
:10ADC0008091510190915201A0915301B091540191
:10ADD0008DA79EA7AFA7B8AB80EB9CE00E94BE33C7
:10ADE0004CA15DA16EA17FA183EA9CE00E94E933A2
:10ADF000B301A20189EE9EE20E94E933B501A401EC
:10AE000086EE9EE20E94E9338EEA9CE00E94BE3309
:10AE100086EA9CE00E94BE33B701A60183EA9CE06B
:10AE20000E94E93348A559A56AA57BA589EE9EE253
:10AE30000E94E9334DA55EA56FA578A986EE9EE236
:10AE40000E94E9338AE00E949D330C9466490E9477
:10AE5000A63D082F87FF02C00C94664983E50E9437
:10AE6000E919002E000C110B7801EE0CFF1C882351
:10AE700009F10E94FA1DF701EB5AFE4F918380837E
:10AE8000000F111F000F111F04591E4FBC01990F15
:10AE9000880B990B0E945DE52AE037ED43E25CE305
:10AEA0000E94BCE5D8016D937D938D939C9313977D
:10AEB0000C9466490E94653D85E40E949D3380E3C1
:10AEC000800F0E949D33F701EB5AFE4F6081718124
:10AED00087ED9CE00E947B3F85E20E949D338AE0E3
:10AEE0000E949D330C94664985E293E10E94F631FD
:10AEF0000C9466490E94653D70E060E088EF9CE03C
:10AF00000E947B3F80912713A8E5CA2EA2E0DA2E8B
:10AF1000C81AD10887FDD394CC0CDD1CCC0CDD1CE9
:10AF20000D2C000CEE08FF088091261398E8892E5E
:10AF3000912C881A910887FD9394880C991C880C91
:10AF4000991C092C000CAA08BB088091251390E0DD
:10AF50008F3FC9F1FC01EE0FFF1FE80FF91FE05012
:10AF6000FD4E81819281E3E0880F991FEA95E1F718
:10AF7000B0E0A0E0F4E0B595A79597958795FA9590
:10AF8000D1F702969C012F5F3F4F032E000C440B1C
:10AF9000550B281939094A095B09A4EBB0E00E9456
:10AFA000C3EBA7019601281939094A095B090E94D8
:10AFB000A7EBB90185EF9CE00E947B3F8AE00E94ED
:10AFC0009D330C94664980E0DDCF0E94613DB8015D
:10AFD0008EEE9CE00E947B3F8FED9CE00E94BE3392
:10AFE0000C9466498091130490911404A091150467
:10AFF000B0911604892B8A2B8B2B29F481E00E94B7
:10B0000023400C94664980E50E94E919882311F4D5
:10B010000C9466490E94FA1D8C01892BD1F48CE4B2
:10B020000E947219882331F00E94FA1D9093E6065F
:10B030008093E50685E50E947219882311F40C942B
:10B0400066490E94FA1D9093E8068093E7060C94E7
:10B0500066490E94613DB8018FE09DE00E947B3F00
:10B0600080E09DE00E94BE330C94664980E50E941A
:10B07000E919882311F40C9466490E94FA1D8C0189
:10B08000892B09F431CF0E94653DB80185E29DE02E
:10B090000E947B3F86E19DE00E94BE330C9466498E
:10B0A00083E50E94E91981110C94C24D8091150429
:10B0B00087FD14C080911604837081F40E94653D61
:10B0C00040913013509131136091321370913313CA
:10B0D0008CE29DE00E9428340C94664982E50E942F
:10B0E00072198111EBCF0C94664983E50E94E9192E
:10B0F00004E011E0882319F00E94AF1D8B0180E568
:10B100000E94E919882369F00E94AF1DCB016938BC
:10B11000734110F088E893E1B8010E94738B0C949E
:10B12000664988EE93E0F8CF8091130483FD09C04F
:10B1300080911404817829F481E00E946D3D0C9483
:10B14000664980E50E94E919882351F00E94091E92
:10B15000609398127093991280939A1290939B1215
:10B1600089E40E94E919882381F00E94091E2CEAD3
:10B1700035EC47E25EE30E94BCE560939C1270935D
:10B180009D1280939E1290939F1284E40E94E9196D
:10B19000882311F40C9466490E94091E20E030E5D2
:10B1A00043EC50E40E94BCE56093A0127093A1129E
:10B1B0008093A2129093A3120C94664983E50E9497
:10B1C0007219182F882369F00E94FA1D9C01909330
:10B1D00071018093700191E0232B09F090E090932E
:10B1E0007F1280E50E947219882361F0209170011E
:10B1F00030917101232B11F00E94DA1D80937F1290
:10B200000C94664911110C9466490E94653D86E6CE
:10B210009DE00E94BE3380917F12882391F08EE4DE
:10B220009DE00E94BE33609170017091710185E5CF
:10B230009DE00E947B3F81E59DE00E94BE330C941F
:10B2400066498AE49DE0EDCF0E942B340C94664958
:10B2500083E50E94721981110C94664981E00E9475
:10B260007E870E94A4850C9466490E94CE3D0C9472
:10B270006649A3940C949C4E0E94613D89E99DE02F
:10B280000E94BE330C9466490E94579C0C946649F8
:10B290000E9429A60C9466490E9474860C94664903
:10B2A00061E083E50E94E91D91E089270E944071D9
:10B2B0000C9466498091B71482FF0CC087FD0AC0C8
:10B2C0000E94E82B9091B71480FB97F99093B714E4
:10B2D0000C94664984FD02C00C9466490E949AD27F
:10B2E0000C946649409028135090291360902A13BB
:10B2F00070902B1380912C1390912D13A0912E13ED
:10B30000B0912F138CA39DA3AEA3BFA3C090301305
:10B31000D0903113E0903213F090331388E50E94FF
:10B32000E919182F882309F482C00E94091E4B01D5
:10B330005C0120E030E041E653EC0E9414EE87FD12
:10B340000BC020E030E041E653E4C501B4010E94A7
:10B3500057E518160CF06DC061EE70E08AEF9DE0C5
:10B360000E947B3F61EE70E085EF9DE00E947B3F95
:10B3700082EF9DE00E94BE3310E089E50E94E9194A
:10B38000882341F10E94091E4B015C0120E030E05E
:10B3900041E653EC0E9414EE87FD0BC020E030E044
:10B3A00041E653E4C501B4010E9457E518160CF0BC
:10B3B00043C061EE70E08FED9DE00E947B3F61EE47
:10B3C00070E08AED9DE00E947B3F87ED9DE00E944A
:10B3D000BE3310E08AE50E94E919882391F10E94AA
:10B3E000091E6B017C0120E030E040EA51EC0E9434
:10B3F00014EE87FD0AC020E030E040EA51E4C701C6
:10B40000B6010E9457E51816E4F46CEE7FEF85EC68
:10B410009DE00E947B3F64E170E080EC9DE00E9433
:10B420007B3F8DEB9DE00E94BE330C94664911E09A
:10B43000A4CF24013501A1CF8CA29DA2AEA2BFA2B0
:10B44000C9CF112311F40C946649409228135092ED
:10B45000291360922A1370922B138CA19DA1AEA187
:10B46000BFA180932C1390932D13A0932E13B09310
:10B470002F13C0923013D0923113E0923213F09216
:10B4800033130C94664983E080932C071092771055
:10B4900060E083E50E94E91D81110C9466490E94D9
:10B4A000F8BF0C9466490091190410911A040E9487
:10B4B00095CA60931C0470931D0480931E0490939E
:10B4C0001F04002311F40C9466490E94653D84E535
:10B4D0000E949D33802F0E94182880E20E949D3395
:10B4E0008DE29EE00E94BE330C94664911110FC09C
:10B4F00011E08091130490911404A0911504B0916F
:10B5000016043B2F3170B32E13130C9465488C2D09
:10B510008170B12E18130C94654811E0BB24B394CC
:10B520009924939482E50E94E919882311F40C94DC
:10B53000C6490E94091E68A379A38AA39BA320E0A1
:10B5400030E0A9010E9457E5882359F0111105C088
:10B55000B11003C0992009F427C1CE0180960E9442
:10B56000EDC0112309F48AC0BB2009F484C01092F5
:10B570007201109273011092740110927501109271
:10B5800076011092770110927801109279010E9451
:10B590007E8584E59CE10E9497276B017C0188E50C
:10B5A0009CE10E9497272B013C01AC019B01C70144
:10B5B000B6010E9414EE181614F00C94CC49A701A1
:10B5C0009601C301B2010E94EFEC9B01AC010E9405
:10B5D000BCE520E030E040E85FE30E9475EC0E94AB
:10B5E00053EE21E030E048E452E40E94BCE5698378
:10B5F0007A838B839C8380917A0190917B01A091C7
:10B600007C01B0917D018CA39DA3AEA3BFA320E0DC
:10B6100030E040EC5FE3C301B2010E94BCE52B01C6
:10B620003C0177FA709477F8709420E030E040ECB9
:10B630005FE3C701B6010E94BCE59058DE01119698
:10B640006D01ECA0FDA00EA11FA1A30192010E941B
:10B650004C840E941789109272011092730110920B
:10B660007401109275011092760110927701109278
:10B6700078011092790180E00E94EC87BB2019F0DC
:10B6800081E00E94EC87992009F48EC083E00E943B
:10B69000C280811189C00E947E8580917A0190913B
:10B6A0007B01A0917C01B0917D0180938F049093E8
:10B6B0009004A0939104B0939204009134131091DC
:10B6C0003513F801C080D180E280F380A701960194
:10B6D00060E070E080EE92E40E9474EC609383047A
:10B6E000709384048093850490938604D801149603
:10B6F0004D905D906D907C901797A301920160E052
:10B7000070E080EE92E40E9474EC60938704709382
:10B7100088048093890490938A042DE030E044EEFD
:10B7200052E4C301B2010E9414EE181614F40C94F2
:10B73000D2492EE030E042EE52ECC301B2010E9449
:10B7400057E587FF02C00C94D2492DE030E04EEE61
:10B7500052E4C701B6010E9457E5181614F40C9480
:10B76000D2492EE030E042EE52ECC701B6010E9411
:10B7700014EE87FF02C00C94D2491C8E1D8E1E8EC3
:10B780001F8E88E0E3E8F4E0DE01119601900D924F
:10B790008A95E1F7BE01645E7F4FCE0101960E945B
:10B7A00032C482E00E94EC870E947E858091E2068E
:10B7B0008093E306AA2019F081E00E94F5290E94F7
:10B7C000148483E0809367010E94A4850C946649E9
:10B7D00083E50E94E919882311F40C94E8510E9432
:10B7E000AF1D8B010C94E8510E94613D89E79DE0FB
:10B7F0000E94BE330C946649882309F479CE8DCE1D
:10B80000B0E0A0E0E6E0FCE50C943FEC7C014DB636
:10B810005EB660906C0770906D078DB69EB66AE05C
:10B8200070E0C7010E9494E46C018C010E191F099D
:10B83000892B21F4C7010E94A6E48C01C80101965E
:10B840002DB73EB7281B390B0FB6F8943EBF0FBE7D
:10B850002DBF8DB79EB701965C01A801B7010E946C
:10B86000C7E4F501E00FF11F1082C5010E943B26DD
:10B8700081E00E94C647C114D10451F076019FEFC8
:10B88000E91AF90A0FB6F8949EBE0FBE8DBEC5CF59
:10B890000FB6F8949EBE0FBE8DBEC3010E943B261C
:10B8A0000FB6F8945EBE0FBE4DBEE0E10C945BECAB
:10B8B000AEE3B0E0EEE5FCE50C943DEC0E9495CAE9
:10B8C00060931C0470931D0480931E0490931F04C6
:10B8D00080919F04811145C08091130490911404BC
:10B8E000A0911504B09116043DE0B695A7959795E3
:10B8F00087953A95D1F780FF03C08CE595E080DF0E
:10B9000087E00E94C280811133C080919F04888BA0
:10B910008091130490911404A0911504B091160421
:10B92000AC01BD0126E176956795579547952A9517
:10B93000D1F740FFECC020E030E0A9016091A00405
:10B940007091A1048091A2049091A3040E9457E5F4
:10B95000811112C00E94613D8AE495E00E94BE33CD
:10B9600007C060E08FE40E94E91D882309F4B4CF8A
:10B97000EE96E2E10C9459EC8AE50E94E9198823DD
:10B98000E9F00E94091E6B017C0120E030E040E2FA
:10B9900051ECC701B6010E9457E587FD0AC020E0BF
:10B9A00030E040E251E4C701B6010E9414EE1816DF
:10B9B00074F40E94613D8DE395E0D0CFC0907A0190
:10B9C000D0907B01E0907C01F0907D01DECF40E0E3
:10B9D00050E060EC7FE788E50E94311E2B013C01BE
:10B9E00040E050E060EC7FE789E50E94311E6FA7E0
:10B9F00078AB89AB9AAB6FEF89E40E94D01D6FEFF3
:10BA00008AE40E94D01D8BA09CA0ADA0BEA020E027
:10BA100030E040E05FE3C501B4010E94BCE5209145
:10BA200093043091940440919504509196040E949F
:10BA300074ECA30192010E9475ECA50194010E948F
:10BA4000EFEC0E9457ED2B013C01162F8FA098A41C
:10BA5000A9A4BAA420E030E040E05FE3C501B4014E
:10BA60000E94BCE52091970430919804409199047C
:10BA700050919A040E9474EC2FA538A949A95AA99B
:10BA80000E9475ECA50194010E94EFEC0E9457ED15
:10BA9000062F042C000C550857FC31C027E0421635
:10BAA00051047CF5062E000C770B77FD2CC0673017
:10BAB00071055CF5173008F05BCF073008F058CF00
:10BAC00080E00E94F52937E01302F0011124E00F15
:10BAD000F11D07FDFA95EE0FFF1FEE0FFF1FE0555A
:10BAE000FB4FC082D182E282F38288890E94F529CD
:10BAF0008889882309F43CCF0E94A48539CF10E0BF
:10BB0000D1CF16E0CFCF00E0D5CF06E0D3CFE9E02C
:10BB1000B695A79597958795EA95D1F780FD0CC0C6
:10BB200070E060E086E50E94FD1D9A838983059799
:10BB300030F088E195E012CF0E94372A19CF60E0FB
:10BB400084E40E94E91D8F8740E050E0BA018AE555
:10BB50000E94311E6BA77CA78DA79EA740E050E6F0
:10BB600069EF75E483E50E94311E29E838E848E86A
:10BB70005CE30E94BCE56093680170936901809367
:10BB80006A0190936B01E0903413F0903513D70164
:10BB90004D905D906D907C9020E030E040EE50E460
:10BBA000C301B2010E9474EC4B015C0120E030E063
:10BBB00040E251E40E9414EE87FF06C0812C912CD4
:10BBC00070E2A72E71E4B72E20E030E041E653E4A6
:10BBD000C301B2010E9475EC6BAB7CAB8DAB9EAB2D
:10BBE00020E030E047E553E40E9457E5181644F49E
:10BBF00080E090E0A7E5B3E48BAB9CABADABBEAB14
:10BC0000D7011496CD90DD90ED90FC90179720E031
:10BC100030E040E050E4C701B6010E9474EC2B0113
:10BC20003C0120E030E040E251E40E9414EE87FF46
:10BC300006C0412C512C60E2662E61E4762E20E095
:10BC400030E041E653E4C701B6010E9475EC6FA7EE
:10BC500078AB89AB9AAB20E030E047E553E40E9433
:10BC600057E5181644F480E090E0A7E5B3E48FA709
:10BC700098ABA9ABBAAB88E40E947219882309F487
:10BC8000DDC00E94091E0E9457ED6BAF7CAF8DAFE7
:10BC90009EAF6BAD7CAD77FF02C06F5F7F4F759538
:10BCA000679571956195710960597F4F072E000C5A
:10BCB000880B990B0E945DE56B017C01CFAAD8AE81
:10BCC000E9AEFAAEA30192010E9414EE87FF04C010
:10BCD0004FAA58AE69AE7AAEA5019401C701B6016C
:10BCE0000E9414EE87FF02C075016401CB8ADC8AD2
:10BCF000ED8AFE8A8FA998ADA9ADBAAD8F8B988FCA
:10BD0000A98FBA8FABADBCADBD01BB0F880B990B32
:10BD10000E945DE54B015C01A70196010E9475EC54
:10BD20006B017C012BA93CA94DA95EA90E9457E596
:10BD3000181624F4CBA8DCA8EDA8FEA8CB8EDC8EC8
:10BD4000ED8EFE8E2FA938AD49AD5AADC501B401B7
:10BD50000E9475EC6B017C012FA538A949A95AA94D
:10BD60000E9457E5181624F4CFA4D8A8E9A8FAA889
:10BD7000CF8ED8A2E9A2FAA2BE01695E7F4FCE01A2
:10BD800043960E947DC1882309F481C0BE01615E93
:10BD90007F4FCE014B960E947DC1E82E882309F487
:10BDA00076C02F89388D498D5A8D6F8D78A189A1E4
:10BDB0009AA10E9474EC2BEA3AEA4AE25EE30E94FE
:10BDC000BCE54B015C012B893C894D895E896B8DFB
:10BDD0007C8D8D8D9E8D0E9474EC2BEA3AEA4AE2AE
:10BDE0005EE30E94BCE56BA37CA38DA39EA38FA200
:10BDF00098A6A9A6BAA689819A811816190674F47C
:10BE000086EE94E00E94BE338F85882321F08CED6E
:10BE100094E00E94BE338AE00E949D330E948372A8
:10BE20000E942D8480E00E94F52981E00E947E8797
:10BE3000882381F188890E94F5299ACDB301A20156
:10BE400086E40E94311E6B017C01B501A4018CE4E3
:10BE50000E94311E6B8B7C8B8D8B9E8BCF8AD88EF4
:10BE6000E98EFA8E4FA558A969A97AA982E40E94A1
:10BE7000311E6B017C014BA95CA96DA97EA982E5ED
:10BE80000E94311E6B8F7C8F8D8F9E8F71CF8CEFB8
:10BE900094E064CD2091A0043091A1044091A204CB
:10BEA0005091A3046BA17CA18DA19EA10E9457E596
:10BEB000811130C02091A4043091A5044091A604C2
:10BEC0005091A7046FA178A589A59AA50E9457E56E
:10BED000811120C0209193043091940440919504E5
:10BEE000509196046B897C898D899E890E9457E5C3
:10BEF000811110C0209197043091980440919904C9
:10BF000050919A046F89788D898D9A8D0E9457E59A
:10BF10008823A9F00E94372A88E0FE01B396A0EAA0
:10BF2000B4E001900D928A95E1F788E0FE017396E6
:10BF3000A3E9B4E001900D928A95E1F7188A60E0D8
:10BF400085E40E94E91DCC24C394811102C043E022
:10BF5000C42E1B861C861D861E861A8ADE2C97E040
:10BF6000792E2CEAA22E24E0B22E3AEB832E34E076
:10BF7000932E8A8987300CF0A8C0DD2009F49CC07C
:10BF800066246394B7E0BFA790E021E0D226879DA6
:10BF9000F02C1124F394998B19896A89FFA51F1736
:10BFA00009F490C0062E000C770B880B990B0E94A9
:10BFB0005DE52FA138A549A55AA50E94BCE52F89AA
:10BFC000388D498D5A8D0E9475EC1B012C01612F13
:10BFD000110F770B880B990B0E945DE52BA13CA1FB
:10BFE0004DA15EA10E94BCE52B893C894D895E89EB
:10BFF0000E9475EC6B837C838D839E832F823886B1
:10C0000049865A8689819A81892B89F088EC94E047
:10C010000E94BE338F2D0E94182861E370E086ECE9
:10C0200094E00E947B3F83EC94E00E94BE331F9219
:10C0300021E32F931F92FF92BF92AF929F928F9214
:10C040001F920E94019C29814C2DBE01695F7F4F88
:10C05000CE0103960E94B3C29B01AC012B873C87A3
:10C060004D875E8709898A89672D0603800111241F
:10C07000080F111D87FD1A95000F111F000F111FCA
:10C0800000551B4F6BA57CA58DA59EA50E9475EC48
:10C09000D8016D937D938D939C931397188A81E0BB
:10C0A0000E94AF40F3948989860D898B0FB6F8946E
:10C0B000DEBF0FBECDBF70CF66246A94EFEFEFA74F
:10C0C00096E063CF6F5F6A8B54CF0E943BC10E94A2
:10C0D0009D27882359F088890E94F52980E090E007
:10C0E000A0ECBFE78B879C87AD87BE870E94F63C9C
:10C0F0000E944E2B8F85811122C08AE791E00E9419
:10C10000A0274B015C0182E791E00E941E28A50157
:10C1100094010E94BCE59B01AC0160917A01709191
:10C120007B0180917C0190917D010E9474EC609371
:10C130007A0170937B0180937C0190937D018F85C0
:10C140008111E888E0929F040E94148480919F04EA
:10C15000882309F4D1CC0E947E85CECCCF93DF9387
:10C16000C091800E81E6C89FE0011124CE57D14FC7
:10C1700080914B0D80FF05C00E94653DCE010E945D
:10C18000AF33CE010E943B2680E00E94C647DF917C
:10C19000CF910895A0E1B0E0E0EDF0E60C944BEC17
:10C1A0008C01DC01ED91FC910280F381E02DBE0158
:10C1B0006F5F7F4F0995882309F45DC08981807C7A
:10C1C00091F56F81637070E0762F6627770F770F98
:10C1D0008885B4E08B9FC0011124682B792B898559
:10C1E0008295869586958370682B6F5F7F4F90E070
:10C1F00080E02A852370220F3B8537FB332730F9F7
:10C20000232B3E813F70230F3327331F27503109E3
:10C2100004C0660F771F881F991F2A95D2F7609672
:10C22000E4E00C9467EC803419F5688566956695B2
:10C2300070E090E080E0CB01772766272A85622BAB
:10C24000098510E0102F0027012E000C220B330B64
:10C25000602B712B822B932B6F5F7F4F8F4F9F4FE4
:10C260004AE0660F771F881F991F4A95D1F7D7CFED
:10C270008BE0F801848360E070E0CB01D0CF0895BB
:10C28000FC0182810895FC0190E1A7E5B6E00190F0
:10C290000D929A95E1F70895EF92FF920F931F93F5
:10C2A000E0927605F0927705009378051093790572
:10C2B000B62F172F022FF32E242F582FB0937A0565
:10C2C00010937B0550937C056FEFFF27B01B1F0970
:10C2D000520B30F450951095B195160B560B6627FE
:10C2E0006093A002A6E0BA9F00929402712DEE27FF
:10C2F0001A9F700DE11D5A9FE00D70939502E09317
:10C300009602AFE0BA9F00929802712DEE271A9F15
:10C31000700DE11D5A9FE00D70939902E0939A020F
:10C32000AAE0BA9F00929C02712DEE271A9F700D11
:10C33000E11D5A9FE00D70939D02E0939E021F91B4
:10C340000F91FF90EF900895A5E0B0E0EAEAF1E6E2
:10C350000C9444EC6F3671058105910578F4FB016E
:10C36000EE0FFF1FEE0FFF1FE459F24E659175911E
:10C37000859194912596EBE00C9460ECF62EE72ED7
:10C38000282FECE6FCE10027BB275F2D8E2D922F96
:10C39000992341F4982F852FB85F992319F4982F8A
:10C3A0008827B85F903138F482959295582F5F7046
:10C3B000807F952BBC5F903428F4880F991F880FDD
:10C3C000991FBE5F903818F4880F991FB395880F96
:10C3D000991FE90FF01F549181E09927B85079F126
:10C3E000C0F0B0FF02C0550F881FB1FF04C0550F49
:10C3F000881F550F881FB2FF06C082955295152FD2
:10C400001F70507F812BB3FF1AC0982F852F55279F
:10C4100016C0B195B0FF02C085955795B1FF04C015
:10C420008595579585955795B2FF05C08295507FA4
:10C430005295582B8F70B3FF02C0582F8827BB240A
:10C440007727AA27B2E0F59EB0187109A00BB00BB0
:10C45000E59E7019A109B00B259FA019B109F89E9E
:10C460007019A109B00BE89EA019B109289FB01955
:10C47000F99EA019B109E99EB0195B9DA12C9924E0
:10C480004427662733278B9DA00C911C401F601FFB
:10C49000301F9B9D900C411D601F301F579FA00CAB
:10C4A000911C401F601F301F879F900C411D601F13
:10C4B000301F979F400D611D301F5A9F900C411DEA
:10C4C000601F301F8A9F400D611D301F9A9F600DB5
:10C4D000311D5B9F400D611D301F8B9F600D311D15
:10C4E0009B9F300DB1E0AA277727BB24F49EB0189C
:10C4F0007109A00BB00BE49E7019A109B00B249F29
:10C50000A019B109F69E7019A109B00BE69EA019F9
:10C51000B109269FB019F39EA019B109E39EB01985
:10C52000BF187E09A20B20F0B1E04B0F601F301F37
:10C530001124762F642F90E0832F1CCFFC01708193
:10C54000472F50E0062E02C0559547950A94E2F712
:10C5500040FF14C04091EF0550E0062E02C05595F3
:10C5600047950A94E2F740FF09C021E030E001C09E
:10C57000220F6A95EAF720952723208308958F924A
:10C580009F92AF92BF92CF92DF92EF92FF92FC0107
:10C59000C080D180E280F38020E030E048EC52E4BB
:10C5A000C701B6010E94BCE54B015C0120E030E010
:10C5B000A901C701B6010E9457E520E030E040EA3A
:10C5C00050E487FF04C020E030E040EA50ECC501B1
:10C5D000B4010E9475EC2DEC3CEC4CEC5DE30E9448
:10C5E000BCE50E9457ED9B018BE237FF05C0222777
:10C5F0003327261B370B8DE280937C04C90168EE3C
:10C6000073E00E940FECCB01EAE0F0E0BF010E9472
:10C610000FEC805D80937D04C90164E670E00E94A8
:10C620000FECCB01BF010E940FEC805D80937E0474
:10C63000C901BF010E940FEC9C01CB01BF010E9408
:10C640000FEC805D80937F048EE280938004205DF8
:10C65000209381048CE794E0FF90EF90DF90CF90DF
:10C66000BF90AF909F908F9008954F925F926F927E
:10C670007F928F929F92AF92BF92CF92DF92EF9272
:10C68000FF92FC01C080D180E280F38020E030E0A6
:10C690004AE754E4C701B6010E94BCE54B015C01C6
:10C6A00020E030E040E251ECC701B6010E9457E5BE
:10C6B000181654F420E030E048EC52E4C701B6010B
:10C6C0000E9414EE87FD8AC020E030E0A901C70176
:10C6D000B6010E9457E587FF72C060E070E080EA13
:10C6E00090ECA50194010E9475EC2DEC3CEC4CEC17
:10C6F0005DE30E94BCE50E9457ED6B017C01F7FCF5
:10C7000063C020E137E240E050E00E94A7EBCA019D
:10C71000B9012AE030E040E050E00E94A7EB605D04
:10C7200060937C04C701B60128EE33E040E050E09E
:10C730000E94A7EB9AE0892E912CA12CB12CCA0162
:10C74000B901A50194010E94A7EB605D60937D048F
:10C75000C701B60124E630E040E050E00E94A7EBBC
:10C76000CA01B901A50194010E94A7EB605D609325
:10C770007E048EE280937F04C701B601A501940177
:10C780000E94A7EB6B01CA01B901A50194010E94A7
:10C79000A7EB605D60938004F0E3CF0EC09281044C
:10C7A0008CE794E0FF90EF90DF90CF90BF90AF9038
:10C7B0009F908F907F906F905F904F90089560E072
:10C7C00070E080EA90E48DCFF094E094D094C0942F
:10C7D000C11CD11CE11CF11C6DE2A2CF20E030E0B5
:10C7E000A901C701B6010E9457E587FF6BC060E051
:10C7F00070E080EA90ECA50194010E9475EC2DECAC
:10C800003CEC4CEC5DE30E94BCE50E9457ED4B0113
:10C810005C0120E030E0A901C701B6010E9457E5A4
:10C8200087FD0BC020E030E040E251E4C701B601D3
:10C830000E9414EE60E287FD13C0B7FC48C0C5013A
:10C84000B40128EE33E040E050E00E94A7EBCA01BB
:10C85000B9012AE030E040E050E00E94A7EB605DC3
:10C8600060937D04C501B40124E630E040E050E06F
:10C870000E94A7EB8AE0482E512C612C712CCA0132
:10C88000B901A30192010E94A7EB605D60937E0451
:10C890008EE280937F04C501B401A30192010E943E
:10C8A000A7EB6B01CA01B901A30192010E94A7EB9A
:10C8B000605D6093800480E3C80EC09281048DE7C0
:10C8C00094E070CF60E070E080EA90E494CFB094A0
:10C8D000A09490948094811C911CA11CB11C6DE2C9
:10C8E000BFCF282F81E3243609F080E280937E04B5
:10C8F00090E22A3040F03AE0822F632F0E94E2EB70
:10C900000E94E2EB905D90937F04822F6AE00E9488
:10C91000E2EB905D9093800485E2809381048EE742
:10C9200094E008956091550170915601072E000C16
:10C93000880B990B0E945DE52AE037ED43E25CE34A
:10C940000E94BCE560936C0170936D0180936E0151
:10C9500090936F010895CF93DF93EC01CB01BA015F
:10C960000E945DE523E333E343E250E40E94BCE52B
:10C9700020E030E040E05FE30E9475EC0E945CED57
:10C980006883DF91CF9108950E945DE523E333E34F
:10C9900043E250E40E94BCE520E030E040E05FE389
:10C9A0000E9475EC0E945CED24E6629FC001112498
:10C9B00081589F4F6FEF70E00E940FEC862F91CF50
:10C9C00080915607811104C080912D0780938A07BA
:10C9D00008958091AD148823C1F081508093AD14E7
:10C9E000ECEDF2E1882351F08150990B2BE1289F67
:10C9F000F001299FF00D1124E156FC4E8BE1A1ECD2
:10CA0000B2E101900D928A95E1F72091AD142111C8
:10CA100005C08091B71480648093B71481E090E0E2
:10CA2000A0E0B0E0211103C080E090E0DC01809341
:10CA30004C0790934D07A0934E07B0934F07109269
:10CA4000470781E08093490783E080936701089559
:10CA5000CF93DF93EC01CB01BA010E945DE56883BF
:10CA600079838A839B83DF91CF910895CF93DF935E
:10CA7000EC01CB01BA010E945DE52DEC3CEC4CECE5
:10CA80005DE30E94BCE5688379838A839B83DF91A1
:10CA9000CF910895CF93DF93EC01CB01BA010E94AF
:10CAA0005DE52AE037ED43E25CE30E94BCE5688384
:10CAB00079838A839B83DF91CF910895CF92DF9210
:10CAC000EF92FF92CF93DF9300D000D0CDB7DEB7C7
:10CAD0000E945DE52AE037ED43E25CE30E94BCE59D
:10CAE0006B017C0120E030E0A9010E9457E52DEBAD
:10CAF00037E346E055E387FF04C02DEB37E346E01C
:10CB000055EBC701B6010E9475EC69837A838B836C
:10CB10009C83CE010196A9DD0F900F900F900F908E
:10CB2000DF91CF91FF90EF90DF90CF900895CF935A
:10CB3000DF93EC01CB01BA010E945DE50E9457ED45
:10CB400079836883DF91CF9108958F929F92AF92FE
:10CB5000BF92CF92DF92EF92FF92FC01C080D18012
:10CB6000E280F38020E030E0A901C701B6010E9415
:10CB700057E587FD99C06DEB77E386E095E3A70164
:10CB800096010E9475EC9F7720E030E048EC52E47B
:10CB90000E94BCE520E030E040EA50E40E9475ECE1
:10CBA0002DEC3CEC4CEC5DE30E94BCE50E9457EDA3
:10CBB0006B017C0180E280937B0460E2F0E1CF16A0
:10CBC000F7E2DF06E104F1048CF0C701B60120E1D1
:10CBD00037E240E050E00E94A7EBCA01B9012AE029
:10CBE00030E040E050E00E94A7EB605D60937C0481
:10CBF00060E288EEC81683E0D806E104F1048CF008
:10CC0000C701B60128EE33E040E050E00E94A7EBF8
:10CC1000CA01B9012AE030E040E050E00E94A7EBF1
:10CC2000605D60937D0460E2E4E6CE16D104E10429
:10CC3000F1048CF0C701B60124E630E040E050E09A
:10CC40000E94A7EBCA01B9012AE030E040E050E0C1
:10CC50000E94A7EB605D60937E048AE0882E912C91
:10CC6000A12CB12CC701B601A50194010E94A7EB2C
:10CC70006B01CA01B901A50194010E94A7EB605D97
:10CC800060937F048EE280938004F0E3CF0EC09225
:10CC900081048BE794E0FF90EF90DF90CF90BF90FE
:10CCA000AF909F908F9008956DEB77E386E095EBC2
:10CCB00066CFA4E0B0E0EFE5F6E60C944DEC0E9400
:10CCC0005DE52DEC3CEC4CEC5DE30E94BCE569833A
:10CCD0007A838B839C83CE01019637DF2496E2E032
:10CCE0000C9469ECCF93DF93EC018D810E949E4000
:10CCF00060E08B810E94ADC9DF91CF910895CF9202
:10CD0000DF92EF92FF920F931F93CF938C01C62F68
:10CD100069017A01E7DF0E947FCB8C2F80640E943B
:10CD200092408F2D0E9492408E2D0E9492408D2D18
:10CD30000E9492408C2D0E94924087E8C11101C050
:10CD400085E90E949240CC3011F40E949740C0E0E7
:10CD50000E949740F801868387FF04C0CF3F11F0FF
:10CD6000CF5FF6CFCF911F910F91FF90EF90DF90A3
:10CD7000CF90089561E0FC0183810E94ADC98FEFDF
:10CD80000C9492400F931F93CF938C01ABDF0E94C2
:10CD90007FCBC82F882369F08DEF0E9492400E94BC
:10CDA0007FCBC82FC801E6DF8C2FCF911F910F9149
:10CDB000089582E1F8018483F5CFB0E0A0E0E3EECE
:10CDC000F6E60C9443ECEC016A017B014801590141
:10CDD00020E030E0A90167E392DFA501980167E157
:10CDE000CE018DDF81111DC08F81833039F089E044
:10CDF000CC0CDD1CEE1CFF1C8A95D1F7A701960117
:10CE000069E1CE017CDF11E0882319F010E087E0B2
:10CE10008C83CE01AFDF812FCDB7DEB7ECE00C9471
:10CE20005FEC89E08C8310E0F4CFCF93DF93EC01CB
:10CE30006EBDFA01CA019E5F0DB407FEFDCF2081D1
:10CE40002EBD0DB407FEFDCF21812EBD3296E81711
:10CE5000F90791F70DB407FEFDCF8FEF0E949240C6
:10CE60008FEF0E9492400E9497408E838F71853091
:10CE700041F083E18C83CE017DDF80E0DF91CF91B3
:10CE8000089581E0FBCF0F931F93CF93DF93EC01C5
:10CE90008B0128DF0E947FCB81110BC085E18C8341
:10CEA00010E0CE0167DF812FDF91CF911F910F91AD
:10CEB0000895A8016CEFCE01B8DF182F882371F315
:10CEC000F0CF0F931F93CF93DF93EC0189018F81F4
:10CED000833039F089E0440F551F661F771F8A950C
:10CEE000D1F79A01AB0168E1CE0109DF811127C0BA
:10CEF000A8016EEFCE0199DF182F8823A9F00E94B8
:10CF00007FCB182F8823C1F020E030E0A9016DE02D
:10CF1000CE01F5DE882321F086E18C8310E004C089
:10CF20000E9497408111F8CFCE0124DF812FDF913D
:10CF3000CF911F910F91089587E18C83F5CF86E003
:10CF4000ECCF1F93CF93DF93EC01CCDE20E030E0F9
:10CF5000A9016CE0CE01D3DE11E0882319F010E0C6
:10CF600083E08C83CE0106DF812FDF91CF911F916B
:10CF700008951F93CF93DF93EC018F81833039F0B5
:10CF800089E0440F551F661F771F8A95D1F79A01D4
:10CF9000AB0162E1CE01B3DE11E0882319F010E0AD
:10CFA00085E08C83CE01E6DE812FDF91CF911F914A
:10CFB00008958F929F92AF92BF92EF92FF920F933C
:10CFC0001F93CF93DF938C01EB017A010E9495CAE6
:10CFD0004B015C012CE2820E21E0921EA11CB11CCF
:10CFE0000E949740F80186838F3F69F40E9495CA9A
:10CFF000681979098A099B0997FDF2CF81E1F80147
:10D000008483C0E021C08E3F69F5F1E0EF1AF1089A
:10D010008FEF8EBDFE012FEF0DB407FEFDCF8EB555
:10D0200081932EBDCF018C1B9D0B8E159F05A0F308
:10D030000DB407FEFDCF8EB5CE0DDF1D88830E9497
:10D0400097400E949740C1E0C80194DE8C2FDF9189
:10D05000CF911F910F91FF90EF90BF90AF909F9055
:10D060008F9008958FE0CBCF0F931F93CF93DF93D3
:10D07000EC018B0137DE40E052E0B801CE0199DFD0
:10D08000DF91CF911F910F9108950F931F93CF932D
:10D09000DF93EC0189018F81833039F089E0440FFF
:10D0A000551F661F771F8A95D1F79A01AB0161E181
:10D0B000CE0125DE882351F084E08C83CE015ADE38
:10D0C00080E0DF91CF911F910F91089540E052E0F1
:10D0D000B801CE016EDFF5CFB0E0A0E0E2E7F8E600
:10D0E0000C9443ECEC01162F1F821C824B830E9490
:10D0F00095CA6B017C0120EDC20E27E0D21EE11C17
:10D10000F11CA89561E08B810E94ADC98B810E94C2
:10D1100042B0249A2C9A279A2698259A81E00E9458
:10D120009E4085E08D830E949E400AE08FEF0E9422
:10D1300092400150D9F7A89520E030E0A90160E0C5
:10D14000CE01DDDD8E83813079F00E9495CA6C19A5
:10D150007D098E099F0997FDEFCF81E08C83CE0179
:10D1600009DE1A8280E065C0A8952AEA31E040E035
:10D1700050E068E0CE01C3DD853031F581E08F837A
:10D18000A8958F81812C912C5401823029F4812C17
:10D19000912CA12C80E4B82E20E030E0A90167E3B7
:10D1A000CE01ADDDA501940169E2CE01A8DD8E833B
:10D1B0008823F1F00E9495CA6C197D098E099F0998
:10D1C00097FDEACF8AE0CACF04E00E9497408E83A1
:10D1D0000150D9F78A3A11F482E0D1CF0E9495CA62
:10D1E0006C197D098E099F0997FDBFCF82E0B6CFEC
:10D1F0008F818230B9F420E030E0A9016AE3CE01EA
:10D200007EDD882311F088E0A9CF0E949740807CC2
:10D21000803C11F483E08F830E9497400E949740E6
:10D220000E949740CE01A6DD81E08A83173030F45A
:10D230001D83CDB7DEB7ECE00C945FEC88E18C8306
:10D2400091CF0F931F93CF93DF93EC018B0120E0DD
:10D2500030E0A90169E053DD882351F080E18C833F
:10D26000CE0188DD80E0DF91CF911F910F9108956D
:10D2700040E150E0B801CE019CDEF5CFCF93C82F3E
:10D28000CB010E94BE3388EA9BE10E94BE3389E94C
:10D290009BE1CC2311F08EE99BE10E94BE338AE032
:10D2A0000E949D33CF9108950C94A1CA40917405BA
:10D2B00021E042276CE070E00C9416B040917405B8
:10D2C00021E0422764E070E00C9416B040917405B0
:10D2D00021E0422761E070E00C9416B040917405A3
:10D2E00021E0422761E070E00C9416B04091740593
:10D2F00021E0422768E070E00C9416B0409174057C
:10D3000021E042276CE070E00C9416B041E061E04F
:10D3100070E00C9416B04091740521E042270C9403
:10D3200016B06CE070E00C943CCA61E070E00C94C4
:10D330003CCA6CE070E00C943CCA64E070E00C9471
:10D340003CCA90919F0481E089270C94F52961E003
:10D350008DE297E00C94812A20E030E0A901BC0125
:10D3600082E791E00C9450C080E090E0A0E8B0E447
:10D3700080937A0190937B01A0937C01B0937D010F
:10D3800083E492E0E9DF80E090E0A0EFB1E48093F5
:10D39000720190937301A0937401B093750180930F
:10D3A000760190937701A0937801B0937901E09191
:10D3B000CC05EE0FFF0BED5DFD4F80819181833039
:10D3C000910539F184309105C9F1029761F480E04B
:10D3D00090E0A3E4B3E48093720190937301A0936F
:10D3E0007401B09375018BE292E0B6DF10927A017E
:10D3F00010927B0110927C0110927D0183E492E0F7
:10D40000ABDF8091CC058F5F8430ECF48093CC054A
:10D41000089580E090E0A3E4B3E4809372019093D8
:10D420007301A0937401B09375018093760190937A
:10D430007701A0937801B0937901D5CF80E090E097
:10D44000A3E4B3E4F2CF1092CC050895B0E0A0E0DD
:10D45000ECE2FAE60C944DEC20E24F8158856E81A7
:10D460008D810E9460C5E2E00C9469EC80912D07EB
:10D4700090912E070C94D6CA6CE174E982E00C946A
:10D480006EC760E274E981E00C946EC764E274E9EF
:10D4900080E00C946EC768E274E983E00C946EC778
:10D4A000109247070C94B5D54FE350E06DED79E14C
:10D4B0008CEE96E00C9429EF8091391390913A13F9
:10D4C000891B8F7011F40C94D52B81E00895809105
:10D4D0006701882341F06091C4057091C50541E062
:10D4E00081E00C9400C50895CF93DF93EC010E9476
:10D4F00067D21B82DF91CF910895CF93DF93EC0128
:10D50000462F41706C857D858E859F850E9478CFE2
:10D51000882351F0888920E2829FC0011124885815
:10D520009F4EDF91CF91089590E080E0FACFCF93A6
:10D53000DF93EB01FC012381211104C080E0DF9126
:10D54000CF9108952250223028F48FE288831982E7
:10D5500081E0F5CF60E0D1DF009781F3DC0160E08E
:10D5600080E09EE22D91203299F0883031F49E01C6
:10D57000260F311DF90190836F5F9E01260F311D2B
:10D58000AD0141505109FA014081F90140836F5FBB
:10D590008F5F8B3039F7FE01E60FF11D1082D8CF77
:10D5A000ACE0B0E0E6EDFAE60C943EEC5C01DC01A8
:10D5B00059968D909C90F40181859285A385B485C0
:10D5C0009C01AD012F5F3F4F4F4F5F4F29873A8737
:10D5D0004B875C87D50114964D905D906D907C9043
:10D5E0001797411451046104710409F459C0BFEF45
:10D5F0004B1A5B0A6B0A7B0A312C730162011D8294
:10D600001E821F821886F40181859285A385B485C8
:10D610002D813E814F815885281739074A075B07BE
:10D6200008F056C089859A85AB85BC858C159D050B
:10D63000AE05BF0550F482E0C82ED12CE12CF12CB0
:10D6400092E0492E512C612C712C9E012F5F3F4F8F
:10D65000B701A601C4010E9482D18823C9F1898142
:10D660009A81AB81BC81892B8A2B8B2B01F12601FE
:10D6700037019FEF491A590A690A790A2D813E81BB
:10D680004F8158852F5F3F4F4F4F5F4F2D833E8314
:10D690004F8358873FEFC31AD30AE30AF30AB3CF85
:10D6A000408051806280738033243394A6CFC414A9
:10D6B000D504E604F70411F70FEF1FEF2FEF3FE05B
:10D6C000B701A601C4010E9408D1782E811106C0BD
:10D6D000712C872D2C96E1E10C945AECF5014481D4
:10D6E000558166817781411551056105710539F0D4
:10D6F00097018601C4010E9408D1882349F3D5010E
:10D700001496CD92DD92ED92FC921797332051F052
:10D71000D701C6010196A11DB11DF401808391833B
:10D72000A283B383F50185899689A789B08D892B5A
:10D730008A2B8B2B71F6C58AD68AE78AF08E818177
:10D7400080688183C6CF40E050E0BA010C94B0D22B
:10D750004F925F926F927F92AF92BF92CF92DF9281
:10D76000EF92FF920F931F93CF93DF931F92CDB74A
:10D77000DEB78C017B015A01C22EDB0159968D91D7
:10D780009C91F801928F818FCB01DDDF712CF70125
:10D7900080859185A285B385418952896389748981
:10D7A00084179507A607B70708F052C055E0B6954D
:10D7B000A795979587955A95D1F7F82FFF70DF2E8B
:10D7C000D70113968C91823010F480E0DAC041E0EA
:10D7D00050E0BE016F5F7F4FC7010E94ABD301973E
:10D7E000A1F7F70180859185A285B3854F96A11D8C
:10D7F000B11D80879187A287B387F0E2DF9EB001D9
:10D80000112468587F4E61157105F9F2DB018C9186
:10D81000882341F0853E09F04BC0772029F077241A
:10D820007394B5CF71100EC08091781290917912D7
:10D83000A0917A12B0917B12F80184879587A68710
:10D84000B787D08ADB018C918111E9CF772473945B
:10D850008C2D8274823409F0B8CF772009F4A1C0EE
:10D86000F801D08861E0C80148DE009709F4ADCF27
:10D8700020E2DC011D922A95E9F72BE0F501DC019D
:10D8800001900D922A95E1F721E238E2FC01318BFB
:10D89000208B40E058E057874687338B228B318FAF
:10D8A000208F578B468B0E942FCF811109C08DCFBF
:10D8B0004BE050E0C5010E94D9EE892B09F067CFFB
:10D8C000F0E2DF9ED00111249D0128583F4EF9015E
:10D8D0008385817121F08C2D827109F000C1F801DE
:10D8E000818D928D409178125091791260917A12C7
:10D8F00070917B124487558766877787D08AFD01B0
:10D90000E858FF4E44885588712C612C320155240B
:10D910004424D80155964D925D926D927C92589711
:10D92000428D538D70E060E044295529662977299E
:10D9300055964D935D936D937C935897D9011B96A3
:10D940002C91287109F0BDC0848D958DA68DB78D61
:10D95000F801818B928BA38BB48B81E083838C2D18
:10D960008F70F801818314821582168217821086C7
:10D9700011861286138681E0C4FE03C0C8010E948E
:10D9800035D30F90DF91CF911F910F91FF90EF90C2
:10D99000DF90CF90BF90AF907F906F905F904F904F
:10D9A0000895D70113968C911397823009F40DCF07
:10D9B00051968D919D910D90BC91A02D803E9F4FD1
:10D9C000AF41B10508F001CFC701EADD882309F4B2
:10D9D000FCCE0E942FCF882309F4F7CED7015996A9
:10D9E000ED91FC915A9714964D905D906D907C90BE
:10D9F0001797B2E04B1A510861087108858504C079
:10DA0000440C551C661C771C8A95D2F78685978531
:10DA1000A089B189480E591E6A1E7B1E81E0809341
:10DA20007C12409278125092791260927A1270921F
:10DA30007B12E8E7F0E180E092E0DF019C011D92BB
:10DA400021503040E1F7DD24D394D7015996ED9170
:10DA5000FC918481D816C0F480917D1290917E1241
:10DA6000DC01ED91FC910288F389E02D28E730E19B
:10DA7000B301A2014D0D511D611D711D0995882332
:10DA800009F4A3CED394E1CF258580E092E0A0E015
:10DA9000B0E004C0880F991FAA1FBB1F2A95D2F7B8
:10DAA000F7014189528963897489840F951FA61FE4
:10DAB000B71F818B928BA38BB48B88E790E1D12C1D
:10DAC000D7CE203161F498012F5E3F4F0E94FED1E6
:10DAD000882329F084E0D80113968C9340CFD80195
:10DAE00013961C9272CEFC0123812111FDCC089566
:10DAF000A1E4B0E0EEE7FDE60C943DEC4C015B01E7
:10DB00007A01222E19821C821C8E1F8E61157105CE
:10DB100069F410E0CE014C96E6DFCE010196E3DF1A
:10DB2000812FCF5BDF4FE2E10C9459ECFC01838144
:10DB30008111EFCFFA0180818F3251F18B01CE013B
:10DB400001966C012C0180E2382E360122963FAE00
:10DB5000229721963FAE21973FAE3EAE3DAE3CAE02
:10DB60003BAE3AAE39AE38AE3FAA970190E047E0FF
:10DB7000D9018D91882309F447C08F3209F444C03C
:10DB80008E3209F54A3029F298E04AE09D01F0CF43
:10DB9000FB01838182508230A0F0618D728DCE01B5
:10DBA0004C960E9466D5882309F4B3CF8E01045E9B
:10DBB0001F4FC7017C010196F70120812F32D1F35D
:10DBC000BECF8B01F6CFE7EDF9E22491222321F0BD
:10DBD00031968213FACF9DCF491708F49ACF81323C
:10DBE00008F497CF8F3709F494CF3FE9380F3A31D3
:10DBF00008F420EEE7E3F0E0EC0FFD1FE90FF11D64
:10DC0000820F80839F5FC2CF8FA9803209F481CFBA
:10DC10007901F90180812F5F3F4F8F32C9F388234B
:10DC2000C1F021E0AE01495C5F4FB801C60190DD53
:10DC3000882309F46ECF0A151B0511F0C80154DCC6
:10DC4000CE014C964C145D0409F0C30186016C01B1
:10DC50007DCF222DAE01495C5F4FB801C40178DD54
:10DC6000182F58CF8F929F92AF92BF92CF92DF9290
:10DC7000EF92FF920F931F93CF93C82F0DE812E1FD
:10DC8000F80160857185072E000C880B990B0E94A6
:10DC90005DE56B017C01F80184809580A680B780EA
:10DCA00080E20E949D3384E50E949D338AE30E94B6
:10DCB0009D3342E0C501B4010E9461B080ED99E25C
:10DCC0000E94BE3342E0C701B6010E9461B062E02B
:10DCD00070E080E090E00E9409CA87E1C802F0018C
:10DCE0001124E357FD4E628570E083ED99E20E94B6
:10DCF0007B3FCF911F910F91FF90EF90DF90CF90DE
:10DD0000BF90AF909F908F9008950F930FB70F9390
:10DD100000916E000B7F00936E0078940F930BB709
:10DD20000F930CB70F921F922F933F934F935F93D4
:10DD30006F937F938F939F93AF93BF93EF93FF93D3
:10DD400011240E94ECA1FF91EF91BF91AF919F919F
:10DD50008F917F916F915F914F913F912F911F9084
:10DD60000F900CBF0F910BBF0F910460F8940093BC
:10DD70006E000F910FBF0F911895CF93DF93109204
:10DD80007E05CDE8D2E1198618860E94A1CA1A86BE
:10DD90005D98DF91CF910895EF92FF920F931F93BB
:10DDA000CF93C82F7B018A0180912C078330E0F04C
:10DDB0000E94613DC7010E94BE3386E599E20E9440
:10DDC000BE33C7FD0EC084E599E20E94BE336C2FBE
:10DDD000CC0F770B880B990B0E9417AE8AE00E943C
:10DDE0009D338AE00E949D33C8DFA8958091670625
:10DDF000811128C081E08093670682E080932C0720
:10DE0000BCDFC5E1C150149AB9F069E170E080E06F
:10DE100090E00E9409CAA895149868E270E080E03A
:10DE200090E00E9409CAA89568E270E080E090E066
:10DE30000E9409CAA895E6CF40E061E579E2C801F1
:10DE40000E94893FCF911F910F91FF90EF9008950D
:10DE5000CF93DF93A89580918F12909190120E949A
:10DE60008FAF60939112709392128093931290935C
:10DE70009412C0918F12D091901280916001909174
:10DE80006101C817D90734F442E959E26FE979E230
:10DE900080E082DF809195129091961218161906F3
:10DEA0006CF480915E0190915F018C179D0734F4B2
:10DEB00041EB59E26EEB79E280E06EDFDF91CF91CA
:10DEC00008958F929F92AF92BF92CF92DF92EF927E
:10DED000FF92CF93DF9300D000D0CDB7DEB7809113
:10DEE0002C07811110C0A8950F900F900F900F90E4
:10DEF000DF91CF91FF90EF90DF90CF90BF90AF90E8
:10DF00009F908F900895809168068111EDCF81E0F8
:10DF10008093680680917F05811103C01092680686
:10DF2000E3CF96DF10927F050E9495CA6B017C01BA
:10DF30000E9432AE4B015C016091640170916501F9
:10DF4000072E000C880B990B0E945DE59B01AC012C
:10DF5000C501B4010E9414EE18160CF469C060915A
:10DF6000951270919612072E000C880B990B0E9447
:10DF70005DE569837A838B839C83CE0101960E9441
:10DF8000E0CA8090911290909212A0909312B0905B
:10DF900094126091620170916301072E000C880B4E
:10DFA000990B0E945DE59B01AC01C501B4010E9483
:10DFB00014EE1816CCF46091640170916501072E7F
:10DFC000000C880B990B0E945DE59B01AC01C5011B
:10DFD000B4010E9457E587FF07C00E943BAE0E9434
:10DFE00057ED7595679501C060E060939712809139
:10DFF000891290918A12A0918B12B0918C12009785
:10E00000A105B10509F48ACFC81AD90AEA0AFB0AA0
:10E01000F7FC84CF0E9432AE0E9457ED2091871208
:10E02000309188126217730754F00E94A1CA76CF0C
:10E0300042E959E26FE979E280E0AEDE90CF44E751
:10E0400059E263E879E280E0A7DE68CFCF92DF9201
:10E05000EF92FF92CF93DF93EC01C880D980EA80E2
:10E06000FB8087E499E20E94BE33C701B6010E949B
:10E070003926CC80DD80EE80FF8085ED9FE20E9416
:10E08000BE33C701B6010E943926C884D984EA8408
:10E09000FB8481ED9FE20E94BE33C701B6010E945E
:10E0A00039268AE00E949D33DF91CF91FF90EF9057
:10E0B000DF90CF900895BC01209148063091490629
:10E0C00040914806509149062417350731F481E004
:10E0D0002617370709F080E008959A01F1CF0F93D2
:10E0E0000FB70F9300916E000F930B7F00936E009C
:10E0F00000916F000D7F00936F000F930BB70F938C
:10E100000CB70F921F922F933F934F935F936F9390
:10E110007F938F939F93AF93BF93EF93FF931124BC
:10E12000B8D5FF91EF91BF91AF919F918F917F9162
:10E130006F915F914F913F912F911F900F900CBF66
:10E140000F910BBF0F910260F89400936F000F9135
:10E1500000936E000F910FBF0F91189500C000C083
:10E160008091E40680FF1FC0459A8FEF80930106DF
:10E170008091E40681FF1AC0479A8FEF80930206D0
:10E180008091E40682FF15C02A988FEF80930306E2
:10E190008091E40683FF10C028988FEF80930406D7
:10E1A00000C000C00895459881E0E0CF479881E025
:10E1B000E5CF2A9A81E0EACF289A81E0EFCF8091DB
:10E1C0007505982F977F90937505982F937081E030
:10E1D00011F080E008955E9A08955E98809175052B
:10E1E0008860809375050895E82FF0E021E030E025
:10E1F000082E02C0220F331F0A94E2F720953095B3
:10E2000090917505922390937505E15EFD4F2081F5
:10E21000922321E019F020E0822F0895813079F0D7
:10E2200038F08230C9F7159A90915A079B7F04C045
:10E230005E9A90915A079E7F90935A07EDCF5E9A0F
:10E2400090915A079D7FF8CF80E0CEDF81E0CCDF50
:10E2500082E0CADFB4CF813079F070F0823071F0A3
:10E2600021E030E001C0220F8A95EAF78091750520
:10E27000822B8093750508955E98F2CF1598F0CFA4
:10E28000B0E0A0E0E6E4F1E70C9447ECC82F6AE1C7
:10E2900071E20E948EC08C2F0E94693D82E191E262
:10E2A0000E94BE338EE790E20E94BE338AE00E9455
:10E2B0009D3360E071E28C2F0E948EC08C2F0E94F3
:10E2C000693D83EE90E20E94BE338C2F0E94ADC068
:10E2D0008C2F0E945A388C2F0E9481388C2F0E94DC
:10E2E0003A388C2F0E9406386AE970E28C2F0E941F
:10E2F000A5C0D0919F0481E990E20E94BE336D2FAA
:10E3000070E090E080E00E9417AE40919B04509135
:10E310009C0460919D0470919E0486EE9EE20E9492
:10E32000E93384E890E20E94BE3380919F040E940A
:10E33000553D20E030E0A9016091A0047091A10456
:10E340008091A2049091A3040E9457E5882399F13B
:10E3500080EBE82E84E0F82E10E0670100E08C2FBF
:10E360000E94693D89ED90E20E94BE33802F0E9499
:10E37000182886ED90E20E94BE33812F0E94182853
:10E3800086EE9EE20E94BE33F60160817181828139
:10E39000938145E00E9461B08AE00E949D330F5F47
:10E3A000FCE1CF0ED11C0730D1F61F5F84E0E80EF0
:10E3B000F11C173091F68C2F0E9423406BEB70E21A
:10E3C0008C2F0E948EC008EA14E0D0E08C2F0E94AF
:10E3D000693D82EB90E20E94BE338D2F0E94182887
:10E3E000F80160817181072E000C880B990B0E9447
:10E3F0005DE5AB01BC018FEA90E20E94E933F801D0
:10E40000628173818CEA90E20E9415400C5F1F4F7D
:10E41000D13059F48C2F0E946D3D8C2F0E94FA331D
:10E42000CDB7DEB7E8E00C9463ECD1E0CFCFB0E03D
:10E43000A0E0EDE1F2E70C9445ECCCE4DDE002E78E
:10E4400017E08CE5A82E8DE0B82EC12CD12C7601DA
:10E45000C39469917991899199910E945BE528898A
:10E4600039894A895B890E94BCE50E945CEDF8010C
:10E4700061937193819391938F01C616D706E80635
:10E48000F90610F46B017C01AC16BD0611F76FEFB5
:10E490007FEFCB01A70196010E9485EB20938207B5
:10E4A000309383074093840750938507CDB7DEB739
:10E4B000EAE00C9461EC0F931F93CF93DF9300E697
:10E4C0001DE0CBE8D7E0F8012191319141915191C4
:10E4D0008F0160E070E080E89FE30E94EFEC6993B9
:10E4E000799389939993F7E0CB39DF0761F70E941D
:10E4F00073C09DDFDF91CF911F910F910895DBCF06
:10E50000DACFD9CFD8CF9091391380913A1398139D
:10E5100006C08091940D9091950D892B21F080E09B
:10E520000E94AF40F0CF08959091391380913A1333
:10E53000981307C08091940D9091950D892B09F443
:10E5400083CE80E00E94AF40EFCFCF92DF92EF9278
:10E55000FF92CF93DF9320919F04222319F1EC01C6
:10E5600008960E94A0276B017C0120E030E0A90101
:10E570000E9457E520E030E0A901882349F0CE0150
:10E580000E941E28A70196010E94BCE59B01AC01D8
:10E59000688579858A859B850E9474EC6887798770
:10E5A0008A879B87DF91CF91FF90EF90DF90CF908C
:10E5B0000895CF92DF92EF92FF92CF93DF93209155
:10E5C0009F04222319F1EC0108960E94A0276B01F9
:10E5D0007C0120E030E0A9010E9457E520E030E016
:10E5E000A901882349F0CE010E941E28A7019601A7
:10E5F0000E94BCE59B01AC01688579858A859B8575
:10E600000E9475EC688779878A879B87DF91CF9115
:10E61000FF90EF90DF90CF900895AEE1B0E0E3E19E
:10E62000F3E70C943FEC9E8F8D8F5B018A01FC0118
:10E63000EA5BFF4F2081318142815381298B3A8BE4
:10E640004B8B5C8BCA01B9010E945BE56B017C01BD
:10E65000D5012D913D914D915C910E94BCE50E94A8
:10E66000D9EC2B013C01F801208131814281538199
:10E67000C701B6010E94BCE50E94D9EC4B015C01C8
:10E68000C301B2010E945CED6D8B7E8B8F8B988FE6
:10E69000683771058105910540F428E730E040E0D6
:10E6A00050E02D8B3E8B4F8B588FC501B4010E94DB
:10E6B0005CED698F7A8F8B8F9C8F68377105810530
:10E6C000910540F488E790E0A0E0B0E0898F9A8F50
:10E6D000AB8FBC8FED8DFE8DEE5AFF4F20813181C7
:10E6E0004281538129873A874B875C87CA01B901E8
:10E6F0000E945DE52B013C016D897E898F89988D93
:10E700000E945BE56D837E838F83988720E030E0F5
:10E71000A901C301B2010E9457E5882309F4BBC1D6
:10E72000A7019601C701B6010E94BCE54B015C013F
:10E730002D813E814F815885CA01B9010E94BCE5F7
:10E740009B01AC01C501B4010E9474EC4B015C015A
:10E75000A3019201C301B2010E9475EC9B01AC01BF
:10E76000C501B4010E94EFEC0E94D9EC0E945CED5F
:10E7700069837A838B839C8369857A858B859C8565
:10E7800090958095709561957F4F8F4F9F4F0E9418
:10E790005DE54B015C01698D7A8D8B8D9C8D0E94AE
:10E7A0005BE569877A878B879C8720E030E0A90149
:10E7B000C501B4010E9457E5882309F470C1298579
:10E7C0003A854B855C85CA01B9010E94BCE56D871D
:10E7D0007E878F87988BA7019601C701B6010E949B
:10E7E000BCE59B01AC016D857E858F8598890E9473
:10E7F00074EC6B017C01A5019401C501B4010E9478
:10E8000075EC9B01AC01C701B6010E94EFEC0E94C0
:10E8100088EDAD8DBE8D95962D913D914D915C917C
:10E8200098972D873E874F87588B69017A012981F8
:10E830003A814B815C81C21AD30AE40AF50A0E942C
:10E840005CEDC61AD70AE80AF90AF7FE8CC02D81DA
:10E850003E814F815885CA01B9010E94BCE56B0118
:10E860007C0120E030E0A901C301B2010E9457E51C
:10E87000882309F418C16D857E858F8598890E944B
:10E880005BE59B01AC010E9475ECA30192010E9423
:10E89000BCE54B015C0129853A854B855C85CA0145
:10E8A000B9010E94BCE59B01AC01C501B4010E9405
:10E8B00075ECA70196010E9474EC4B015C0120E00D
:10E8C00030E040E850E4C301B2010E94BCE59B0186
:10E8D000AC01C501B4010E94EFEC0E94D9EC4B01E0
:10E8E0005C0120E030E0A9010E9414EE87FF03C024
:10E8F000812C912C5401C501B4010E945CED698307
:10E900007A838B839C832D853E854F855889261776
:10E9100037074807590720F429833A834B835C83E0
:10E9200069817A818B819C810E945BE54B015C014E
:10E93000A3019201C301B2010E9475EC9B01AC01DD
:10E94000C501B4010E94BCE5A70196010E9475ECC7
:10E950000E9453EE0E945CED698B7A8B8B8B9C8BB3
:10E96000C12CD12C760169897A898B899C892D8962
:10E970003E894F89588D621B730B840B950B0E9447
:10E980005BE5A30192010E94EFEC20E034E244EF4A
:10E9900059E40E94BCE50E945CED4B015C01698971
:10E9A0007A898B899C89298D3A8D4B8D5C8D621B70
:10E9B000730B840B950B0E945BE5A30192010E94EF
:10E9C000EFEC20E034E244EF59E40E94BCE50E9401
:10E9D0005CED6D837E838F839887C501B4010E94AF
:10E9E000A4612B013C016D817E818F8198850E94FD
:10E9F000A46129813A814B815C81AD8DBE8D999650
:10EA00002D933D934D935C939C9789019A010C0D36
:10EA10001D1D2E1D3F1DFD0105A716A727A730AB05
:10EA2000E65BFF4F2D893E894F89588D20833183C6
:10EA300042835383D5968D929D92AD92BC92D89786
:10EA40002D813E814F815885D9962D933D934D93CD
:10EA50005C93DC973D974082518262827382349648
:10EA6000608371838283938329893A894B895C8986
:10EA7000D1962D933D934D935C93D4973D96298DDC
:10EA80003A8D4B8D5C8D20833183428353836E9608
:10EA9000E0E10C945BEC60E070E0CB0165CE60E0FF
:10EAA00070E0CB01B4CE60E070E0CB0116CF909166
:10EAB0006F0081E091FD02C080E0089590916F00A9
:10EAC0009D7F90936F000895EFE6F0E08081826073
:10EAD00080830895CF93C82FEADF94E0C99F900107
:10EAE0001124F901E55BF94F295A394FD9014D91AC
:10EAF0005D916D917C91408351836283738391E03A
:10EB000090934A068111E0DFCF910895CF93DF9370
:10EB10008091E306811105C08091E906882309F4FC
:10EB20004EC08091DC05329B4DC081608093DC0536
:10EB30008091DC05339B48C082608093DC05809126
:10EB4000DC05349B43C084608093DC05C0913B06A8
:10EB5000C0FF0FC08091E40680FF0BC08091DC05F0
:10EB600080FF07C08091590781608093590780E03A
:10EB7000B1DFC1FF0FC08091E40681FF0BC080911F
:10EB8000DC0581FF07C08091590782608093590797
:10EB900081E0A0DFC2FF13C08091E40682FF0FC0B6
:10EBA0008091E906882359F08091DC0582FF07C037
:10EBB0008091590784608093590782E08BDFDF9151
:10EBC000CF9108958E7FB2CF8D7FB7CF8B7FBCCF93
:10EBD0006EDF1092860710928707109288071092B6
:10EBE0008907811171CF08950F931F938091391375
:10EBF00090913A13891B8F7009F449C09091361394
:10EC0000992361F0833040F48FEF890F29F08093CE
:10EC1000361390E080E038C01092361380913A139A
:10EC20002BE5829FC00111248556984FFC0120815D
:10EC300020FDEFCF409186075091870760918807AC
:10EC400070918907E95AFF4F008111812281338138
:10EC5000401B510B620B730B409386075093870741
:10EC6000609388077093890720913A132F5F2F7064
:10EC70002093371330913A1320913813321304C084
:10EC800020913713209338131F910F910895A0DF1F
:10EC9000C0CFA3E1B0E0EFE4F6E70C943DEC8FEFDA
:10ECA0009FEF90938900809388002AE02983312C7C
:10ECB000212C78948091440690914506A0914606B7
:10ECC000B0914706892B8A2B8B2B09F0C2C180910A
:10ECD0004A068823D1F08091480690914906109207
:10ECE0004A06892B91F0109249061092480610921C
:10ECF0003B069091391380913A13981731F0809127
:10ED00003A138F5F8F7080933A13809148069091E9
:10ED10004906892B09F49DC1409140065091410656
:10ED2000609142067091430680913C0690913D06A9
:10ED3000A0913E06B0913F060091320610E030E00F
:10ED400020E0841B950BA60BB70B081719072A07A1
:10ED50003B0710F4D901C8018A8B840F951FA61FA9
:10ED6000B71F8093400690934106A0934206B0934C
:10ED70004306E1E0C0900906D0900A06E0900B0639
:10ED8000F0900C068091190690911A06A0911B062E
:10ED9000B0911C06C80ED91EEA1EFB1EC0921906B1
:10EDA000D0921A06E0921B06F0921C06F7FC33C0C4
:10EDB00040910106042E000C550B660B770B8091D9
:10EDC000570690915806A0915906B0915A06840FA3
:10EDD000951FA61FB71F8093570690935806A093C0
:10EDE0005906B0935A068091050690910606A091A7
:10EDF0000706B0910806B701A601481B590B6A0B1C
:10EE00007B0BDB01CA018093190690931A06A0932D
:10EE10001B06B0931C0600910D0610910E06209162
:10EE20000F063091100680911D0690911E06A0914C
:10EE30001F06B0912006080F191F2A1F3B1F0093C1
:10EE40001D0610931E0620931F063093200637FDE3
:10EE500033C040910206042E000C550B660B770B55
:10EE600080915B0690915C06A0915D06B0915E0674
:10EE7000840F951FA61FB71F80935B0690935C06B7
:10EE8000A0935D06B0935E068091050690910606FC
:10EE9000A0910706B091080628013901481A590ABD
:10EEA0006A0A7B0AD301C20180931D0690931E0655
:10EEB000A0931F06B09320064091110650911206B0
:10EEC000609113067091140680912106909122069C
:10EED000A0912306B0912406480F591F6A1F7B1F7B
:10EEE00040932106509322066093230670932406D4
:10EEF00077FD33C080900306082C000C9908AA08FF
:10EF0000BB0880915F0690916006A0916106B09168
:10EF10006206880D991DAA1DBB1D80935F06909304
:10EF20006006A0936106B0936206809105069091F9
:10EF30000606A0910706B09108063A014B01681A2F
:10EF4000790A8A0A9B0AD401C3018093210690930F
:10EF50002206A0932306B093240680901506909075
:10EF60001606A0901706B09018068091250690917D
:10EF70002606A0912706B0912806880D991DAA1D86
:10EF8000BB1D8093250690932606A0932706B09379
:10EF90002806B7FD33C040900406042C000C550829
:10EFA000660877088090630690906406A0906506D6
:10EFB000B0906606840C951CA61CB71C8092630654
:10EFC00090926406A0926506B0926606809005064F
:10EFD00090900606A0900706B09008062C013D010F
:10EFE000481859086A087B08530142018092250697
:10EFF00090922606A0922706B0922806E11104C03E
:10F00000E0918400F0918500F7FE5F9A37FF469A01
:10F0100077FF2B9AB7FF299AE0918400F091850041
:10F02000E0918400F0918500F7FE5F9837FF4698E5
:10F0300077FF2B98B7FF29985A88552021F08091A7
:10F040008400909185002A8921502A8BE0E02111CB
:10F0500091CE8091440690914506A0914606B091CC
:10F060004706892B8A2B8B2B09F0B0C640904806A7
:10F07000509049065B8A4A8A4114510409F402C738
:10F080008091400690914106A0914206B0914306BE
:10F0900040913C0650913D0660913E0670913F06BE
:10F0A00084179507A607B70708F449C010924906C8
:10F0B0001092480610923B069091391380913A13B2
:10F0C000981709F4DFC680913A138F5F8F70809391
:10F0D0003A13A0EDCA2EA7E0DA2EE12CF12C809194
:10F0E000480690914906892B09F068C67DDD90930A
:10F0F000490680934806892B09F460C6409048066B
:10F10000509049065B8A4A8AD2018C9183FF08C5D8
:10F11000C20145960E94436110924906109248062A
:10F1200010923B069091391380913A139817F1F29F
:10F1300080913A138F5F8F7080933A13D7CF4091AD
:10F140003706509138066091390670913A06481793
:10F1500059076A077B0708F40FC2409133065091A4
:10F1600034066091350670913606EA89FB8985A9D7
:10F1700096A9A7A9B0AD481759076A077B0708F0F9
:10F18000D0C1411551056105710509F066C0809037
:10F190007A0590907B05A0907C05B0907D0587E274
:10F1A00099E2A1E0FC010591159125913491081592
:10F1B00019052A053B0558F4B694A79497948794AB
:10F1C000AA0F0496E3E4F9E2E817F90759F7A093C8
:10F1D0003206F0E28F169104A104B10428F4E0E2B3
:10F1E0008E2E912CA12CB12C20E2821A9108A1081C
:10F1F000B108811438E09306A104B10408F49AC15F
:10F20000A4E09A9EC0011124895D9A4DFC013296BA
:10F2100025913491B82DEE27B39F8001B29F010D47
:10F220001E1F06940E1F1E1F112430E020E0FC015B
:10F23000C590D490F12CE12CC01AD10AE20AF30A4D
:10F240004C0D5D1D6E1D7F1D40933306509334069B
:10F25000609335067093360642CF10E00A81942FF2
:10F26000852E862FBC81AD81FE81EF813885298571
:10F270004B80E0917605E99FA12DFF27309177051E
:10F28000399FA00DF11D10907805199EF00DE89D95
:10F29000A00DF11D389DF00DE89FF00D4A2EBF2FF7
:10F2A0004A9EE12D332722274F9EE00D311D211F5D
:10F2B000BA9FE00D311D211FBF9F300D211D432E30
:10F2C000B22F4A9E012D332722274F9E000D311D5C
:10F2D000211FBA9F000D311D211FBF9F300D211D21
:10F2E000432EB22FEE2790917A0580907B05809176
:10F2F0007C050090A002012A09F483C030919C0291
:10F30000349DE119910B810A810B20919D02249D6E
:10F31000E0199109810A810B00919E02049D9019C8
:10F320008108810B3B9FE0199109810A810B2B9F7A
:10F3300090198108810B0B9F801881094A9E012D2D
:10F34000332722274F9E000D311D211FBA9F000D2C
:10F35000311D211FBF9F300D211D432EB22F309133
:10F360009802349DE10D911F811E811F2091990209
:10F37000249DE00D911D811E811F00919A02049D24
:10F38000900D811C811F3B9FE00D911D811E811FEF
:10F390002B9F900D811C811F0B9F800C811D4A9E0D
:10F3A000012D332722274F9E000D311D211FBA9FAB
:10F3B000000D311D211FBF9F300D211D432EB22F87
:10F3C00030919402349DE119910B810A810B2091B7
:10F3D0009502249DE0199109810A810B0091960202
:10F3E000049D90198108810B3B9FE0199109810AC6
:10F3F000810B2B9F90198108810B0B9F801881092D
:10F4000082C030919C02349DE10D911F811E811FAD
:10F4100020919D02249DE00D911D811E811F009170
:10F420009E02049D900D811C811F3B9FE00D911D4C
:10F43000811E811F2B9F900D811C811F0B9F800CB3
:10F44000811D4A9E012D332722274F9E000D311D1D
:10F45000211FBA9F000D311D211FBF9F300D211D9F
:10F46000432EB22F30919802349DE119910B810AFD
:10F47000810B20919902249DE0199109810A810B49
:10F4800000919A02049D90198108810B3B9FE0191D
:10F490009109810A810B2B9F90198108810B0B9F89
:10F4A000801881094A9E012D332722274F9E000D87
:10F4B000311D211FBA9F000D311D211FBF9F300D2F
:10F4C000211D432EB22F30919402349DE10D911FE6
:10F4D000811E811F20919502249DE00D911D811EAA
:10F4E000811F00919602049D900D811C811F3B9FFE
:10F4F000E00D911D811E811F2B9F900D811C811F8E
:10F500000B9F800C811D11244B820A83BC83AD8329
:10F51000FE83EF8338872987982C892EB12CA82E5B
:10F520003ECEAA89BB89D1968D909D90AD90BC901E
:10F53000D49735CED501C401B695A79597958795F3
:10F540008C7F895D9E4DFC01C590D490FC01329664
:10F5500025913491E82DE7708E2EE29FC001E39F44
:10F56000900D112433E0969587953A95E1F7C81AE6
:10F57000D90AF12CE12C64CE40912E0650912F0631
:10F580006091300670913106481759076A077B076A
:10F5900008F030C28090290690902A06A0902B0691
:10F5A000B0902C0680912D06EA89FB8981117CC0E0
:10F5B000EF5BFF4FE080F18002811381EA89FB89D4
:10F5C000E25BFF4F2081318142815381AA89BB894F
:10F5D000D1966D917D918D919C91D4970E944C61B3
:10F5E000B1E0B0932D06EA89FB8941A952A963A92C
:10F5F00074A987E299E2A1E0FC010591159125919A
:10F600003491041715072607370758F47695679540
:10F6100057954795AA0F0496E3E4F9E2E817F9072E
:10F6200059F7A0933206403251056105710520F467
:10F6300040E250E060E070E0405251096109710918
:10F640004115F8E05F076105710508F4B3C124E0D6
:10F65000529FC0011124895D9A4DFC01329625917B
:10F660003491AA27439FF001429FE10DFA1F0694AF
:10F67000EA1FFA1F1124AF0170E060E0FC01C590A1
:10F68000D490F12CE12CC41AD50AE60AF70A8C0CA6
:10F690009D1CAE1CBF1C8092290690922A06A09247
:10F6A0002B06B0922C061BCD81AD92ADA3ADB4ADAF
:10F6B00088169906AA06BB0608F072C18114910447
:10F6C000A104B10449F440917A0550917B05609101
:10F6D0007C0570917D058DCFA0E0BA85982D492DD0
:10F6E0008A2DFB85EC857D856E855F853889298926
:10F6F00050917605599F712D662730917705399F76
:10F70000700D611D10907805199E600D549F700D4D
:10F71000611D349F600D589F600DF72FE62FF79FF6
:10F72000512D33272227F69F500D311D2A1FE79FA9
:10F73000500D311D2A1FE69F300D211DF32FE22FA2
:10F74000F79FB12D33272227F69FB00D311D2A1FB9
:10F75000E79FB00D311D2A1FE69F300D211DF32FAD
:10F76000E22F552790917A0540917B0580917C0589
:10F770000090A0020A2A09F483C030919C023F9FA6
:10F7800051199A0B4A0B8A0B20919D022F9F5019F9
:10F7900091094A0B8A0BB0919E02BF9F90194109B3
:10F7A0008A0B3E9F501991094A0B8A0B2E9F901984
:10F7B00041098A0BBE9F40198109F79FB12D33275C
:10F7C0002227F69FB00D311D2A1FE79FB00D311D76
:10F7D0002A1FE69F300D211DF32FE22F3091980252
:10F7E0003F9F510D9A1F4A1F8A1F209199022F9FF8
:10F7F000500D911D4A1F8A1FB0919A02BF9F900D14
:10F80000411D8A1F3E9F500D911D4A1F8A1F2E9F2A
:10F81000900D411D8A1FBE9F400D811DF79FB12D88
:10F8200033272227F69FB00D311D2A1FE79FB00D09
:10F83000311D2A1FE69F300D211DF32FE22F30913D
:10F8400094023F9F51199A0B4A0B8A0B2091950203
:10F850002F9F501991094A0B8A0BB0919602BF9FB6
:10F86000901941098A0B3E9F501991094A0B8A0B46
:10F870002E9F901941098A0BBE9F4019810982C0B1
:10F8800030919C023F9F510D9A1F4A1F8A1F209161
:10F890009D022F9F500D911D4A1F8A1FB0919E02FD
:10F8A000BF9F900D411D8A1F3E9F500D911D4A1F05
:10F8B0008A1F2E9F900D411D8A1FBE9F400D811DE6
:10F8C000F79FB12D33272227F69FB00D311D2A1F38
:10F8D000E79FB00D311D2A1FE69F300D211DF32F2C
:10F8E000E22F309198023F9F51199A0B4A0B8A0BD5
:10F8F000209199022F9F501991094A0B8A0BB091C0
:10F900009A02BF9F901941098A0B3E9F5019910995
:10F910004A0B8A0B2E9F901941098A0BBE9F4019F2
:10F920008109F79FB12D33272227F69FB00D311D96
:10F930002A1FE79FB00D311D2A1FE69F300D211DA4
:10F94000F32FE22F309194023F9F510D9A1F4A1FCF
:10F950008A1F209195022F9F500D911D4A1F8A1FCB
:10F96000B0919602BF9F900D411D8A1F3E9F500D82
:10F97000911D4A1F8A1F2E9F900D411D8A1FBE9FF9
:10F98000400D811D1124BA87FB87EC877D876E8728
:10F990005F87388B298B542F492F70E0682F29CE31
:10F9A0002A893B89225B3F4FD9014D915D916D9131
:10F9B0007C911FCEDB01CA01B695A79597958795D7
:10F9C0008C7F895D9E4DFC01C590D490FC013296E0
:10F9D000259134914770429FC001439F900D11249F
:10F9E000A3E096958795AA95E1F7C81AD90AF12C54
:10F9F000E12C4DCE8091570190915801A091590171
:10FA0000B0915A01B7FF61C0EA89FB89EA5BFF4FF9
:10FA1000C080D180E280F38087E299E221E0FC019E
:10FA200045915591659174914C155D056E057F0565
:10FA300058F4F694E794D794C794220F049643E4BD
:10FA400059E24817590759F72093320650E2C51674
:10FA5000D104E104F10428F470E2C72ED12CE12C8A
:10FA6000F12C60E2C61AD108E108F108C11478E06F
:10FA7000D706E104F10408F431C0A4E0DA9EC00125
:10FA80001124895D9A4DFC01329625913491BC2D4B
:10FA90006627B39FA001B29F410D561F0694461FD3
:10FAA000561F112470E060E0FC0185919491B0E054
:10FAB000A0E0841B950BA60BB70B80935701909386
:10FAC0005801A0935901B0935A01C0905701D090AA
:10FAD0005801E0905901F0905A0101CBD701C601BD
:10FAE000B695A795979587958C7F895D9E4DFC016E
:10FAF00025913491FC01329645915491EC2DE7709B
:10FB0000E49FC001E59F900D112463E096958795D1
:10FB10006A95E1F7281B390BC901B0E0A0E0CDCF11
:10FB2000EA89FB8985889688A788B08C81E0811452
:10FB30009104A104B10409F480E0AA89BB89599613
:10FB4000CD90DD90ED90FC905C97C114D104E10460
:10FB5000F10409F08260EA89FB89458D568D678D35
:10FB600070A1411551056105710509F0846080930C
:10FB70003B061092290610922A0610922B0610922C
:10FB80002C0610923306109234061092350610920D
:10FB90003606EA89FB8985A196A1A7A1B0A5809325
:10FBA0003C0690933D06A0933E06B0933F06442446
:10FBB00055243201481A590A6A0A7B0A40921906EA
:10FBC00050921A0660921B0670921C0640921D0607
:10FBD00050921E0660921F067092200640922106E7
:10FBE00050922206609223067092240641A052A0F1
:10FBF00063A074A0440C551C661C771C880C991CCF
:10FC0000AA1CBB1C8092090690920A06A0920B06C1
:10FC1000B0920C06CC0CDD1CEE1CFF1CC0920D0635
:10FC2000D0920E06E0920F06F0921006440F551F78
:10FC3000661F771F409311065093120660931306B8
:10FC4000709314064092150650921606609217069D
:10FC500070921806880F991FAA1FBB1F8093050674
:10FC600090930606A0930706B093080610924006EC
:10FC700010924106109242061092430681A592A569
:10FC8000A3A5B4A58093370690933806A0933906B0
:10FC9000B0933A0685A596A5A7A5B0A980932E0690
:10FCA00090932F06A0933006B0933106EB5BFF4F85
:10FCB00080819091E406891721F08093E4060E94E8
:10FCC000AE700E94867544244A94542C32014092AE
:10FCD0005701509258016092590170925A01EA8975
:10FCE000FB89FD96E080F18002811381AA89BB899E
:10FCF000D1962D913D914D915C91D4976D01BAE4CF
:10FD0000CB0ED11CF60160817181828193810E94AA
:10FD10004C6110922D06D6014D915D916D917C91B3
:10FD200087E299E2A1E0FC010591159125913491BA
:10FD3000041715072607370758F4769567955795E2
:10FD40004795AA0F0496E3E4F9E2E817F90759F793
:10FD5000A0933206403251056105710520F440E25E
:10FD600050E060E070E040525109610971094115AD
:10FD7000F8E05F076105710508F462C024E0529F56
:10FD8000C0011124895D9A4DFC0132962591349170
:10FD9000AA27439FF001429FE10DFA1F0694EA1F34
:10FDA000FA1F1124AF0170E060E0FC01C590D4900F
:10FDB000F12CE12CC41AD50AE60AF70AC0924406CF
:10FDC000D0924506E0924606F0924706809144069E
:10FDD00090914506A0914606B0914706AC01BD0141
:10FDE000009731E0A307B10520F04FEF5FEF60E02F
:10FDF00070E0841B950BA60BB70B80934406909381
:10FE00004506A0934606B0934706F8948091840077
:10FE1000909185004096A981A150A983AA2381F1E0
:10FE2000240E351E2816390610F40C94597630929B
:10FE300089002092880078946396E2E10C9459EC52
:10FE4000DB01CA01B695A795979587958C7F895D4B
:10FE50009E4DFC01C590D490FC01329625913491C1
:10FE60004770429FC001439F900D112433E0969547
:10FE700087953A95E1F7C81AD90AF12CE12C9ECF63
:10FE80001C01D5CF80EDC82E87E0D82EE12CF12CB7
:10FE90002DC9CF93DF938091391390913A13891B29
:10FEA00080958F7019F40E94AF40F5CF809139137F
:10FEB0008F5F8F70A09139139BE5A99FD00111240A
:10FEC000FD01E556F84FEF0119929A95E9F798E090
:10FED0009083A055B84F90E1EBE3F3E101900D92D0
:10FEE0009A95E1F72091391390913A13291303C0A1
:10FEF00094E690933613809339130E946475DF91D2
:10FF0000CF910895FC01208131814281538160911C
:10FF10006C0D70916D0D80916E0D90916F0D0E9422
:10FF2000BCE50E9419EE60934713709348138093C9
:10FF3000491390934A139091391380913A1398176B
:10FF400009F0A7CF0E9483720E9457754091471312
:10FF5000509148136091491370914A13409363067E
:10FF600050936406609365067093660681110C9445
:10FF7000647508954F925F926F927F928F929F92D5
:10FF8000AF92BF92CF92DF92EF92FF92CF93DF9327
:10FF9000EC0120916C0D30916D0D40916E0D5091E2
:10FFA0006F0D6C857D858E859F850E94BCE50E94C6
:10FFB00019EE6B017C012091680D3091690D409123
:10FFC0006A0D50916B0D688579858A859B850E94A5
:10FFD000BCE50E9419EE4B015C012091640D30914B
:10FFE000650D4091660D5091670D6C817D818E810C
:10FFF0009F810E94BCE50E9419EE2B013C012091DB
:020000021000EC
:10000000600D3091610D4091620D5091630D6881DA
:1000100079818A819B810E94BCE50E9419EE6093E0
:100020003B1370933C1380933D1390933E13409287
:100030003F1350924013609241137092421380928A
:10004000431390924413A0924513B0924613C0926A
:100050004713D0924813E0924913F0924A139091BB
:10006000391380913A13981781F013DFDF91CF9104
:10007000FF90EF90DF90CF90BF90AF909F908F90C8
:100080007F906F905F904F9008950E9483720E94BE
:100090005775C82F8BE393E10E944361CC2331F362
:1000A0000E946475E3CFCF92DF92EF92FF92CF93DD
:1000B000DF93C82F0E94577594E0C99FE001112477
:1000C000FE01E95AF94FC080D180E280F3808111AE
:1000D0000E946475C557D84FC701B6010E945DE5FF
:1000E000288139814A815B810E94BCE5DF91CF91F3
:1000F000FF90EF90DF90CF900895CF92DF92EF9234
:10010000FF92CF93DF93C82F0E94577594E0C99F49
:10011000E0011124FE01E55BF94FC080D180E2804F
:10012000F38081110E946475C557D84FC701B6018D
:100130000E945DE5288139814A815B810E94BCE58E
:10014000DF91CF91FF90EF90DF90CF900895A1E0E5
:10015000B0E0EDEAF0E80C944DEC898360E0CE016C
:1001600001960E949E6261E0CE0101960E949E620D
:1001700062E0CE0101960E949E6289812196E2E0B2
:100180000C9469ECA2E1B0E0E8ECF0E80C9449ECE6
:10019000DEDF8823C1F1EDB6FEB642E952E082FF10
:1001A00002C049E852E022E932E081FF02C02BE8B8
:1001B00032E080FD25C082E992E05F934F933F9348
:1001C0002F939F938F9381E19CE19F938F938E0157
:1001D0000F5F1F4F1F930F930E94F0E40E94653D35
:1001E000C8010E94AF33C8010E94BCBF0FB6F8948B
:1001F000DEBF0FBECDBF81E06296E6E00C9465ECF9
:100200008DE892E0DACF80E0F7CFA0E2B0E0EBE05B
:10021000F1E80C943DEC80913B01882309F4BEC0C9
:100220008091EF05082F10E080FF3CC0C0903D0199
:10023000D0903E01E0903F01F09040012091830476
:10024000309184044091850450918604C701B60121
:100250000E9414EE181644F4C0928304D0928404D1
:10026000E0928504F0928604C0904901D0904A0142
:10027000E0904B01F0904C01209183043091840474
:100280004091850450918604C701B6010E9457E54C
:1002900087FF08C0C0928304D0928404E092850452
:1002A000F092860401FF3CC0C0904101D090420111
:1002B000E0904301F090440120918704309188043C
:1002C0004091890450918A04C701B6010E9414EE3E
:1002D000181644F4C0928704D0928804E0928904EE
:1002E000F0928A04C0904D01D0904E01E0904F01F1
:1002F000F090500120918704309188044091890446
:1003000050918A04C701B6010E9457E587FF08C0D3
:10031000C0928704D0928804E0928904F0928A0403
:1003200002FF3CC0C0904501D0904601E0904701DB
:10033000F090480120918B0430918C0440918D0401
:1003400050918E04C701B6010E9414EE181644F4B1
:10035000C0928B04D0928C04E0928D04F0928E04B3
:10036000C0905101D0905201E0905301F09054019F
:1003700020918B0430918C0440918D0450918E0417
:10038000C701B6010E9457E587FF08C0C0928B04E1
:10039000D0928C04E0928D04F0928E0480914B0DEB
:1003A00083FD61C020917E0130917F0140918001E9
:1003B0005091810160918F0470919004809191041B
:1003C000909192040E9457E5882309F44CC00E9442
:1003D0000FB1182F882331F00E94653D86EF9BE115
:1003E0000E94BE3320917E0130917F0140918001B7
:1003F0005091810160918F047091900480919104DB
:10040000909192040E9474EC9F7720916C0130913E
:100410006D0140916E0150916F010E94BCE520E09A
:1004200030E046E154E40E9414EE1816D4F40E9421
:10043000653D87ED9BE10E94BE3380918F049091D2
:100440009004A0919104B091920480937E019093C6
:100450007F01A0938001B09381018FE894E052DD89
:1004600002C01111EACF2AE037ED43E25CE360916C
:1004700035017091360180913701909138010E94C9
:10048000BCE56B017C016091390170913A01072E46
:10049000000C880B990B0E945DE59B01AC01C70124
:1004A000B6010E94BCE5698B7A8B8B8B9C8B80910B
:1004B0009F04882309F180909B0490909C04A09055
:1004C0009D04B0909E04C0908B04D0908C04E0906A
:1004D0008D04F0908E0420E030E0A901C501B40144
:1004E0000E9457E58823F9F0A7019601C501B401E0
:1004F0000E9414EE1816BCF020E030E0A901BE0105
:100500006F5E7F4F83E894E00E9450C080E1E3E893
:10051000F4E0A2E7B1E001900D928A95E1F7A09690
:10052000E2E10C9459EC20917201309173014091F9
:1005300074015091750160918304709184048091DD
:100540008504909186040E9474EC4B015C0120911B
:100550007601309177014091780150917901609155
:100560008704709188048091890490918A040E9484
:1005700074EC6D8B7E8B8F8B988F20917A013091EC
:100580007B0140917C0150917D01C701B6010E9421
:1005900074EC6D8F7E8F8F8F98A320917E013091A8
:1005A0007F01409180015091810160918F04709191
:1005B000900480919104909192040E9474EC698F50
:1005C0007A8F8B8F9C8F20E030E0A901C501B401A8
:1005D0000E9457E581110CC020E030E0A9016D892F
:1005E0007E898F89988D0E9457E5882309F484CFEE
:1005F000A5019401C501B4010E94BCE56B017C0119
:100600002D893E894F89588DCA01B9010E94BCE5E8
:100610009B01AC01C701B6010E9475EC6B017C0126
:100620002D8D3E8D4F8D58A1CA01B9010E94BCE5A8
:100630009B01AC01C701B6010E9475EC6B017C0106
:10064000298D3A8D4B8D5C8DCA01B9010E94BCE5A4
:100650009B01AC01C701B6010E9475EC6B017C01E6
:100660000E9453EE2B013C012CEC3CEB4CE85BE28E
:10067000C701B6010E9457E587FF06C0498C5A8C16
:100680006B8C7C8CE89477F82DEB37E346E855E3E8
:10069000C301B2010E9457E587FD38CF2DEC3CEC39
:1006A0004CE45EE3C301B2010E94BCE50E945CED34
:1006B0001B01672B19F422242394312CB10190E003
:1006C00080E00E945BE59B01AC0160E070E080E8A7
:1006D0009FE30E94EFEC6B017C01AC019B01C30125
:1006E000B2010E94BCE52B013C01A7019601C501A6
:1006F000B4010E94BCE54B015C01A70196016D8924
:100700007E898F89988D0E94BCE56D8B7E8B8F8B47
:10071000988FA70196016D8D7E8D8F8D98A10E9477
:10072000BCE56D8F7E8F8F8F98A3A7019601698D91
:100730007A8D8B8D9C8D0E94BCE5698F7A8F8B8F13
:100740009C8F80E1E2E7F1E08E010F5F1F4FD8013F
:1007500001900D928A95E1F70E9495CA6B017C0188
:1007600028ECC20ED11CE11CF11C81E0281A3108D2
:1007700009F454C00E9495CA9B01AC012C193D0993
:100780004E095F0957FD4DC06B017C0128ECC20E7C
:10079000D11CE11CF11C80E00E94AF40A501940136
:1007A00069817A818B819C810E9475EC69837A834F
:1007B0008B839C832D893E894F89588D6D817E81E5
:1007C0008F8198850E9475EC6D837E838F839887D7
:1007D0002D8D3E8D4F8D58A169857A858B859C85A1
:1007E0000E9475EC69877A878B879C87298D3A8D63
:1007F0004B8D5C8D6D857E858F8598890E9475EC0B
:100800006D877E878F87988BA3019201BE016F5EF3
:100810007F4FC8010E9450C08111A7CFA301920150
:100820006ECE0E94616FBACF8091EB059091EC057E
:10083000A091ED05B091EE058093350190933601BE
:10084000A0933701B09338018091E9059091EA05B2
:1008500090933A01809339010895809135019091E8
:100860003601A0913701B09138018093EB05909348
:10087000EC05A093ED05B093EE05809139019091C0
:100880003A019093EA058093E90584E690E090931D
:100890003A01809339010895ACE0B0E0E2E5F4E874
:1008A0000C943FEC2B013C0129873A874B875C87EE
:1008B00047015801D601CD90DD90ED90FC9020E0ED
:1008C00030E0A901C701B6010E9457E5811171C04E
:1008D0008091680190916901A0916A01B0916B01CA
:1008E00089839A83AB83BC8320E030E0A901C701F0
:1008F000B6010E9457E5811106C0C12CD12C80E8B9
:10090000E82E80E4F82ECD82DE82EF82F886A50103
:10091000940160917A0170917B0180917C019091AA
:100920007D010E9457E587FF0CC080927A0190926A
:100930007B01A0927C01B0927D01CE0105960E94C0
:10094000AC6940927201509273016092740170928E
:10095000750189859A85AB85BC85809376019093D6
:100960007701A0937801B0937901CE0101960E949E
:10097000AC69A501940160917A0170917B0180912D
:100980007C0190917D010E9414EE181664F480920F
:100990007A0190927B01A0927C01B0927D01CE0100
:1009A00005960E94AC690E9483722C96E0E10C943B
:1009B0005BECD701C60194CFCF92DF92EF92FF920A
:1009C0000F931F936B01FC01E080F1800281138182
:1009D000E2E7F1E0248135814681578160817181B0
:1009E0008281938159DF1F910F91FF90EF90DF90EB
:1009F000CF9008958F929F92AF92BF92CF92DF9245
:100A0000EF92FF921F93CF93DF93CDB7DEB760973E
:100A10000FB6F894DEBF0FBECDBF182F80E043DBCA
:100A20004B015C018092DD059092DE05A092DF050E
:100A3000B092E00581E037DB6B017C01C092E105FB
:100A4000D092E205E092E305F092E40582E02BDB30
:100A50006093E5057093E6058093E7059093E805BC
:100A60001D861E861F86188A89829A82AB82BC8266
:100A7000CD82DE82EF82F88669877A878B879C87B2
:100A800083E011DB6D877E878F87988BCE0101967F
:100A90000E94A5721E3FD9F480E1FE013196A2E7C3
:100AA000B1E001900D928A95E1F760960FB6F89447
:100AB000DEBF0FBECDBFDF91CF911F91FF90EF90B2
:100AC000DF90CF90BF90AF909F908F90089584E07B
:100AD000189FF0011124DF01AE58BE4F81E090E075
:100AE0008C0F9D1FE80FF91F408151816281738136
:100AF0004D935D936D937C931397D7CF0C9473C0F4
:100B0000CF930E945775C82F80913A138093391361
:100B1000809338138093371384E6809336130E94B2
:100B2000E87580ED93E09093950D8093940DC1113D
:100B30000E94647581E080934A060E9483728EEF62
:100B400059DFDCDFCF910895ACE0B0E0EAEAF5E8E8
:100B50000C944DEC0E94CEB00E9457759CE0E7E5E6
:100B6000F6E0DE01119601900D929A95E1F7811160
:100B70000E946475CE0101960E9426702C96E2E0D8
:100B80000C9469ECB0E0A0E0E8ECF5E80C943FECE4
:100B900040907201509073016090740170907501E3
:100BA0008090760190907701A0907801B0907901C3
:100BB000C0907A01D0907B01E0907C01F0907D01A3
:100BC0000E9417726091550170915601072E000C1A
:100BD000880B990B0E945DE52AE037ED43E25CE368
:100BE0000E94BCE560936C0170936D0180936E016F
:100BF00090936F010DE311E0D0E0C0E0CE018C5C7A
:100C0000904E0E949727F80161937193819391937D
:100C10008F01CE01885D904E0E949727F801608772
:100C20007187828793872496CC30D10539F760E0AD
:100C30008DEF95E00E94812A0E944E2B0E945B72EC
:100C4000A30192016091720170917301809174010E
:100C5000909175010E9457E581111BC0A501940177
:100C6000609176017091770180917801909179017E
:100C70000E9457E581110DC020917A0130917B01CE
:100C800040917C0150917D01C701B6010E9457E55A
:100C900081115ADFCDB7DEB7E0E10C945BEC8DEB50
:100CA0009BE10E94BE3386B167EB7BE182FB882724
:100CB00080F90E943E6986B161EB7BE183FB882766
:100CC00080F90E943E6986B16BEA7BE18295817072
:100CD0000C943E698091E306811103C08091E9067E
:100CE00081110C9486750895ACE0B0E0EAE7F6E86F
:100CF0000C944DECACE4BDE090E080E0FC01E259E6
:100D0000FF4D45915591659174914D935D936D9310
:100D10007D93FC01E25AFF4D459155916591749187
:100D200050964D935D936D937C935397FC01E25BDA
:100D3000FF4D459155916591749190964D935D93BA
:100D40006D937C939397049680319105B9F680E278
:100D50009EE4A0E0B0E080935C0D90935D0DA093C5
:100D60005E0DB0935F0D80E090E0AAEFB3E4809356
:100D7000800D9093810DA093820DB093830D80938D
:100D8000840D9093850DA093860DB093870D80936D
:100D9000880D9093890DA0938A0DB0938B0D1092BE
:100DA0008C0D10928D0D10928E0D10928F0D109251
:100DB000900D1092910D1092920D1092930D8AE069
:100DC00097EDA3EABDE380936E0790936F07A0931E
:100DD0007007B093710780E090E0A0E2B1E48093E7
:100DE000FD059093FE05A093FF05B09300060E94B9
:100DF000372A8CE0EEEAF1E0DE01119601900D92C7
:100E00008A95E1F789819A81AB81BC81809328130F
:100E100090932913A0932A13B0932B138D819E8155
:100E2000AF81B88580932C1390932D13A0932E132C
:100E3000B0932F1389859A85AB85BC858093301339
:100E400090933113A0933213B093331380914F02D8
:100E500090915002A0915102B09152028093E50608
:100E60009093E606A093E706B093E8068EEB90E039
:100E70009093A9048093A8041092AB041092AA0442
:100E800086EE90E09093AD048093AC041092AF0492
:100E90001092AE048FE892ECADE8B1E48093981222
:100EA00090939912A0939A12B0939B128CE998EFA9
:100EB000A5E4BEE380939C1290939D12A0939E1292
:100EC000B0939F1281E49CEBABECB3E48093A0124F
:100ED0009093A112A093A212B093A3121092E306D2
:100EE0001092E206F7DE4EDE0E94653D8BE290E254
:100EF0000E94BE332C96E2E00C9469ECA4E0B0E0D2
:100F0000E4E8F7E80C943EEC9091E906981709F4B0
:100F10005EC0382E80E090E0A0E2B1E489839A833D
:100F2000AB83BC83409030135090311360903213E8
:100F30007090331320E030E0A901C301B2010E9498
:100F400057E587FF0CC0A301920160E070E080E2EA
:100F500091E40E9474EC69837A838B839C83CE0135
:100F600001960E94EDC04090720150907301609014
:100F70007401709075018090760190907701A09037
:100F80007801B0907901E1E0E325F0E0EE0FFF1F7A
:100F9000EB51F94F6081718185E293E10E94173234
:100FA00019821A821B821C82E0907A01F0907B01E8
:100FB00000917C0110917D01CE0101966C01A5018B
:100FC0009401C301B20168DC3092E90683DE80E05F
:100FD0002496E1E10C945AEC4F925F926F927F92CB
:100FE0008F929F92AF92BF92DF92EF92FF920F93F8
:100FF0001F93CF93DF93D82EC82FD0E0FE01E55783
:10100000F14DF49082E0D81609F4E3C06F2DFF0C87
:10101000770B880B990B0E945DE52B013C01CE01FB
:10102000880F991F880F991F805A934E0E94972707
:101030004B015C01A3019201C501B4010E94BCE512
:101040004B015C017E01EE0CFF1CEE0CFF1CC70186
:101050008C5A934E0E9497279B01AC01C301B201A9
:101060000E94BCE520E030E040EC5FE30E94BCE57C
:10107000AB01BC0100E010E098018D2D0E9453C42B
:1010800020E030E0A901C501B4010E9457E58823A2
:1010900009F440C082E000E010E020E830E4D81617
:1010A00019F000E010E09801B501A40170588D2DF1
:1010B0000E9453C4A5019401C501B4010E9475ECBE
:1010C0004B015C0182E000E010E020E030E4D81643
:1010D000E1F0FE01EB5BF34E6491611107C00E94E9
:1010E000653D83E29CE10E94BE336AE070E090E0DF
:1010F00080E00E945BE59B01AC0161E070E088E468
:1011000092E40E94EFEC8B019C01B501A4018D2DAE
:101110000E9453C481E090E00D2C01C0880F0A9416
:10112000EAF790915A07982B90935A079091EF0500
:10113000892B8093EF05C701885B934E0E94972708
:10114000F701EE58FE4F608371838283938382E0C0
:10115000D8121AC0209130133091311340913213BC
:101160005091331360917A0170917B0180917C01E1
:1011700090917D010E9474EC60937A0170937B01E1
:1011800080937C0190937D01B9DCF701ED57FB4F13
:10119000D701AE58BE4F8D919D910D90BC91A02D61
:1011A00080839183A283B38382E0D81202C00E941D
:1011B0009D27DF91CF911F910F91FF90EF90DF90CE
:1011C000BF90AF909F908F907F906F905F904F9067
:1011D000089581E093DE8111ECCF88E69CE10E94C6
:1011E000972720E030E0A9010E9457E5882309F401
:1011F0000DCF6F2DFF0C770B880B990B0E945DE5CF
:101200002B013C0188E69CE10E9497274B015C0181
:1012100020E030E040EA50E40E9414EE87FF0ACF5D
:10122000812C912C90EAA92E90E4B92E03CF8091C5
:101230005907882319F010925907089540E070E08B
:1012400060E08BE89BE10E94893F1F920F920FB6EE
:101250000F9211240BB60F922F933F934F935F93EE
:101260006F937F938F939F93AF93BF93EF93FF936E
:101270000E948675FF91EF91BF91AF919F918F91E1
:101280007F916F915F914F913F912F910F900BBE86
:101290000F900FBE0F901F9018950F931F93809182
:1012A0006A07813019F50E9495CA0091D405109102
:1012B000D5052091D6053091D705601B710B820BA7
:1012C000930B28EE33E040E050E00E9485EB609104
:1012D000D0057091D1058091D2059091D305620F10
:1012E000731F841F951F1F910F9108956091D8055A
:1012F0007091D9058091DA059091DB05D6CF1092D7
:101300006A071092D4051092D5051092D605109256
:10131000D7051092D8051092D9051092DA051092CF
:10132000DB051092D0051092D1051092D2051092D3
:10133000D305089580916A078130E1F08230C1F4CD
:10134000ACDF6093D0057093D1058093D205909364
:10135000D30581E080936A070E9495CA6093D40503
:101360007093D5058093D6059093D70581E00895B5
:10137000C6DFEFCF80E008950E943BC10E94E82BBA
:10138000882351F08091B71482FD06C08AE397E16B
:101390009093EB068093EA06CDCF80916A07813067
:1013A00079F482E080936A070E9495CA6093D80519
:1013B0007093D9058093DA059093DB0581E0089559
:1013C00080E0089580916A078150823070F4109215
:1013D0006A070E9495CA6093D8057093D9058093D7
:1013E000DA059093DB0581E0089580E008959C0183
:1013F00097FF26C0EE27FF27E81BF90B2D398FEF4B
:1014000038070CF05DC08DE280937E04CF0164E666
:1014100070E00E940FECCB012AE030E0B9010E949D
:101420000FEC805D80937F04CF01B9010E940FEC27
:10143000CB01B9010E940FEC805D809380042AC02B
:10144000283E83E03807B4F1C90168EE73E00E94DA
:101450000FECCB01EAE0F0E0BF010E940FEC805DF1
:1014600080937E04C90164E670E00E940FECCB011A
:10147000BF010E940FEC805D80937F04C901BF0112
:101480000E940FECCB01BF010E940FEC805D8093A6
:101490008004F901CF016AE070E00E940FEC805DEA
:1014A000809381048EE794E008958DE237FDC5CFE7
:1014B00080E2C3CFF90180E2243631050CF0A4CFDD
:1014C00080E280937E0480937F04EA30F1056CF320
:1014D0008DE237FF80E280937F04CF016AE070E005
:1014E0000E940FEC605D60938004D4CF9C0197FD57
:1014F0002DC080E2243631055CF0C90164E670E05D
:101500000E940FECCB016AE070E00E940FEC805D5E
:1015100080937F0480E22A3031055CF0EAE0F0E05D
:10152000C901BF010E940FECCB01BF010E940FEC6B
:10153000805D80938004C9016AE070E00E940FEC36
:10154000805D809381048FE794E008953195219523
:1015500031098DE2DDCFCF92DF92EF92FF92FC0155
:10156000C080D180E280F38020E030E0A901C70193
:10157000B6010E9457E587FD26C06DEB77E386E054
:1015800095E3A70196010E9475EC6B017C0120E0B8
:1015900030E0A9010E9457E520E030E040E05FE341
:1015A00087FF04C020E030E040E05FEBC701B601F8
:1015B0000E9475EC0E9457EDCB0198DFFF90EF90F1
:1015C000DF90CF9008956DEB77E386E095EBD9CF70
:1015D000A4E0B0E0EEEEFAE80C944DEC0E945DE57C
:1015E00069837A838B839C83CE010196B4DF249632
:1015F000E2E00C9469ECFC0160817181828193814D
:101600000E9457EDCB0172CFA4E0B0E0EAE0FBE826
:101610000C944DEC0E945DE569837A838B839C83F7
:10162000CE010196E8DF2496E2E00C9469EC0F937A
:101630001F930E9495CA0091DE061091DF0620914B
:10164000E0063091E1060115110521053105D9F5B6
:1016500020914D132223A1F1E0914B1321502093AF
:101660004D1321E02E0F20934B1330914E13231373
:1016700002C010924B1324E0E29FF0011124E15BC1
:10168000FC4E00811181228133810093DA06109390
:10169000DB062093DC063093DD06600F711F811D91
:1016A000911D6093DE067093DF068093E0069093B1
:1016B000E1068091DC069091DD06892B09F0149AF1
:1016C0001F910F910895601B710B820B930B97FD77
:1016D000F7CF14981092DE061092DF061092E00603
:1016E0001092E106EDCF0F931F93CF93DF938C0100
:1016F000EB0190914D1320914E13921304C097DF8C
:101700000E94616FF6CF80914C1334E0839FF0010B
:101710001124E15BFC4E11830083D383C2839F5F5E
:1017200090934D138F5F281739F080934C13DF91FE
:10173000CF911F910F91089510924C13F8CF8823E9
:1017400051F063E972E084E690E0CDDF6AEB72E08D
:1017500084E690E0C8CF68EB71E084E190E0FACFD6
:10176000C3DA81E0ECCF8F929F92AF92BF92EF925B
:10177000FF920F931F93CF93DF93EC018B01E42E25
:10178000F22E80915F13909160138C179D07C9F121
:101790002FE9CD33D20709F03FC0865F9B4271F439
:1017A0000E9495CA6E517B4F8F4F9F4F6093C0052B
:1017B0007093C1058093C2059093C305D0936013C5
:1017C000C0935F1330E020E000934C0710934D0767
:1017D00020934E0730934F07E0924707F092480757
:1017E000C65FDB4221F410927A041092BF0582E0BA
:1017F0008093670181E080934907109279041092E9
:10180000CB05DF91CF911F910F91FF90EF90BF908B
:10181000AF909F908F9008952BE2C63FD20771F64C
:101820008D539F49D9F40E9495CA8090C00590902D
:10183000C105A090C205B090C305681979098A094D
:101840009B0997FF0BC080915A078770873031F44E
:101850000E945C6AC1EED7E98111B0CFC6EFDBE22E
:10186000ADCF20E040E070E060E08BE49AE67BCF13
:101870000E940FB1882339F020E040E070E060E082
:1018800083E097E970CFEDCF21E020937A04FC014B
:1018900080819181A281B381809331019093320143
:1018A000A0933301B093340120E040E070E060E0A9
:1018B000809136079091370756CFA4E0B0E0E3E679
:1018C000FCE80C944DEC8DEC9CECACECBCE3898317
:1018D0009A83AB83BC83CE010196D6DF2496E2E0E7
:1018E0000C9469ECA4E0B0E0E8E7FCE80C944DEC63
:1018F0008DEC9CECACECBDE389839A83AB83BC8319
:10190000CE010196C1DF2496E2E00C9469ECA4E0DC
:10191000B0E0EDE8FCE80C944DEC80E090E0A0E84D
:10192000BFE389839A83AB83BC83CE010196ACDF8E
:101930002496E2E00C9469ECA4E0B0E0E2EAFCE872
:101940000C944DEC80E090E0A0E2B1E489839A83AE
:10195000AB83BC83CE01019697DF2496E2E00C9422
:1019600069EC81E080937A0480915A078770873010
:1019700051F010925A071092EF0585E29BE1909387
:10198000EB068093EA0680919F048093CD0580E06A
:101990000E94F52920E040E070E060E081ED9CE8E5
:1019A000E2CE80916701882331F041E065EF78E174
:1019B00082E00E9400C58091EF058770873071F446
:1019C0001092CC0520E040E070E060E083E897E909
:1019D000CADE81E08093CB050C94B469089520E0C1
:1019E00040E070E060E086EF9BE2BDCE10928A0797
:1019F0000E94BD6EF4CFCF93DF93C0912D07C7FD3A
:101A00001FC084E0C802E0011124FE01E855FB4F2D
:101A100080819181181619063CF4863F910514F0D7
:101A200085EF90E00E94D6CAC855DB4F8A819B8122
:101A30008F3F910519F010F08FEF90E080938A07A7
:101A4000CEDFDF91CF910895B0E0A0E0EAE2FDE8BB
:101A50000C9447ECCDB6DEB6EDE5F7E0DF010D9076
:101A60000020E9F7CD01855597402DB73EB7281BDB
:101A7000390B0FB6F8943EBF0FBE2DBF0DB71EB782
:101A80000F5F1F4FFF93EF938CE69AE19F938F9325
:101A90001F930F930E94F0E4780134E0E30EF11CF1
:101AA0000F900F900F900F900F900F90D7018D9186
:101AB0007D01882349F0082E000C990B0E94D1EE7D
:101AC000F70131978083F2CF67E67AE1C8010E947F
:101AD00089E44FE350E0B8018CEE96E00E9429EFD4
:101AE0000FB6F894DEBE0FBECDBE79DF0E943BC1BB
:101AF000E8E00C9463EC80932D0720E040E070E078
:101B000060E081EA97E92FCECF93DF93C091BF05C4
:101B1000CC23B1F0C150C093BF0589E0C89FE0015C
:101B20001124C757DA4F6A817B812F814E818881CA
:101B3000998119DE888580937A04DF91CF91089589
:101B40004EDFFBCFA4E0B0E0E8EAFDE80C9441EC06
:101B50000E9414C6F090470785E0782E7F0C85E040
:101B6000E82EEF1884E0D82EDF18AA24AA94B12C0E
:101B700083E0C82ECF1882E0982E9F1881E0882E2F
:101B80008F186F2C6194F11027C080914A07882329
:101B9000A1F080916701882359F081E090914A0774
:101BA000911180E024E046E85BE1662D0E9460C56B
:101BB00080918A0780932D0768C080913107109229
:101BC0003107882331F3A0DF80914907882309F387
:101BD0002496EEE00C945DEC21E0F21276C0809148
:101BE0004A07813009F458C080916701882301F3C6
:101BF00011E080914A07813009F010E060913901CD
:101C000070913A01072E000C880B990B0E945DE53C
